:100000000C942D030C944C030C944C030C944C0353
:100010000C944C030C944C030C944C030C944C0324
:100020000C944C030C944C030C944C030C944C0314
:100030000C944C030C944C030C944C030C944C0304
:100040000C944C030C944C030C944C030C944C03F4
:100050000C944C030C944C030C944C030C944C03E4
:100060000C944C030C94D3890C94018A0C944C038B
:100070000C944C030C944C030C944C030C944C03C4
:100080000C944C030C944C030C944C030C944C03B4
:100090000C94C10B0C944C030C94ED0B0C944C037E
:1000A0000C944C030C944C030C944C030C944C0394
:1000B0000C944C030C944C030C944C030C944C0384
:1000C0000C944C030C944C030C944C030C944C0374
:1000D0000C944C030C944C030C944C030C944C0364
:1000E0000C944C030C94D20C0C94DC0C0C94C80CA7
:1000F0000C94720C0C949D0C0C94E60C0C94470C14
:100100000C94FA0C0C94A5110C94B8110C944C039B
:100110000C944C030C944C030C94040D0C94F00CB4
:100120006E616E00696E6600202065202E2E2E2ED8
:100130002E2E2E20457261736520454550524F4D3D
:100140002C206C6F61642064656661756C7420633B
:100150006F6E66696775726174696F6E0047656E70
:100160006572616C20436F6E6669673A0D0A002004
:1001700020736D63202E2E2E2E2E20536574206D3D
:100180006F646520746F20636F6F7264696E617451
:100190006F720D0A002020736D72202E2E2E2E2ECF
:1001A00020536574206D6F646520746F20726F75C5
:1001B0007465722F656E646E6F64650D0A00202091
:1001C00073633135202E2E2E2E20536574206368E4
:1001D000616E6E656C20746F2069653A2031350D53
:1001E0000A002020737042414444202E2E20536583
:1001F000742050414E494420746F2069653A203084
:1002000078424141440D0A003830322E31352E34C7
:1002100020436F6D6D616E64733A0D0A0020206992
:1002200070202E2E2E2E2E2E205072696E74206677
:10023000756C6C204950204D656E750D0A00495053
:1002400020436F6D6D616E64733A0D0A0020206467
:10025000202E2E2E2E2E2E2E2044756D7020726193
:1002600064696F207265676973746572730D0A0043
:10027000202069202E2E2E2E2E2E2E20496E666FC7
:100280000D0A00446562756767696E673A0D0A007A
:10029000556E6B6E6F776E20277365742720636FC2
:1002A0006D6D616E643F0D0A006E6F646520747938
:1002B0007065206368616E6765642E205265626FA9
:1002C0006F74206E6F77202E2E2E0D0A006E6F64D5
:1002D000652074797065206368616E6765642E209F
:1002E0005265626F6F74206E6F77202E2E2E0D0A6E
:1002F000002C207265736574206E6F646520746FC6
:100300002074616B65206566666563742E0D0A0056
:1003100053657474696E67206368616E6E656C20E6
:10032000746F20000D0A53657474696E6720504124
:100330004E494420746F200003020201010000FFB7
:10034000FEFDFCFBF9F7F4EFA820341D9F1C772776
:1003500000000000C32E00006B2B9C2A000013330A
:1003600000009634282F00002B203B2000000120A5
:100370001A2000000000E31F000000000000411FE1
:10038000931F0000811F311F631F0000221F721F77
:100390000104010101020101010101010101010149
:1003A000040108020101010102010102010201012F
:1003B00002010202010101012201110104010401F3
:1003C00001010108020200011001080848545450BC
:1003D0002F312E3120323030204F4B0D0A536572B1
:1003E0007665723A2041746D656C2F75495076368A
:1003F0000D0A4C6173742D4D6F6469666965643ACA
:10040000205765642C203238204170722032303100
:10041000302032313A32303A313520474D540D0ACE
:10042000455461673A2022366566383537322D34B7
:10043000662D3438353532393337623831633022FE
:100440000D0A4163636570742D52616E6765733A7E
:100450002062797465730D0A436F6E74656E742D36
:100460004C656E6774683A2037390D0A4B656570C4
:100470002D416C6976653A2074696D656F75743DC0
:1004800031352C206D61783D39390D0A436F6E6E20
:10049000656374696F6E3A204B6565702D416C69B8
:1004A00076650D0A436F6E74656E742D54797065B0
:1004B0003A20746578742F68746D6C3B20636861B2
:1004C000727365743D5554462D380D0A0D0A3C482B
:1004D0004541443E0D0A3C5449544C453E736D61C0
:1004E0006C6C3C2F5449544C453E0D0A3C2F4845FA
:1004F00041443E0D0A3C424F44593E5468652048F1
:100500007970657274657874205472616E73663C9C
:100510002F424F44593E0D0A00485454502F312E5B
:100520003120323030204F4B0D0A436F6E74656EB0
:10053000742D547970653A20746578742F68746DE1
:100540006C0D0A0D0A48656C6C6F20576F726C64F5
:100550000D0A0000407A10F35A00A0724E180900EC
:1005600010A5D4E80000E87648170000E40B540218
:100570000000CA9A3B000000E1F505000080969853
:1005800000000040420F000000A0860100000010A3
:100590002700000000E803000000006400000000E5
:1005A000000A00000000000100000000002C76D8C6
:1005B00088DC674F0823DFC1DFAE59E1B1B796E5AC
:1005C000E3E453C63AE651997696E8E6C28426EB10
:1005D000898C9B62ED407C6FFCEFBC9C9F40F2BA23
:1005E000A56FA5F490055A2AF75C936B6CF9676DBB
:1005F000C11BFCE0E40D47FEF520E6B500D0ED9010
:100600002E0300943577050080841E080000204EDC
:100610000A000000C80C333333330F986E12831175
:1006200041EF8D2114893BE65516CFFEE6DB18D14C
:10063000844B381BF77C1D901DA4BBE4242032841E
:10064000725E228100C9F124ECA1E53D2763646953
:100650006E6F70737578585B000011241FBECFEF6A
:10066000D1E4DEBFCDBF16E1A0E0B2E0ECE8FBE6EE
:1006700001E00BBF02C007900D92AC35B107D9F76E
:1006800019E3ACE5B6E101C01D92A731B107E1F76E
:100690000E9430090C94DD640C94000008950895C4
:1006A00008956F927F928F929F92AF92BF92CF9256
:1006B000DF92EF92FF920F931F93DF93CF93CDB70B
:1006C000DEB7EC970FB6F894DEBF0FBECDBF80E06B
:1006D0000E94CF8F00D000D000D0EDB7FEB731968A
:1006E0004E010894811C911CADB7BEB712969C9226
:1006F0008E92119780E092E09383828380918907A4
:1007000090918A07958384830E94A1B1EDB7FEB7CB
:1007100036960FB6F894FEBF0FBEEDBF82E0B4016F
:100720000E943D8A80E197E20E94100E8091161C83
:10073000882319F42EE032E002C022E132E000D03A
:1007400000D000D0EDB7FEB731968E010F5F1F4F7E
:10075000ADB7BEB712961C930E93119785E192E048
:1007600093838283358324830E94A1B1EDB7FEB7C2
:1007700036960FB6F894FEBF0FBEEDBF83E0B4010E
:100780000E943D8AC80162E272E00E945AB0D8011C
:100790000D900020E9F77D010894E108F10880E15F
:1007A00097E20E94100ECC24DD2429E2622E22E082
:1007B000722E58018E01095F1F4F00D000D000D06B
:1007C000EDB7FEB73196ADB7BEB71296FC92EE927A
:1007D000119773826282D601AD51B64D8C9184839C
:1007E00015820E94A1B1E2E0F0E0EE0EFF1E8DB78F
:1007F0009EB706960FB6F8949EBF0FBE8DBF97E0CA
:10080000C91661F4D7011C9284E0B4010E943D8AAC
:10081000C5016EE272E00E945AB078010894C11CD2
:10082000D11CB0E1CB16D10441F6F701108285E06E
:10083000B4010E943D8A8E010F5F1F4FC80165E31E
:1008400072E00E945AB0D8010D900020E9F77D01B6
:100850000894E108F10893EFC92E99E2D92E870197
:1008600089E2A82E82E0B82E00D000D000D0EDB7EB
:10087000FEB73196ADB7BEB712961C930E93119783
:10088000B382A282D6018D916D01848315820E946C
:10089000A1B10E5F1F4FEDB7FEB736960FB6F894B5
:1008A000FEBF0FBEEDBFFBEFCF16F9E2DF06E1F6AC
:1008B000D70150961C9280E197E20E94100E86E0CC
:1008C000B4010E943D8A83E040E452E46FE070E0AE
:1008D00020E030E005E814E0EE24FF240E9424101C
:1008E000EC960FB6F894DEBF0FBECDBFCF91DF916F
:1008F0001F910F91FF90EF90DF90CF90BF90AF903E
:100900009F908F907F906F900895EF92FF920F933A
:100910001F93DF93CF93CDB7DEB7EC970FB6F89464
:10092000DEBF0FBECDBF80E00E945D8D81E00E94E2
:100930005D8D82E00E945D8D80E00E946C8C2DB701
:100940003EB7285030400FB6F8943EBF0FBE2DBFC3
:10095000EDB7FEB731968E010F5F1F4FADB7BEB733
:1009600012961C930E9311972CE332E0338322836B
:1009700064837583868397830E94A1B12DB73EB7A8
:10098000285F3F4F0FB6F8943EBF0FBE2DBF87E0E4
:10099000B8010E943D8A81E00E946C8CADB7BEB761
:1009A00018970FB6F894BEBF0FBEADBFEDB7FEB738
:1009B000319612961C930E93119726E432E03383FE
:1009C000228364837583868397830E94A1B12DB7A8
:1009D0003EB7285F3F4F0FB6F8943EBF0FBE2DBF06
:1009E00088E0B8010E943D8A82E00E946C8CADB71D
:1009F000BEB718970FB6F894BEBF0FBEADBFEDB728
:100A0000FEB7319612961C930E93119720E532E0B3
:100A10003383228364837583868397830E94A1B185
:100A20002DB73EB7285F3F4F0FB6F8943EBF0FBEBD
:100A30002DBF89E0B8010E943D8A83E040E452E482
:100A40006FE070E020E030E001E513E0EE24FF24E9
:100A50000E942410EC960FB6F894DEBF0FBECDBFF7
:100A6000CF91DF911F910F91FF90EF900895AF927A
:100A7000BF92CF92DF92EF92FF920F931F93CF938B
:100A8000DF938AE592E00E946CB1C6E0D6E046E6CC
:100A9000E42E43E0F42E37E6A32E32E0B32EE881B5
:100AA000F981108100D000D000D0EDB7FEB73196AB
:100AB000ADB7BEB71296BC92AE921197F382E282A6
:100AC000148315820E9430B107E08DB79EB7069659
:100AD0000FB6F8949EBF0FBE8DBFC12EDD24C60198
:100AE000002E02C0959587950A94E2F780FD03C019
:100AF00080E390E002C081E390E06091133970914F
:100B000014390E9404B1015050F785E792E00E9429
:100B10006CB12296A0E1B0E0EA0EFB1EB6E0CA3549
:100B2000DB0709F0BCCF85E792E00E946CB1DF9152
:100B3000CF911F910F91FF90EF90DF90CF90BF90DA
:100B4000AF9008952F923F924F925F926F927F9253
:100B50008F92AF92CF92EF92FF920F931F93DF93FA
:100B6000CF93CDB7DEB76D970FB6F894DEBF0FBE4B
:100B7000CDBF80915C1690915D16019790935D16A4
:100B800080935C1601969F70892B11F46A9A629A81
:100B90007894B9EA6B2EB2E07B2EADEC4A2EA2E03F
:100BA0005A2EF0E92F2EF2E03F2E80E090E00E94D6
:100BB000BB0A182F8F3F09F43DC38B3121F0809180
:100BC0005E168823D1F180910C39882329F080E0CA
:100BD00090E00E94F09A2EC380915E16882311F453
:100BE00081E005C0813031F41B3521F582E080932E
:100BF0005E1620C38230F1F410925E16113409F0B3
:100C000019C300D000D086E792E0ADB7BEB7129608
:100C10009C938E9311978FE596E114969C938E93F7
:100C200013970E9430B1109227170F900F900F90DA
:100C30000F9000C310925E16FDC280912717883C6A
:100C400050F46091133970911439812F992787FDE1
:100C500090950E9404B180912717883C08F0EAC261
:100C60001D3019F01A3009F0D0C2E82FF0E0E85D2D
:100C7000F84E1082982F9F5F9093271780910C3920
:100C8000882349F088E297E10E94F09A1092281791
:100C9000109227178ACF809128178936E1F08A367B
:100CA00054F4843609F4D0C0853609F418C28C3463
:100CB00009F01BC200C2823709F4E8C1833724F46B
:100CC0008C3609F012C2E5C1833709F4C0C08437FD
:100CD00009F00BC27AC080912917803729F488E285
:100CE00097E10E94739B7AC200D089E792E0EDB74A
:100CF000FEB7928381830E9430B1ADB7BEB718971B
:100D00000FB6F894BEBF0FBEADBFEDB7FEB73196BC
:100D100080E892E012969C938E9311978091202701
:100D200090912127A0912227B0912327828393833A
:100D3000A483B58380911C2790911D27A0911E2725
:100D4000B0911F2786839783A087B1870E9430B117
:100D50000F900F900F900F90EDB7FEB731968AE984
:100D600092E0ADB7BEB712969C938E931197809187
:100D70008807828313828091890790918A079583DF
:100D800084830E9430B1ADB7BEB716960FB6F89403
:100D9000BEBF0FBEADBF8091640390916503892BE8
:100DA00041F400D086EB92E0EDB7FEB792838183E9
:100DB00009C000D0EAECF2E0ADB7BEB71296FC93E2
:100DC000EE9311970E9430B107C2209189073091AC
:100DD0008A07FE0133968BE0DF011D928A95E9F7C1
:100DE00082E08B833D832C83933048F488E297E143
:100DF00062EE72E00E945AB085E0809327178091DE
:100E000064039091650340912717BE016D5F7F4F8A
:100E1000892B51F485E090E09F838E83415082E0DE
:100E200029E237E100E205C0415082E029E237E1E2
:100E300003E2EE24E394E5E0CE2EAA24A3948824D2
:100E400083940E944D37CAC10E943705C7C1809163
:100E500029178D3609F491C08E3634F48336F1F1BA
:100E60008B3609F003C16EC0803721F0833709F05B
:100E7000FDC0C6C08AE297E10E94A8869A83898352
:100E800000D084E293E0EDB7FEB7928381830E94A5
:100E900042B100D0E7EEF2E0ADB7BEB71296FC93D8
:100EA000EE93119789819A8114969C938E93139750
:100EB0000E9430B10F900F900F900F9080E58E013F
:100EC0000F5F1F4FB8010E94CE3780E50E94883621
:100ED0008EE090E062E070E0A80176C019828AE2BC
:100EE00097E10E94EFAE898380E190E061E070E0DD
:100EF000AE014F5F5F4F0E94130D00D080E193E081
:100F0000ADB7BEB712969C938E9311970E9442B1D3
:100F100000D0EDB7FEB731968EEE92E0ADB7BEB71A
:100F200012969C938E9311978981828313820E94DB
:100F300030B10F900F9081EF92E0EDB7FEB7928342
:100F4000818348C10AE217E16EE0E62EF12CEC0E37
:100F5000FD1EC8010E944886D7018D937D010E5F5A
:100F60001F4FB7E10A341B07A1F784E190E060E16D
:100F700070E0AE01425F5F4F27C080912A17823731
:100F800061F481E090E0909365038093640300D066
:100F9000EDB7FEB7528241820DC08336C1F4109284
:100FA00065031092640300D0ADB7BEB712967C9271
:100FB0006E9211970E9442B10F900F9081E190E0E4
:100FC00062E070E044E653E00E94130D07C10AE2BC
:100FD00017E153EFE52E59E2F52EC8010E9448862D
:100FE000F70181937F010E5F1F4FF7E10A331F075F
:100FF000A1F784E290E068E070E043EF59E2E4CFCB
:1010000080912A17813321F581E08093161C8DE5AC
:1010100066E17CE10E94CE3787E766E17CE10E94D1
:10102000CE3780E866E17CE10E94CE3782E866E157
:101030007CE10E94CE370E94FF370E94FF3781E893
:1010400063EE79E20E94CE3783E863EF79E205C070
:101050001092161C8DE566E17CE10E94CE3783E19B
:1010600090E061E070E046E15CE1AECF00D0ADB76A
:10107000BEB712963C922E9211970E9442B10F90E9
:101080000F9080E090E00E945103A8C00E94850468
:10109000A5C04EB120912917332727FD3095205345
:1010A000304081E090E002C0880F991F2A95E2F756
:1010B0008C71842B12C04EB120912917332727FD44
:1010C00030952053304081E090E002C0880F991F96
:1010D0002A95E2F78C71809584238EB97FC08EE4C7
:1010E00090E06FEF0E942DB579C000D083E892E0C8
:1010F000EDB7FEB7928381830E9442B1E0E7F2E050
:10110000ADB7BEB71296FC93EE9311970E9442B111
:10111000EDE4F2E0ADB7BEB71296FC93EE931197F3
:101120000E9442B1EEE3F2E0ADB7BEB71296FC9377
:10113000EE9311970E9442B1EDE1F2E0ADB7BEB778
:101140001296FC93EE9311970E9442B1E8E0F2E010
:10115000ADB7BEB71296FC93EE9311970E9442B1C1
:10116000E2EEF1E0ADB7BEB71296FC93EE931197A5
:101170000E9442B1EEEBF1E0ADB7BEB71296FC9320
:10118000EE9311970E9442B1E5E9F1E0ADB7BEB729
:101190001296FC93EE9311970E9442B1EFE6F1E0B4
:1011A000ADB7BEB71296FC93EE9311970E9442B171
:1011B000EDE5F1E0ADB7BEB71296FC93EE93119753
:1011C0000E9442B1E8E2F1E0ADB7BEB71296FC93DF
:1011D000EE9311970E9442B10F900F901092281732
:1011E0001092271780910C39882309F0DECC00D0AB
:1011F000E1EFF2E0ADB7BEB71296FC93EE93119714
:101200000E9430B10F900F90D0CC183051F4882349
:1012100009F4CBCCE82FF0E0E85DF84E1082815065
:1012200006C0E82FF0E0E85DF84E10838F5F8093F2
:101230002717BBCC6D960FB6F894DEBF0FBECDBF9F
:10124000CF91DF911F910F91FF90EF90CF90AF90D2
:101250008F907F906F905F904F903F902F90089568
:101260000F931F93DF93CF93CDB7DEB728970FB6B9
:10127000F894DEBF0FBECDBF0E941538882311F051
:101280000E940E0D0E94CD11789481E00E942C0CDA
:10129000882311F00E940E0D0E94CE888AB1806DC5
:1012A0008AB98BB1806C8BB95C988CE364E070E098
:1012B00048EF52E00E942F8980E395E70E94100ECC
:1012C00080E395E70E94100E80E395E70E94100EE0
:1012D0000E94528B8DEE9AE064ED7AE00E94B8B0E5
:1012E00000D000D000D0EDB7FEB731968DEF92E080
:1012F000ADB7BEB712969C938E9311978FE193E092
:10130000938382838BE293E0958384830E9430B140
:10131000EDB7FEB736960FB6F894FEBF0FBEEDBF21
:101320008EE490E00E9425B5893A09F069C084E313
:1013300093E00E946CB180E090E060E170E041E0F9
:1013400050E028E837E00E94450D80E090E061E140
:1013500070E042E050E024E633E00E94450D80E07A
:1013600090E06EE070E042E050E029E837E00E9453
:10137000450D80E090E068E070E046E050E025E256
:1013800037E20E94450D80E090E063E170E041E0CB
:1013900050E026E13CE10E94450D80E090E064E1F0
:1013A00070E040E150E023EE39E20E94450D80E01C
:1013B00090E064E270E048E050E023EF39E20E9400
:1013C000450D80E090E06CE470E042E050E026E8FB
:1013D00037E00E94450D80E090E06CE370E040E172
:1013E00050E029E538E00E94450D80E090E06CE295
:1013F00070E040E150E029E638E00E94450D89C0E8
:1014000082E493E00E946CB198E190938807809108
:101410002427882399F49093252780EF809326270B
:101420008FE98093272785EE809328270E94DFAEDF
:10143000809329270E94DFAE80932A278E010F5FB9
:101440001F4F88E0D8011D928A95E9F781E08983D2
:1014500082E08A8383E08B8384E08C8385E08D83C4
:1014600086E08E8387E08F8381E090E060E070E02B
:1014700048E050E098010E94450D80E090E068E06F
:1014800070E0A8010E94130D80E190E061E070E03F
:1014900048E857E00E94130D81E190E062E070E0BF
:1014A00044E653E00E94130D8EE090E062E070E0AD
:1014B00049E857E00E94130D8CE490E062E070E090
:1014C00046E857E00E94130D88E090E066E070E087
:1014D00045E257E20E94130D8CE390E060E170E07A
:1014E00049E558E00E94130D8CE290E060E170E065
:1014F00049E658E00E94130D83E190E061E070E05E
:1015000046E15CE10E94130D8EE490E069EA0E94DE
:101510002DB50E94278681E00E94A8368091640341
:1015200090916503892B21F485E297E20E948C85D6
:1015300000D081EF92E0EDB7FEB7928381830E94E5
:1015400030B18EB18C618EB98DB18C618DB984B1A1
:101550008F6784B96F9A85B1807885B977988FE75E
:1015600085B9779A0F900F900E94FF370E94A205CD
:101570000E94528BF9CFDF93CF930F92CDB7DEB796
:1015800081E0BE016F5F7F4F41E00E941A0C813005
:1015900019F02FEF3FEF03C08981282F30E0C901F8
:1015A0000F90CF91DF9108950F931F93DF93CF9307
:1015B0000F92CDB7DEB78E010F5F1F4F81E0B801EC
:1015C00041E00E941A0C8823C9F3898190E00F90B2
:1015D000CF91DF911F910F9108950F931F93DF9388
:1015E000CF930F92CDB7DEB789838A3071F48DE047
:1015F00089838E010F5F1F4F81E0B80141E00E9497
:10160000230C8823C9F38AE089838E010F5F1F4F63
:1016100081E0B80141E00E94230C8823C9F380E0F7
:1016200090E00F90CF91DF911F910F9108959B0152
:10163000AC016050774F824C9F4FF2E0660F771FEE
:10164000881F991FFA95D1F7E3E0220F331F441F3B
:10165000551FEA95D1F70E940BAD215030403093D1
:10166000CD002093CC0082E08093C80086E0809378
:10167000CA0088ED8093C9000895DC018091C900FB
:101680008F7B8093C90020917127809172278217E8
:1016900030F0275F922F981B892F295005C02150C9
:1016A000922F981B892F2F5F482F681708F4462F19
:1016B000342F12C090917227E92FF0E0E35AF84DD1
:1016C0008C918083993019F41092722703C09F5F28
:1016D0009093722731501196332361F780917527CB
:1016E000882351F4E22FF0E0E35AF84D8081809393
:1016F000CE0081E0809375278091C900806480933B
:10170000C900842F0895DC0120917627222311F44B
:1017100080E008958091C9008F778093C9002A30B6
:1017200058F080917427809373278AE080937627FE
:101730006A3020F02AE003C0261708F0262F322F47
:1017400017C0E0917327F0E0E35AF84D82858C933F
:10175000909173279F5F9093732780917627815094
:10176000809376279A3011F4109273271196315096
:10177000332339F78091C90080688093C900822F94
:1017800008951F920F920FB60F920BB60F9211246D
:101790008F939F93EF93FF93909174278091762777
:1017A0008F5F809376278091CE00E92FF0E0E35A97
:1017B000F84D8287993019F41092742703C09F5F07
:1017C00090937427FF91EF919F918F910F900BBE93
:1017D0000F900FBE0F901F9018951F920F920FB68B
:1017E0000F920BB60F9211248F93EF93FF9380917A
:1017F0007127893019F41092712703C08F5F80938D
:101800007127E091712780917227E81739F0F0E095
:10181000E35AF84D80818093CE0002C01092752764
:10182000FF91EF918F910F900BBE0F900FBE0F9015
:101830001F901895813011F080E00895CB01642F3E
:101840000E94830B0895813011F080E00895CB0150
:10185000642F0E943D0B0895813011F085E80895B2
:1018600060E076E980E090E00E94170B80E0089548
:101870009093F1178093F01708959093F317809346
:10188000F21708959093F5178093F41708951F9217
:101890000F920FB60F920BB60F9211242F933F9316
:1018A0004F935F936F937F938F939F93AF93BF9368
:1018B000EF93FF93E091F017F091F1170995FF91E5
:1018C000EF91BF91AF919F918F917F916F915F91B8
:1018D0004F913F912F910F900BBE0F900FBE0F9025
:1018E0001F9018951F920F920FB60F920BB60F9282
:1018F00011242F933F934F935F936F937F938F9315
:101900009F93AF93BF93EF93FF93E091F217F09102
:10191000F3170995FF91EF91BF91AF919F918F912F
:101920007F916F915F914F913F912F910F900BBEDF
:101930000F900FBE0F901F9018951F920F920FB629
:101940000F920BB60F9211242F933F934F935F93F7
:101950006F937F938F939F93AF93BF93EF93FF9377
:10196000E091F417F091F5170995FF91EF91BF9170
:10197000AF919F918F917F916F915F914F913F9127
:101980002F910F900BBE0F900FBE0F901F901895C8
:101990001F920F920FB60F9211240F900FBE0F904F
:1019A0001F9018951F920F920FB60F9211240F904F
:1019B0000FBE0F901F9018951F920F920FB60F92A7
:1019C00011240F900FBE0F901F9018951F920F9229
:1019D0000FB60F9211240F900FBE0F901F90189505
:1019E0001F920F920FB60F9211240F900FBE0F90FF
:1019F0001F9018951F920F920FB60F9211240F90FF
:101A00000FBE0F901F9018951F920F920FB60F9256
:101A100011240F900FBE0F901F9018958FEF9FEF1E
:101A20000E94100EFBCFCF92DF92EF92FF920F93A6
:101A30001F93CF93DF938C017B016A01CB01800F51
:101A4000911F8150904110F085E816C0C0E0D0E0B1
:101A50000FC0C8010E9425B5F601EC0FFD1F608183
:101A6000861719F0C8010E942DB50F5F1F4F2196F0
:101A7000CE15DF0570F380E0DF91CF911F910F91BC
:101A8000FF90EF90DF90CF900895CF92DF92EF928A
:101A9000FF920F931F93CF93DF938B017A0169011C
:101AA0008130910531F4862F642FA9010E94D21153
:101AB0001DC0892B11F088EE19C0CA01860F971F2F
:101AC0008150904110F085E811C0C0E0D0E00AC01C
:101AD000CE01800F911F0E9425B5F601EC0FFD1F6E
:101AE00080832196CE15DF0598F380E0DF91CF91BA
:101AF0001F910F91FF90EF90DF90CF9008950E947B
:101B0000EE0F08950E948A0D0E94CF110E94AB0D26
:101B100080E008959FB7F894E0E0F0E089E08093DA
:101B2000570084919FBF8F70823011F090E001C008
:101B30009FE080E80FB6F894809361009093610075
:101B40000FBE80E18093350180933401809333018F
:101B50008093320108951092F6171092F7178FEFC5
:101B60008093F8178093F9178093FA17EBE7F7E261
:101B70009FEF948311821082399688E2ED31F80745
:101B8000C1F780E28093B60088EA8093DC008FE0A2
:101B90008093F4009093F3009093F2009093F100FF
:101BA00082E08093E0008091DF0082608093DF001C
:101BB00008950895FC018091DE0080FDFCCF209106
:101BC000E100822F2091E200922F2091E300A22FCA
:101BD0002091E400B22F24E0880F991FAA1FBB1F99
:101BE0002A95D1F780839183A283B3830895FC0162
:101BF0002091E900822F2091EA00922F2091EB00A2
:101C0000A22F2091EC00B22F34E0880F991FAA1F59
:101C1000BB1F3A95D1F780839183A283B383089544
:101C2000AC018436910518F060E070E01EC07FB70B
:101C3000F89461E01AC057FD02C09A0102C02FEF6C
:101C40003FE7C901880F991F909581959F4F909309
:101C5000250180932401FABBE0932101D09BFECFA4
:101C6000421B530B1092210102C0F1E0E2E041154A
:101C7000510509F761117FBF089520E090E0FC0154
:101C8000B3E0EE0FFF1FBA95E1F7E80FF91FE9582F
:101C9000F84D84819581892B09F021E0822F0895E8
:101CA000EF92FF920F931F938091F81790E0FC0141
:101CB00013E0EE0FFF1F1A95E1F7E80FF91FE9583F
:101CC000F84DE080F180028113818091F61788231E
:101CD00009F449C01093F8000093F700F092F60061
:101CE000E092F5008091DF0080FD08C081E08093E4
:101CF000E0008091DF0081608093DF002091E100AF
:101D0000822F2091E200922F2091E300A22F2091B8
:101D1000E400B22F9C01AD012F5F3F4F4F4F5F4F4B
:101D2000DA01C9018E259F25A027B1278070907008
:101D3000A070B87F0097A105B10531F4E216F30653
:101D400004071507B0F018C08FEF9FEFAFEFB7E0B3
:101D5000E822F9220A231B2357702E153F0540075E
:101D6000510738F009C08091DF008E7F8093DF003B
:101D700003C081E08093F7171F910F91FF90EF90C0
:101D800008951F931FB7F8948091F717882309F4DB
:101D90004CC01092F7173091F617332309F445C061
:101DA0008091F9178F3F59F48091FA178F3F39F4DA
:101DB0008091F8178093FA178093F91712C0209139
:101DC000F8178091FA1790E0FC0153E0EE0FFF1F27
:101DD0005A95E1F7E80FF91FE958F84D208720934D
:101DE000FA178091F81790E0FC0143E0EE0FFF1F17
:101DF0004A95E1F7E80FF91FE958F84D808580937F
:101E0000F8178091FA1790E0FC0123E0EE0FFF1F16
:101E10002A95E1F7E80FF91FE958F84D8FEF808711
:101E200031503093F6170E94500E1FBF1F91089536
:101E3000FF920F931F93182F823110F08AE8C5C0CC
:101E4000FFB6F8940E94C10E0091F617002309F422
:101E5000C0C04091F817242F842F302F1217F1F5AE
:101E6000212F30E0141781F4F901A3E0EE0FFF1FDA
:101E7000AA95E1F7E20FF31FE958F84D80858093AA
:101E8000F8170E94500E18C090E0DC01E3E0AA0FA2
:101E9000BB1FEA95E1F7A80FB91FA958B84DF90182
:101EA00073E0EE0FFF1F7A95E1F7E20FF31FE95899
:101EB000F84D808518968C93812F90E0FC0163E0AB
:101EC000EE0FFF1F6A95E1F7E80FF91FE958F84D8B
:101ED0008FEF808701500093F61762C0822F90E049
:101EE000FC0153E0EE0FFF1F5A95E1F7E80FF91FD1
:101EF000E958F84D50853150822F09F46AC0252FDA
:101F0000ADCF1217D1F52091FA171317B1F41217AC
:101F100021F48FEF8093FA170DC0812F90E0FC0120
:101F200043E0EE0FFF1F4A95E1F7E80FF91FE9586C
:101F3000F84D80858093F91733C0842F90E0DC0141
:101F400033E0AA0FBB1F3A95E1F7A80FB91FA958B4
:101F5000B84D812F90E0FC0103E0EE0FFF1F0A95C2
:101F6000E1F7E80FF91FE958F84D808518968C9332
:101F70001217B1F44093FA1713C0822F90E0FC01BE
:101F800073E0EE0FFF1F7A95E1F7E80FF91FE958AC
:101F9000F84D422F20852F3F09F0B3CF80E00FC0CE
:101FA000812F90E0FC0163E0EE0FFF1F6A95E1F7DF
:101FB000E80FF91FE958F84D1582148281E0FFBE41
:101FC000882311F489E801C080E01F910F91FF90F0
:101FD00008953091F917232F432FDDCF1F930E94CF
:101FE000C10E1FEF25C06FB7F894822F90E0FC015F
:101FF000B3E0EE0FFF1FBA95E1F7E80FF91FE958BC
:10200000F84D2085448155818681978110871582FE
:102010001482178216822F3F09F43FEF6FBF4115DC
:10202000510551F03093FA172093F917FA010995E9
:102030003091FA172091F9172F3FA9F63093FA172C
:102040002093F9171F9108952F923F924F925F921C
:102050006F927F928F929F92AF92BF92CF92DF92B8
:10206000EF92FF920F931F93DF93CF9300D000D096
:102070000F92CDB7DEB7582E1801FB82EA8201E13C
:10208000081710F48AE820C12114310409F419C199
:1020900090E09D838C83FC01A3E0EE0FFF1FAA95C7
:1020A000E1F7E80FF91FE958F84D84819581892BF4
:1020B00011F088E809C1E4E0769567955795479552
:1020C000EA95D1F72115310529F02130310509F0C4
:1020D000F8C026C0DB01CA010897A109B109885FD1
:1020E0009F4FAF4FB74008F0EEC02091E100822F24
:1020F0002091E200922F2091E300A22F2091E40092
:10210000B22F7A018B01E80EF91E0A1F1B1F8FEFF9
:102110009FEFAFEFBFE0E822F9220A231B2320C084
:102120002091E100822F2091E200922F2091E30084
:10213000A22F2091E400B22F8A019B01081B190BEA
:102140002A0B3B0BD901C801BF700897A109B1093F
:10215000885F9F4FAF4FB74008F0B5C07A018B0141
:102160002FB72983F8946FEF862E6FEF962E6FEFBF
:10217000A62E6FE0B62E8E209F20A022B1220E94B4
:10218000C10E6090F8173FEF631671F04090F6179C
:10219000C62CD62C77248FEF9FEFAFEFB7E0E82265
:1021A000F9220A231B2367C05092F817EC81FD81A6
:1021B00053E0EE0FFF1F5A95E1F7AC81BD81EA0FA6
:1021C000FB1FE958F84D60865AC0BFEFDB1609F4D3
:1021D0004DC06D2D70E0FB0143E0EE0FFF1F4A95EF
:1021E000E1F7E60FF71FE958F84D20813181428170
:1021F0005381D501C40182279327A427B527807076
:102200009070A070B87F0097A105B10539F428152A
:1022100039054A055B0508F46FC007C05770E21620
:10222000F3060407150708F467C0EC81FD8133E06D
:10223000EE0FFF1F3A95E1F70C811D81E00FF11FB2
:10224000E958F84DD0866D1419F45092F81717C05C
:102250008C2D90E0FC0123E0EE0FFF1F2A95E1F7A3
:10226000E80FF91FE958F84D508609C08FEFDC2CB4
:102270007394CD2CD82E741408F4A7CF49C0EC81E8
:10228000FD8193E0EE0FFF1F9A95E1F72C813D81D0
:10229000E20FF31FE958F84D80829182A282B38247
:1022A000358224828A819B81978386838091F61769
:1022B0008F5F8093F6170E94500E99819FBF80E038
:1022C00003C088EE01C08BE80F900F900F900F9025
:1022D0000F90CF91DF911F910F91FF90EF90DF90C2
:1022E000CF90BF90AF909F908F907F906F905F90B6
:1022F0004F903F902F900895FB0183E0EE0FFF1F5A
:102300008A95E1F7E60FF71FE958F84D8085B0CFC1
:102310008C2D90E0FC0103E0EE0FFF1F0A95E1F722
:10232000E80FF91FE958F84D5086EC81FD8113E064
:10233000EE0FFF1F1A95E1F7AC81BD81EA0FFB1F7D
:10234000E958F84D8FEF80879ACF1F920F920FB602
:102350000F9211248F938091F617882319F081E052
:102360008093F7178F910F900FBE0F901F901895C5
:102370001F920F920FB60F9211248F938FEF8093BD
:10238000E4008093E3008093E2008093E1008F916A
:102390000F900FBE0F901F90189581E00895A59A99
:1023A0009D9A0895DF93CF93CDB7DEB7C054D04048
:1023B0000FB6F894DEBF0FBECDBFA82FB62F749A0C
:1023C000759A6C9A6D9A5E9A5F9A569A579AA298E5
:1023D0009A9AA5989D9A84B1876084B983E58CBD4B
:1023E000FE0131966E2F93E09E01205C3F4F8E2FB1
:1023F000861BA598000000000000000000000000FF
:1024000000000000000000000000000000000000CC
:10241000000000009EBD0DB407FEFDCF8F778EBD7E
:102420000DB407FEFDCF1EBC0DB407FEFDCF8EB56B
:10243000A59A8083E217F30711F03196D8CF1CBC20
:10244000FE01319620E030E0BE016F5B7F4F81914D
:102450002827022E2295207F2025032E322F229519
:102460002F700226269532272327220F220F220FB4
:102470002025E617F70759F7232B11F085E80CC044
:102480009E012F5F3F4F2A0F311DCA01B9014B2F0B
:1024900050E00E942FB080E0C05CDF4F0FB6F89490
:1024A000DEBF0FBECDBFCF91DF910895BC01009775
:1024B00021F081EC9BE10E948D12089581EC9BE15B
:1024C00060E070E00E942A1308950F931F93CF934A
:1024D000DF9381EC9BE166E00E948512C9EADBE1B3
:1024E0000BEF17E11983088381EC9BE1BE010E9489
:1024F0008D12249603561F4F8BE1C13CD80791F7EC
:10250000DF91CF911F910F910895FC0111821082EC
:1025100013821282158264830895CF93DF93DC01C6
:10252000EB012FB7F89415969C91159714968C9102
:102530001497981711F48CE819C0992321F4119677
:102540007C936E9306C01296ED91FC911397738362
:1025500062831396DC93CE9312971B821A82159690
:102560008C9115978F5F15968C9380E02FBFDF912C
:10257000CF9108959F92AF92BF92CF92DF92EF9248
:10258000FF920F931F93CF93DF938C015B016A013E
:102590009FB6F894DC0115968C91882319F4C0E05D
:1025A000D0E04AC0F801C081D18141155105B1F098
:1025B0007E0111C0D60112966D917C911397ED9119
:1025C000FC91888199810995882359F47E018A813B
:1025D0009B819C01E901209769F72EC0209761F14A
:1025E0007E01AB2849F5F801808191812A813B81E8
:1025F000C817D90719F43183208305C0D701139672
:102600003C932E931297F80182819381C817D907C2
:1026100011F4F382E282D80115968C9115978150BE
:1026200015968C9315978D919C911197892B21F478
:1026300013961C921E9212979FBECE01DF91CF91EE
:102640001F910F91FF90EF90DF90CF90BF90AF90D0
:102650009F900895AB0160E070E00E94BA12089567
:10266000AB0161E070E00E94BA120895CF93DF934E
:10267000EC010BC0CE0160E070E00E942A130097CD
:1026800011F41D8205C00E9456128D81882391F796
:10269000DF91CF9108950F931F93DF93CF93CDB721
:1026A000DEB728970FB6F894DEBF0FBECDBF80917E
:1026B00041018F71883029F581E080934F0189E0D5
:1026C00080934201CE0101960E94DA0D8E010B5FCC
:1026D0001F4F80914F0180FD14C0C8010E94DA0D88
:1026E0008D819E81AF81B88529813A814B815C8142
:1026F000821B930BA40BB50B8D3D9105A105B10574
:1027000040F328960FB6F894DEBF0FBECDBFCF9131
:10271000DF911F910F910895CF93DF93EC0180918A
:102720003A2890913B280F9709F033C080913901E6
:102730008D7F8093390194E6809141018F718830BB
:10274000C9F0915031F48091390182608093390150
:10275000EDCF0000000000000000000000000000BD
:102760000000000000000000000000000000000069
:102770000000E2CFC830D10519F0C330D10549F4CB
:1027800088E090E090933B2880933A2828E030E05E
:10279000E1C18091410190E08F71907090933B284E
:1027A00080933A28C830D10509F44FC0C930D1050B
:1027B00060F4C430D10509F49AC0C630D10509F4DB
:1027C000A3C0239709F0B9C157C0CF30D10579F024
:1027D000C031D10520F4299709F0AFC164C0C631DA
:1027E000D10509F4CBC0699709F0A7C136C183E0D0
:1027F000809342010E94DFAE80936D0180916E0153
:102800009770887F982B90936E0100000000000065
:1028100000000000000000000000000000000000B8
:10282000000000000000000000008091390182607B
:102830008093390183E290E00E94100ED0933B28F0
:10284000C0933A282FE030E085C1089709F475C19C
:1028500088E08093420100000000000000000000BA
:102860000000000000000000000000000000000068
:1028700000000000000061C1089709F45EC183E018
:1028800080934201000000000000000000000000F2
:102890000000000000000000000000000000000038
:1028A000000000004AC18830910539F18930910556
:1028B00020F4069709F041C106C08631910519F050
:1028C000499709F03AC189E0809342010000000075
:1028D00000000000000000000000000000000000F8
:1028E00000000000000000000000000026C1883049
:1028F000910519F0099721F420C10E944B131DC1C5
:1029000084E08093420119C18930910569F08A30D1
:10291000910520F4089709F010C11AC0863191057D
:1029200019F0499709F009C186E08093420100003F
:102930000000000000000000000000000000000097
:102940000000000000000000000000000000F5C0D2
:102950000E944B1386E080934201000000000000BB
:102960000000000000000000000000000000000067
:1029700000000000000000000000DFC0883091056A
:1029800009F18930910520F4069709F0D6C030C0CE
:102990008930910519F0499709F0CFC086E18093FD
:1029A00042010000000000000000000000000000E4
:1029B0000000000000000000000000000000000017
:1029C0000000BBC00E944B1386E1809342010000CF
:1029D00000000000000000000000000000000000F7
:1029E0000000000000000000000000000000A5C082
:1029F00089E0809342010000000000000000000018
:102A000000000000000000000000000000000000C6
:102A100000000000000080914101282F30E02F715C
:102A2000307030933B2820933A282930310509F043
:102A300091C086E180934201000000000000000088
:102A40000000000000000000000000000000000086
:102A5000000000000000000070C08830910509F4FB
:102A600057C08930910520F4069709F066C01BC055
:102A70008930910521F0469709F05FC014C089E1C3
:102A800080934201000000000000000000000000F0
:102A90000000000000000000000000000000000036
:102AA000000000004AC089E080934201000000005D
:102AB0000000000000000000000000000000000016
:102AC00000000000000000000000000080914101B3
:102AD000282F30E02F71307030933B2820933A2814
:102AE0002930310509F036C089E1809342010000A8
:102AF00000000000000000000000000000000000D6
:102B0000000000000000000000000000000015C0F0
:102B10000E944B1389E180934201000000000000F5
:102B200000000000000000000000000000000000A5
:102B30000000000000000000000080914101282FEB
:102B400030E02F7130702F313105B9F320933A28DE
:102B500030933B28C901DF91CF9108958091C71B25
:102B60009091C81B892BA9F48DE90E945E12909365
:102B7000C81B8093C71B892B61F080912A2888236A
:102B800041F080914428882321F486E190E00E945E
:102B90008C1380913028882351F08BE298E260E01A
:102BA00070E00E942A13009711F00E94E0158091B6
:102BB0004428882321F0823011F40E942B170895B5
:102BC000EF92FF920F931F93CF93DF937C01DC0171
:102BD0000D911C91D8011696ED91FC91179780816B
:102BE00080933D28C82FD0E02196CE0FDF1F98811B
:102BF00029812D3310F02CE303C0222309F421E0B6
:102C000092959695969593708FEF989FC001112499
:102C100030E0FC01E29FC001E39F900DF29F900D18
:102C2000112464EB70E00E94E4AC6F3F710511F079
:102C300008F06FEF6883D8011296FC92EE9211971C
:102C4000C8010E949C20DF91CF911F910F91FF90AE
:102C5000EF900895CF92DF92EF92FF920F931F9320
:102C6000CF93DF93E091C71BF091C81BC081D18146
:102C7000C0904701D0907B01D7FC34C082E0D80ED1
:102C80000DE910E00D191109EEEFDE0E0C0F1D1FFE
:102C9000ED2CFF2497012F5F3F4FC80160E871E0E2
:102CA000A9010E942FB0F801D292FF83EE83EE0EAD
:102CB000FF1EF701C2826091C71B7091C81B8BE297
:102CC00098E20E948D128DE90E945E129093C81BBB
:102CD0008093C71B892B31F489E08093420181E006
:102CE00080932A28DF91CF911F910F91FF90EF9051
:102CF000DF90CF900895809144288823F1F080914F
:102D000042018295869587708093C91B1092CA1BD9
:102D100082E0809344288091C71B9091C81B892B27
:102D200041F489E090E00E948C1381E080932A288E
:102D3000089586E190E00E948C130895FF920F930E
:102D40001F93CF93DF93EC018B01442349F09091C3
:102D50006C01809139288295807F9F70892B03C0F8
:102D600080916C018F7080936C010230110598F492
:102D7000442369F090916C0180913128880F8E7006
:102D8000917F892B80936C0110926F0117C0809105
:102D90006C018E6011C0809135288295807F909162
:102DA0003828892B80936F0190916C018091312894
:102DB000880F8E70917F892B80936C0189E190E060
:102DC0000E948C134997D1F7FFB6F8940130110592
:102DD00059F480913D28833118F080E492E002C0DC
:102DE00080E890E00E94100E80913901826080930B
:102DF0003901809139018D7F80933901288130E03C
:102E00002150304080E891E0BE01A9010E942FB01E
:102E100081E080934428FFBEDF91CF911F910F91F5
:102E2000FF900895FC0180914428882311F086E8E2
:102E30000895F0933728E093362886819781909300
:102E40003F2880933E28009711F488EE08950E9451
:102E50009E1680E00895109244288091C91B90919D
:102E6000CA1B83309105B9F08430910528F400978E
:102E700031F00197E1F409C00597C9F412C06091DF
:102E800036287091372880E017C0609136287091FD
:102E9000372887E811C0609136287091372881EE75
:102EA0000BC0609136287091372889EE05C060917B
:102EB00036287091372885E80E9424310895282FFC
:102EC00085FD03C0982F9F7304C0982F91959F7123
:102ED0009195E8E3F3E08491891734F03F9684916B
:102EE000981714F0822F0CC0803E3CF080323CF4E6
:102EF00087FF06C08F71806203C080E201C08FE14E
:102F00008068089584E08093312823E02093382856
:102F10008FEF9FEF90932628809325289093292860
:102F2000809328288BE0809333281092242880E017
:102F300098EFAFEFB7E08093402890934128A0939B
:102F40004228B09343288AE091E09093232880930D
:102F500022288AE080933C2882E08093322885E012
:102F6000809335282093392883E80E945F17809347
:102F7000192881E08093272810923428089585FD30
:102F800003C0982F9F7304C0982F91959F719195BE
:102F9000E8E3F3E080E02491921724F029173CF451
:102FA000815008958F5F31968031A9F780E00895B0
:102FB0008091252890912628809362019093630147
:102FC000EAE1F8E2A4E6B1E081918D9388E2E23291
:102FD000F807D1F7809128289091292880936001E3
:102FE0009093610190914801809127288295880FE4
:102FF00080769F79892B8093480190916F01809111
:1030000038288F70907F892B80936F0190916E018B
:1030100080913428880F880F880F8870977F892BBC
:1030200080936E0190916F01809135288295807F09
:103030009F70892B80936F01909148018091332874
:103040008F71907E892B80934801809119280E946E
:10305000BF17909145018F70907F892B8093450118
:103060000895CF93DF93EB018E3431F0893541F42D
:10307000888180933928EFC0888180933128EBC004
:1030800020913A2830913B282F30310511F481E806
:10309000E3C08B3009F4CDC08C3070F4823009F479
:1030A00087C0833018F48823B1F115C0833009F448
:1030B00090C0843081F466C0833511F1843528F4E2
:1030C0008F3459F0803539F410C0873509F464C065
:1030D000803F09F48BC084EFBFC09881909338285B
:1030E00080916F019F70807F5FC0888199818093FC
:1030F0002528909326288093620190936301ABC0AA
:103100008881998180932828909329288093600151
:1031100090936101A0C080914428882309F097C052
:1031200080E098EFAFEFB7E0088004C0B695A795B0
:10313000979587950A94D2F781709070892B09F43E
:1031400088C02830310519F428E030E008C088E054
:1031500090E00E948C130897D1F726E130E0988127
:1031600090933328809148019F71807E982B909393
:1031700048012830310509F46EC086E190E00E94D4
:103180008C1369C080914428882309F060C088812D
:10319000882309F460C05DC09881909335288091A0
:1031A0006F019295907F8F70982B90936F0153C011
:1031B0008881809319280E945F17809319280E94A4
:1031C000BF17909145018F70907F892B80934501A7
:1031D00042C0888180932728909148018295880F6A
:1031E00080769F79892B8093480135C088818093B0
:1031F0001A28898180931B288A8180931C288B81BF
:1032000080931D288C8180931E288D8180931F2898
:103210008E81809320288F8180932128EAE1F8E233
:10322000A4E6B1E081918D9388E2E232F807D1F70C
:1032300012C088818093342890916E01880F880F86
:10324000880F8870977F892B80936E0104C086E871
:1032500003C088EE01C080E0DF91CF910895DF9335
:10326000CF930F92CDB7DEB781E090E065E170E0DB
:1032700041E050E09E012F5F3F4F0E94450D80913D
:1032800039018D7F8093390180EF90E00E94100E0C
:10329000809139018E7F8093390181E090E00E9416
:1032A000100E8091390181608093390120E030E077
:1032B000809141012F5F3F4F93E0293E390711F480
:1032C00085E815C090E08F7190708830910581F786
:1032D00090933B2880933A289981992339F08091E3
:1032E00052019F70807F982B9093520180E00F9045
:1032F000CF91DF9108950E94DFAE80936D01EEE6DD
:10330000F1E080819770887F982B908380E00E9405
:10331000121B0E94001B0895882311F00E9482173F
:103320000E942F19882311F085E8089580916E017D
:10333000806280936E018CE480934E010E947B1921
:1033400080913028882359F40EC08BE298E260E027
:1033500070E00E942A13009711F00E94561280918B
:103360003028882391F70E94D81710924428109291
:103370002A2888E080934F0180E480934F0184E005
:1033800080934F010E941D3880E008950F931F9392
:10339000CF93DF930E94820D882309F00CC18091A6
:1033A0003901816080933901809139018D7F80934B
:1033B00039018CE791E00E94100E809139018E7FD7
:1033C0008093390181E090E00E94100E80913901D4
:1033D00081608093390188E08093420120E08091F0
:1033E0004101215009F4E7C090E08F71907088305E
:1033F0009105A9F790933B2880933A2880915C012E
:10340000833809F0D8C0DDC080916E01806280935E
:103410006E018CE480934E0186E090E00E948C1354
:1034200010924E01C0E0D0E010E080914601CC0F38
:10343000DD1FCC0FDD1F90E08076907025E0969523
:1034400087952A95E1F7C82BD92B1F5F183069F7AC
:1034500083E090E00E948C1380914F0110934F0104
:1034600080E480934F018CE480934E01CE010E9452
:10347000E4AE0E947B1909C0CAE1D8E20E94DFAE27
:10348000899388E2C232D807C9F780911A2830910F
:103490001B2840911C2860911D2870911E28F091D6
:1034A0001F28B091202850912128082F015091E029
:1034B000081708F090E0832F815021E0831708F06F
:1034C00020E0192F180F91E0181708F090E0292B31
:1034D000842F815031E0841708F030E0A22FA80F2C
:1034E00091E0A81708F090E0392B862F815021E059
:1034F000861708F020E0E32FE80F91E0E81708F0C6
:1035000090E0292B872F815031E0871708F030E0B9
:10351000622F680F91E0681708F090E0392B8F2F29
:10352000815021E08F1708F020E0432F480F91E0F1
:10353000481708F090E0292B8B2F815091E08B17D2
:1035400008F090E0322F380F21E0381708F020E023
:10355000922B5195591779F43F3F69F44F3F59F435
:103560006F3F49F4EF3F39F4AF3F29F41F3F19F49F
:103570000E3F08F081CF88EF9AE10E943D0C80EF6A
:103580009AE10E94380C0E9465128DE90E945E1239
:103590009093C81B8093C71B8BE298E265E00E9462
:1035A00085120E9482170E94D81710924428109208
:1035B0002A2880E001C085E8DF91CF911F910F910B
:1035C000089580E090E060E070E048E050E02AE19B
:1035D00038E20E94450D0E942F19882361F714CF0D
:1035E0001F931FB7F8940E947B161FBF1F91089569
:1035F0001F931FB7F8940E942A161FBF1F910895AA
:1036000080913A2890913B280F9711F082E8089515
:1036100088E090E00E948C13089711F085E80895E7
:1036200080E00895882311F088EE089580913A286B
:1036300090913B280F9711F481E8089580914428D8
:10364000882391F410922A2888E090E00E948C133D
:103650000897D1F78FE090E00E948C130F9721F428
:103660000E941D3880E0089586E80895982F809183
:103670004428882311F086E80895983041F488E0C2
:1036800090E00E948C1310922A2888E0089580917F
:10369000C71B9091C81B892B31F086E190E00E94F6
:1036A0008C1386E0089581E080932A2886E00895AF
:1036B000CF93DF93DC019C9111962C91119780910F
:1036C0004528882321F4CD010E9456121AC0E92F03
:1036D000F22F9F012F5F3F4F48E059E288E0EA0157
:1036E0000990AE01E90109929E018150C1F78091D4
:1036F0001A29818783E180838EE699E2BD010E94C9
:103700008D12DF91CF910895DC01ED91FC9111971D
:1037100084E180836383528341838EE699E2BD0115
:103720000E948D1208950F931F93DF93CF9300D0C3
:10373000CDB7DEB7A091A828B091A928ED91FC9152
:10374000119784E180838BEE83830FEF1FEF128349
:1037500001838EE699E2BD010E948D121092962897
:103760001A83098380E5BE016F5F7F4F0E944F2B54
:103770001093DF280093DE281092ED281092EE2897
:103780001092EF281092F0281092F1281092F2284F
:103790001092F3281092F4280E9499290F900F900C
:1037A000CF91DF911F910F910895EF92FF920F93A8
:1037B0001F93E090E928F090EA2880E061E040E083
:1037C00020E030E000E010E00E94C6238823A9F446
:1037D000A091A828B091A928ED91FC91119784E1BE
:1037E000808381EE83838FEF9FEF928381838EE6C8
:1037F00099E2BD010E948D1219C0A70160E070E03E
:1038000084E0440F551F661F771F8A95D1F780E02B
:1038100020E030E003E91BE1EE24FF240E942410A5
:10382000882321F080E090E00E94931B1F910F916C
:10383000FF90EF900895FF920F931F93DF93CF9324
:1038400000D0CDB7DEB7F0901C290E945612FF20A1
:10385000B1F583E56AE179E20E944F2B20911A29A4
:1038600030911B29809108298093ED2880910929A6
:103870008093EE2880910A298093EF2880910B296C
:103880008093F02880910C298093F12880910D2954
:103890008093F22880910E298093F32880910F293C
:1038A0008093F42881E080932429109296288091B7
:1038B000A228833031F582E08093A22822C01092A2
:1038C00096280FEF1FEF1A83098380E5BE016F5F13
:1038D0007F4F0E944F2B1093DF280093DE28109219
:1038E000ED281092EE281092EF281092F0281092F6
:1038F000F1281092F2281092F3281092F4282FEF5A
:103900003FEFE091A828F091A928A081B18184E13E
:103910008C931396FC92139712963C932E931197C7
:103920008EE699E2BF010E948D120E9499290F90A4
:103930000F90CF91DF911F910F91FF900895CF923B
:10394000DF92EF92FF920F931F93DF93CF93CDB748
:10395000DEB72C970FB6F894DEBF0FBECDBFD82EC2
:10396000C92E082F192FDE011196F801808191814F
:103970009C01F9018CE001900D928150E1F7D80192
:10398000ED90FC90809124298250823020F0C80173
:103990000E9456125AC082E0F7018083D701A956CF
:1039A000BF4FFD0181938A859B8512969C938E93D0
:1039B00011978C8582839D0128503040D901EAE11E
:1039C000F8E288E001900D928150E1F7F901389713
:1039D0009F01AE014E5F5F4F88E0DA010D90AD01AF
:1039E000D9010D929D018150C1F7809125289091B8
:1039F0002628929382938091A32882938F5F80934D
:103A0000A32883E69CEC929382938BE18293D70167
:103A10001796FC93EE93169787E498E2B8010E94FC
:103A20008D128C3829F481EFB8010E94A4290DC0B1
:103A30008D2D9C2D0E94052981E00E943D0E88233A
:103A400011F40E943026F70114822C960FB6F894D8
:103A5000DEBF0FBECDBFCF91DF911F910F91FF90C1
:103A6000EF90DF90CF900895EF92FF920F931F9306
:103A7000DF93CF93CDB7DEB72F970FB6F894DEBFA5
:103A80000FBECDBFAC018C01DE011196FC0180811F
:103A900091819C01F9018FE001900D928150E1F735
:103AA0004093A8285093A9288C81823019F48F81E3
:103AB00098851AC08F818093ED2888858093EE28A1
:103AC00089858093EF288A858093F0288B85809361
:103AD000F1288C858093F2288D858093F3288E853C
:103AE0008093F4288EEF9FEF9093DF288093DE2859
:103AF00080E5BE016B5F7F4F0E944F2B80916C2948
:103B0000813011F40E947429D801ED90FC9081E07D
:103B1000F701808312830183E756FF4F80838F85EF
:103B200081839F0128503040D901EAE1F8E288E022
:103B300001900D928150E1F7F9018FEF9FEF929381
:103B400082938C81823051F48091DE289091DF281D
:103B50009293829345E123E238EC11C0F9013A9740
:103B60009F014DEE58E288E0DA010D90AD01D901D8
:103B70000D929D018150C1F74BE123E23CEC809115
:103B8000252890912628929382938091A32882934E
:103B90008F5F8093A328329322934293D701179685
:103BA000FC93EE93169780E0BE016E5F7F4F0E94FC
:103BB0004F2B84E0BE016D5F7F4F0E944F2B882307
:103BC00061F4C70162E070E041E00E9412178823AF
:103BD00021F481E08093252912C0D801ED91FC9158
:103BE00084E1808381EE83838FEF9FEF92838183D3
:103BF0008EE699E2B8010E948D120E9499292F96B3
:103C00000FB6F894DEBF0FBECDBFCF91DF911F91ED
:103C10000F91FF90EF900895DC011696ED91FC91C5
:103C2000179782818695869583708330A9F4809159
:103C3000CB1B9091CC1B08979093CC1B8093CB1BF4
:103C4000DC01369688E001900D928150E1F7809179
:103C5000CD1B8F5F8093CD1B80E00895FC01A68172
:103C6000B78112968C9112978695869583708230D3
:103C7000A1F4E091CB1BF091CC1B3297F093CC1BBD
:103C8000E093CB1B16968D919C911797918380831F
:103C90008091CD1B8F5F8093CD1B80E00895AF9204
:103CA000BF92CF92DF92EF92FF920F931F93DF9319
:103CB000CF9300D000D0CDB7DEB7FB01A080B1809C
:103CC000D50112967C936E9311978AE08C937BE9D1
:103CD000C72ED12CCA0CDB1C8091A428882319F490
:103CE0006DE0E62E0EC0482F50E0C41AD50A5DE004
:103CF000E52EE80E2AEA38E2C601B90150E00E943A
:103D00002FB0D092CC1BC092CB1B1092CD1B8EE259
:103D10009EE19A83898387E498E28E010F5F1F4FAB
:103D2000B8010E943013F090CD1B1092CD1B8CE097
:103D30009EE19A83898387E498E2B8010E94301358
:103D40008091CD1BE091CB1BF091CC1B319790E083
:103D50009C0144E0220F331F4A95E1F72F2920836D
:103D6000880F991F880F991F8F0D911D880F991F1C
:103D70008093CD1B4E2D480FE82FF0E0E095F09595
:103D8000EC0DFD1D129280912429833019F42FEF40
:103D90003FE402C02FEF3FE0809145288111306859
:103DA000DF013E932E9380912828909129282FEFB0
:103DB0008E3F920789F43A974A5F9F016AE178E261
:103DC00088E0DB010D90BD01D9010D929D0181506C
:103DD000C1F720E030EC05C0FD019293829320E012
:103DE00030E88091252890912628929382938091A3
:103DF000A12882938F5F8093A128329322934293CC
:103E0000D5011796FC93EE931697C50162E070E01A
:103E100040E00E94121781E0809325290F900F90B7
:103E20000F900F90CF91DF911F910F91FF90EF9026
:103E3000DF90CF90BF90AF900895BC0180E00E94CA
:103E40004F1E08950F931F938C01DC01ED91FC919F
:103E500081810E947E3BC8010E9456121F910F91E2
:103E600008950F931F938C01DC01ED91FC918181EA
:103E700062810E94CC3EC8010E9456121F910F9190
:103E80000895AF92BF92CF92DF92EF920F931F935C
:103E90005C01DC01ED91FC91048115812681378163
:103EA000818162814381E08439966F010E94B13F34
:103EB000C5010E9456121F910F91EF90DF90CF9095
:103EC000BF90AF9008950F931F938C01DC01ED918B
:103ED000FC9181810E94A73EC8010E9456121F9149
:103EE0000F9108950F931F938C01DC01ED91FC91CC
:103EF00081810E94513BC8010E9456121F910F916F
:103F000008950F931F938C01DC01ED91FC91818149
:103F100062813396AF010E942A3FC8010E94561267
:103F20001F910F9108950F931F93DF93CF93CDB7F8
:103F3000DEB766970FB6F894DEBF0FBECDBF8C011B
:103F4000DC01ED91FC91818192819B838A83838145
:103F500089839E012C5F3F4FAF014C5F5F4F88E02C
:103F6000DA010D90AD01D9010D929D018150C1F78B
:103F7000818192819E878D8784858C879E01215FB8
:103F80003F4FAF01435F5F4F88E0DA010D90AD0115
:103F9000D9010D929D018150C1F7CE010196BE015C
:103FA000645F7F4F45890E947C3BC8010E94561286
:103FB00066960FB6F894DEBF0FBECDBFCF91DF91EE
:103FC0001F910F910895CF92DF92EF92FF920F937E
:103FD0006C01DC01ED91FC91BF016E5F7F4F248984
:103FE0003589E788F08C8181438906890E944F3B9F
:103FF000C6010E9456120F91FF90EF90DF90CF9074
:104000000895EF92FF920F937C01DC01ED91FC91FA
:1040100021813281438154816581768187819085B8
:1040200001850E945540C7010E9456120F91FF90D2
:10403000EF9008950F931F938C01DC01ED91FC919B
:104040008181928163810E94903EC8010E94561234
:104050001F910F9108950F931F938C01DC01ED9137
:10406000FC91818162810E94533BC8010E945612DB
:104070001F910F9108956F927F928F92AF92CF927E
:10408000EF920F93DF93CF93CDB7DEB766970FB65E
:10409000F894DEBF0FBECDBF3C01DC01ED91FC9179
:1040A00081818983828193819B838A839E012C5F96
:1040B0003F4FAF014C5F5F4F88E0DA010D90AD01DB
:1040C000D9010D929D018150C1F784858C8785852A
:1040D00096859E878D879E01215F3F4FAF01415F8F
:1040E0005F4F88E0DA010D90AD01D9010D929D017D
:1040F0008150C1F7258D368DCE010196BE01645FDA
:104100007F4F448D0789E08CC18CA28C838C0E94E8
:104110001241C3010E94561266960FB6F894DEBF94
:104120000FBECDBFCF91DF910F91EF90CF90AF90A9
:104130008F907F906F900895FC0110826181728151
:104140006115710521F083EE98E20E948D120895A9
:10415000AF92BF92CF92DF92EF92FF920F931F9395
:10416000DF93CF930F92CDB7DEB77C01FC01A08027
:10417000B180F501A681B7813C913093F828FD010B
:10418000E30FF11D8181809318291196CD90DC9069
:104190001297D092F628C092F52813968C91139717
:1041A0008093F928AD014C5F5F4F7D2D7295769518
:1041B000769573706D2D66956695637019F4FA01A6
:1041C00020E049C014968D919C9115979093FC28FE
:1041D0008093FB28FD0136966230E1F41092FD28B1
:1041E0001092FE281092FF281092002910920129A7
:1041F00010920229109203291092042916968D918B
:104200009C9117979093FE288093FD28FD01389686
:1042100024E021C0633011F022E01DC016968C917D
:1042200016978093FD2881818093FE288281809358
:10423000FF288381809300298481809301298581CF
:1042400080930229868180930329878180930429A2
:10425000FD013E962AE0772309F447C0C6FC08C05A
:104260008191919190930729809306292E5F08C030
:104270008091FB289091FC28909307298093062930
:104280007230C1F4109208291092092910920A295B
:1042900010920B2910920C2910920D2910920E29C0
:1042A00010920F2980819181909309298093082988
:1042B0002E5F1BC07330C9F48081809308298181EF
:1042C00080930929828180930A29838180930B2915
:1042D000848180930C29858180930D298681809328
:1042E0000E29878180930F29285F3550321B309328
:1042F0001929709305296093FA288A01020F111D6C
:104300008C2D87708093F728833021F4F801808109
:10431000809317291982C3FE0DC0F501668177814C
:104320006F5F7F4F85EF98E2A8019E012F5F3F4F9F
:104330000E94399E3091F728313009F461C0313044
:1043400020F0333009F04DC16FC02981F801E20F30
:10435000F11D8081918190931B2980931A29822FCE
:104360008E5F8983F801E80FF11D808180931C29FD
:104370002D5F29832350877019F02C5F280F298324
:104380008981F801E80FF11D908190931D29482F34
:104390004F5F4983292F2770892F90E08077907095
:1043A00034E0959587953A95E1F7382F222311F45B
:1043B0008823A1F0C801840F911D90931F29809339
:1043C0001E29222319F0220F240F2983332331F0D1
:1043D000330F330F330F8981380F398380911929B7
:1043E0009981981750F4891B80932029090F111D7A
:1043F0001093222900932129F8C010922029F5C09A
:1044000080911929882369F0863718F086E7809310
:1044100019298981080F111D10931B2900931A294E
:10442000E4C010921929E1C081E089832091172905
:10443000243009F4DAC0253030F4213059F022302C
:1044400009F0CFC00DC0273009F4CFC0283009F0E3
:10445000C8C012C0F801818180931A2982E02EC061
:10446000F8018181928190931B2980931A293983C5
:10447000838180931C29B9C0F80181819281909336
:104480001B2980931A2939838381948190931D2954
:1044900080931C2985E08983858180931E2986E08D
:1044A0008983868197819093202980931F2929836E
:1044B000D4FE9BC080858093212989E0898395C0A3
:1044C0008091F728833061F480911729843011F0AE
:1044D000873031F483EE98E2B7010E948D128BC0D1
:1044E00080919628813009F467C0813020F08430B3
:1044F00008F077C03AC08091A028882341F59091B8
:104500002429933090F0933009F06BC08091F72804
:10451000813009F462C0833009F063C080911729AB
:104520008430B9F1873079F543C08091F728813024
:1045300009F453C0833009F054C0809117298430A6
:1045400041F1873001F5923009F04BC031C0823023
:1045500019F0843009F045C08091F728882309F0CC
:1045600040C0C7010E94912F46C00E94F72E809143
:10457000F728813091F18330A1F58091172984309B
:1045800041F0873089F0813061F5C7010E94581BE6
:1045900032C080914C28882321F0C7010E948924D1
:1045A0002AC00E946D231DC0809124298230C9F445
:1045B000C7010E941D1F1FC08091F728833059F446
:1045C00080911729823069F480E00E94180FC7019A
:1045D0000E941B1C10C0813021F4C7010E944C2690
:1045E0000AC0C7010E94561206C08091252988235F
:1045F00009F066CF75CF0F90CF91DF911F910F918A
:10460000FF90EF90DF90CF90BF90AF900895CF9341
:10461000DF93DB01EC01EE81FF8182818695869537
:104620008370823011F040E009C040E02D913C9150
:10463000868197812817390709F441E0842FDF919B
:10464000CF910895CF93DF93DB01EC01EE81FF81E1
:104650008281869586958370833011F020E02FC08B
:1046600020E09C918681981751F511969C911197A5
:104670008781981721F512969C911297808598173B
:10468000F1F413969C91139781859817C1F41496B1
:104690009C9114978285981791F415969C91159783
:1046A0008385981761F416969C91169784859817C0
:1046B00031F417969C918585981709F421E0822F93
:1046C000DF91CF910895FB0140E0208131812817CF
:1046D000390709F441E0842F08950F931F93CF9376
:1046E000DF938DE90E945E128C01009709F449C0A6
:1046F000DC014D915C918CE0FA018083128301838F
:10470000E556FF4F80910529833069F43897EF0112
:10471000A8E0B9E288E00D9009928150E1F76FE0DE
:1047200021E03CE009C080910829909109299293E9
:10473000829369E021E038E0809106299091072971
:10474000929382938091A32882938F5F8093A32872
:10475000329322936293DA011796FC93EE931697A5
:10476000F8018081918161E070E040E00E941217C1
:10477000882321F481E08093252903C0C8010E9489
:104780005612DF91CF911F910F9108956F927F92F2
:104790009F92AF92BF92CF92DF92EF92FF920F93D0
:1047A0001F93CF93DF93D82E962EC42E5901380134
:1047B0008DE90E945E127C01009709F49BC0DC0128
:1047C0000D911C91DD2021F084E0F801808303C06D
:1047D0008BE0D8018C93F801F282E182E656FF4F1C
:1047E00084E080832091282830912928C9010296ED
:1047F000029710F0992069F03897EF01AAE1B8E22A
:1048000088E00D9009928150E1F762E183E290EC3B
:1048100005C0329322936CE083E290E8CC2061F0F3
:1048200020912528309126286216730629F06E5FA4
:104830003293229370E002C0806471E022E0C216DD
:1048400041F4AC015860D5018D919C919293829373
:1048500028C0B3E0CB1661F4AC015C6038976A5FA6
:10486000EF01D50188E00D9009928150E1F719C060
:104870002091DE283091DF284FEF2E3F340729F0BA
:10488000AC015860329322930CC0AC015C60389745
:104890006A5FEF01ADEEB8E288E00D9009928150B9
:1048A000E1F73297772339F08091252890912628D7
:1048B0009183808302C0718260828091A328829359
:1048C0008F5F8093A328529342936293D8011796E7
:1048D000FC93EE931697C80162E070E041E00E94FD
:1048E0001217882321F481E08093252904C0C70191
:1048F0000E94561280E0DF91CF911F910F91FF909F
:10490000EF90DF90CF90BF90AF909F907F906F908F
:104910000895DF92EF92FF920F931F93DF93CF934F
:1049200000D000D0CDB7DEB7109223290E945612D6
:1049300080912429823008F4BDC0809105298230FD
:1049400021F0833009F0B6C003C087E093E202C0D3
:1049500082E293E29A83898388E099E29C838B8345
:1049600087E498E2BE016F5F7F4F0E943013BC0165
:10497000009789F0DC014D915C91DA011696ED917A
:10498000FC91179720910629309107298481958100
:104990002817390719F00E946D238CC081E0FA01B5
:1049A000848380910529823021F0833009F06DC025
:1049B00023C02091082930910929A3E7B8E2149671
:1049C0008C911497882391F0ED91FC9111970190AF
:1049D000F081E02D8481882349F40680F781E02D61
:1049E000868197812817390709F441C01596E8E2B6
:1049F000A639BE0721F749C0D0900829E0900929BF
:104A0000F0900A2900910B2910910C2930910D2961
:104A100020910E2990910F29A3E7B8E214968C916A
:104A20001497882369F1ED91FC9111970190F08121
:104A3000E02D8481882321F50680F781E02D868191
:104A40008D15F1F487818E15D9F480858F15C1F409
:104A500081858017A9F48285811791F48385831756
:104A600079F48485821761F48585891749F4DA0120
:104A70001696ED91FC91179781818061818305C025
:104A80001596E8E2A639BE0749F6DA0114961C929B
:104A9000149712967C936E931197CA0161E070E0AF
:104AA00040E00E941217882329F481E08093252991
:104AB000809323290F900F900F900F90CF91DF914B
:104AC0001F910F91FF90EF90DF900895DC01ED9121
:104AD000FC911197E081E43278F4F0E0EE0FFF1FD3
:104AE000E85BFC4F259134912115310519F0F9014E
:104AF000099508950E94561208951F9380912529C3
:104B0000882381F480919F28882361F08AE998E2C4
:104B100060E070E00E942A13009721F00E94662551
:104B200011E001C010E08091E828882359F083EE5D
:104B300098E260E070E00E942A13009719F00E944A
:104B4000662511E0812F1F910895DC01ED91FC9104
:104B5000119780E18083418362838EE699E2BD01F3
:104B60000E948D1208957F928F929F92AF92BF9272
:104B7000CF92DF92EF92FF920F931F93DF93CF9329
:104B800000D000D0CDB7DEB703E718E293E6892E58
:104B900093E2992E5E010894A11CB11C80E1782E4D
:104BA000D80114968C9114978823C9F112968D918F
:104BB0009C911397019713969C938E931297892B30
:104BC00071F514961C921497ED90FC90F701C0803B
:104BD000D1809A828982FC82EB8287E498E2B501D7
:104BE0000E942A13D6018C91823019F08D30A1F4E5
:104BF00005C080EFB7010E94A4290EC0F601838191
:104C0000D701ED91FC917082818380EF82838EE6E3
:104C100099E2B7010E948D12F801118210820B5F98
:104C20001F4FF8E206391F0709F0BACF0E94282962
:104C300080914C28882311F00E9430260F900F900D
:104C40000F900F90CF91DF911F910F91FF90EF90F8
:104C5000DF90CF90BF90AF909F908F907F900895FE
:104C6000EF92FF920F931F9381E040E050EE61E0DE
:104C700070E020E030E003EB15E2EE24FF240E9418
:104C80002410882321F080E090E00E94B3251F913A
:104C90000F91FF90EF9008950F931F93DF93CF93A1
:104CA000CDB7DEB728970FB6F894DEBF0FBECDBFE5
:104CB000AC01DC019C9111962C91809119298823DB
:104CC00021F4CA010E94561205C1E92FF22F8091EA
:104CD000F928808F80910529818382508230A8F441
:104CE0008091062990910729938382839F012C5FED
:104CF0003F4F68E079E288E0DB010D90BD01D9010A
:104D00000D929D018150C1F70AC013821282148254
:104D10001582168217821086118612861386208DC0
:104D200080914628281761F5948180916928981709
:104D300039F5958180916A28981711F596818091AF
:104D40006B289817E9F4978180916C289817C1F423
:104D5000908580916D28981799F4918580916E289F
:104D6000981771F4928580916F28981749F493856C
:104D700080917028981721F4CA010E94561260C0D1
:104D800020934628848180936928858180936A28AE
:104D9000868180936B28878180936C28808580939F
:104DA0006D28818580936E28828580936F28838506
:104DB000809370288091FA28848782508230A8F4EA
:104DC0008091FB289091FC28968785879F01215F21
:104DD0003F4F6DEF78E288E0DB010D90BD01D90116
:104DE0000D929D018150C1F70AC01686158617865F
:104DF000108A118A128A138A148A158A168A809157
:104E00001829878B809110298770818F80911029B4
:104E10008695869586958370828F80911629838FDB
:104E200080911929848F80911A2990911B29968F3E
:104E3000858F81E180838EE699E2BA010E948D120E
:104E40008091F52884FF46C080912429833009F49D
:104E500043C080910529823071F480910829909196
:104E600009299A838983009106291091072980E0F6
:104E700060E042E021C0833019F5809108298983E0
:104E8000809109298A8380910A298B8380910B293B
:104E90008C8380910C298D8380910D298E83809144
:104EA0000E298F8380910F29888700910629109100
:104EB000072980E060E043E09E012F5F3F4F07C07D
:104EC00080E060E040E020E030E000E010E00E94A0
:104ED000C62302C00E94992928960FB6F894DEBF17
:104EE0000FBECDBFCF91DF911F910F910895AF926B
:104EF000BF92CF92DF92EF92FF920F931F93DF93B7
:104F0000CF93CDB7DEB768970FB6F894DEBF0FBE6C
:104F1000CDBFB82EA92E082F192FDE011496F80147
:104F2000808191819C01F90185E101900D92815070
:104F3000E1F78A8982FD11C080919628882321F4A7
:104F40008091A028882349F09989D801ED91FC919E
:104F500080E18083918381EE0BC1F801E080F180D4
:104F60008DE0D7018C93898913968C938E898B5F02
:104F7000898385502BE9C22ED12CC81AD108CE0CBA
:104F8000DF1CDB82CA828B89882371F0CE010296F6
:104F9000BE016C5F7F4FAE014F5F5F4F0E94D29D9D
:104FA000282F882309F0C2C08D81823079F4EA81EC
:104FB000FB813297FB83EA8389818E5F89838091AD
:104FC0002828909129289183808313C0833089F405
:104FD0002A813B81285030403B832A838981885F26
:104FE0008983D901EAE1F8E288E001900D928150CD
:104FF000E1F720912528309126288F819885281760
:10500000390749F48D81882331F08E81882319F086
:1050100040E450E00FC08D81882351F0EA81FB818C
:105020003297FB83EA8389818E5F89833183208372
:1050300040E050E03E81332349F18A819B81298100
:10504000323059F4FC013297FB83EA832E5F2983C7
:1050500089859A85918380830DC008979B838A8375
:10506000285F2983FC01DE01199688E00D900192EA
:105070008150E1F7EA81FB813297FB83EA838981E2
:105080008E5F89838F81988591838083EA81FB81FC
:105090003197FB83EA838091A32880838F5F80937D
:1050A000A328BA0161608B89882319F0BA0169606D
:1050B00070618A8980FD60628E89873608F0706130
:1050C0008E81382F330F330F20E04D81942F92952E
:1050D000990F990F907C80E0282B392B8A819B8136
:1050E000FC013297FB83EA83262B372B3183208305
:1050F000298127FF02C025EE19C0FC013397FB83ED
:10510000EA8320838A819B81F701978386838B8939
:10511000882309F465C0C701B601AE014C5F5F4F3B
:105120000E94A69F282F882309F45AC08989D80194
:10513000ED91FC9190E19083818322838EE699E248
:10514000B8010E948D1250C0809124298250823073
:10515000F8F487E498E2B8010E948D128C3851F47B
:105160009989D801ED91FC9180E18083918381EF51
:105170008283E4CF8B2D9A2D0E94052981E00E9425
:105180003D0E882311F40E943026F70114822CC0B2
:1051900080916C29813011F40E947429D7011296F4
:1051A0001C930E931197C70162E070E041E00E94EA
:1051B0001217882321F481E08093252915C099894D
:1051C000D801ED91FC9180E18083918381EE82830F
:1051D0008EE699E2B8010E948D120E94992904C0BE
:1051E0008A8982FFD5CFB0CF68960FB6F894DEBF1C
:1051F0000FBECDBFCF91DF911F910F91FF90EF9028
:10520000DF90CF90BF90AF900895AC01E7E7F8E250
:1052100020E030E080818823A1F4F901EE0FFF1F28
:10522000EE0FFF1FE20FF31FED58F74D8091A528F9
:105230009091A628938382835183408381E0848365
:1052400008952F5F3F4F35962730310519F70895A0
:1052500020E001C0292F822F90E0FC01EE0FFF1FFC
:10526000EE0FFF1FE80FF91FED58F74D8481922FC5
:105270009F5F882379F7392F41E033C0832F90E077
:10528000DC01AA0FBB1FAA0FBB1FA80FB91FAD5887
:10529000B74D14968C911497882311F1822F90E0CA
:1052A000FC01EE0FFF1FEE0FFF1FE80FF91FED5877
:1052B000F74D44838D919C91119791838083129631
:1052C0008D919C9113979383828314961C921497CB
:1052D00011961C921E9213961C921E9212972F5F8B
:1052E0003F5F373058F2089580916C29813051F436
:1052F0000E94001B853831F081E090E00E94D90DBA
:1053000010926C29089580916C29882389F480E09B
:1053100090E00E94D90D80E00E94121B882321F4A6
:1053200081E080936C29089581E090E00E94D90D7E
:10533000089580914D28882331F48091E0288823B6
:1053400011F40E9483290895DF93CF93CDB7DEB780
:1053500028970FB6F894DEBF0FBECDBF482F9B0134
:10536000DB01ED91FC910680F781E02DDE011196C5
:10537000369688E001900D928150E1F7D901ED91C8
:10538000FC918CE18083809125289091262892833E
:10539000818393E0938380911A28848380911B28D2
:1053A000858380911C28868380911D288783809126
:1053B0001E28808780911F288187809120288287DE
:1053C0008091212883879487898185878A81868730
:1053D0008B8187878C81808B8D81818B8E81828B65
:1053E0008F81838B8885848B458B8EE699E2B9010A
:1053F0000E948D1228960FB6F894DEBF0FBECDBF67
:10540000CF91DF9108950F931F93082F10922529B4
:105410001092242910926C291092A0281092A22890
:1054200010929628109246288FEF809369288093D7
:105430006A2880936B2880936C2880936D288093D2
:105440006E2880936F2880937028E3E7F8E2148237
:105450001182108213821282359688E2E639F807AB
:10546000B1F7109223291092E02888E00E94361BA1
:105470001FB7F89480E00E94180F81E00E94180F77
:1054800082E00E94180F1FBF002309F452C010923F
:105490006D2982EC97E0909399288093982880E07A
:1054A00098E79093EA288093E92811E010937228F6
:1054B000109245281092A4280E94DFAE8093A12864
:1054C00084EF91E09093A6288093A52810939728C5
:1054D00086E0809368281092ED281092EE281092B2
:1054E000EF281092F0281092F1281092F2281092D2
:1054F000F3281092F4288FEF9FEF9093DF2880938A
:10550000DE280E94DFAE8093A32810924D281092CF
:10551000482910925A2910925F29109260291092FE
:105520006129109262291092632910924E281092DC
:105530005F281F910F9108950F931F93CF93DF93CF
:10554000EC010881198180916C29813011F40E944D
:105550007429F801018180E090E00E94D90D80E07B
:10556000011181E00E948C19182F81E090E00E94C7
:10557000D90D802F0E94032A0E9499298AE998E276
:105580000E94361383EE98E20E9436138EE699E26B
:105590000E94361387E498E20E943613E881F9816D
:1055A000118380E280838EE699E2BE010E948D1213
:1055B000DF91CF911F910F910895DF93CF9300D08A
:1055C00000D0CDB7DEB780916C29813011F40E94F4
:1055D00074298FEF9FEF9A8389839C838B8383E564
:1055E000BE016F5F7F4F0E944F2B80E5BE016D5F54
:1055F0007F4F0E944F2B81E00E94032A0E9499292D
:105600000F900F900F900F90CF91DF9108950E940F
:10561000C6198823D1F40E94CD118823B1F081E00E
:105620000E94032A0E9499298AE998E26FEF0E945A
:10563000851283EE98E26FEF0E94851287E498E26C
:1056400067E00E94851280E0089585E80895E82FBC
:10565000853419F48091A4280895883030F4E82F17
:10566000F0E0E057FC4F849108958054803228F494
:10567000F0E0E85AFC4F849108958E2F81578331D2
:1056800028F4F0E0E95BFC4F84910895E03F10F4CA
:1056900080E00895F0E0E552FD4F849108951F9356
:1056A000CF93DF93182FEB0180916C29813051F457
:1056B0000E947429812FBE010E943118182F0E9468
:1056C000992904C0812F0E943118182F812FDF9152
:1056D000CF911F9108950F931F93CF93DF938C0168
:1056E000FC01C081D181BE016D5F7F4F898183350F
:1056F00009F4F5C0843508F04CC0823409F4B5C013
:105700008334F8F4843009F4A2C0853068F4813021
:1057100009F4F8C0813008F4F2C0823009F4FBC00B
:10572000833009F07CC0FAC0863009F498C0863016
:1057300008F490C0873009F495C0813409F06FC037
:1057400097C08B3409F4B5C08C3480F4863409F4E6
:105750009CC0873420F4853409F061C08CC0893442
:1057600009F496C08A3409F05AC09AC08F3409F4FB
:10577000ABC0803538F48C3409F4A0C08E3409F005
:105780004EC09FC0803509F4A2C0823509F047C0E1
:10579000A3C0833709F4D1C08437F8F4893509F4FC
:1057A0004BC08A3560F48635E1F1873518F48535CC
:1057B000B1F571C08735C1F1883589F538C08D35AF
:1057C00009F442C08E3518F48A3549F538C081375E
:1057D00009F4A7C0823719F5ADC08C3709F4D2C0DF
:1057E0008D3760F4853709F4B4C0853708F4AEC04E
:1057F000863709F4B7C0873791F4B7C0823809F407
:10580000D6C0833830F4803809F4C5C0813839F403
:10581000C5C0833809F4CFC0803F09F467C094EF56
:10582000D3C080916D29C5C080913528C2C08091B8
:1058300098289091992857C080913928BAC08091B2
:10584000E9289091EA284FC080917228B2C08091D7
:105850002428AFC0809122289091232844C08091B1
:105860003C28A7C080913228A4C080919728A1C06D
:10587000809145289EC04091A4282AEA38E2CB01B5
:10588000B90150E00E942FB09EC08091A42891C021
:105890008091A1288EC08091A5289091A62823C030
:1058A000DB01EDEEF8E288E001900D928150E1F726
:1058B0008AC08091DE289091DF2815C08091A328AE
:1058C00078C08091312875C08091382872C080914D
:1058D00025289091262807C080914D286AC0809184
:1058E0002828909129289C838B836DC0DB01EAE1F5
:1058F000F8E288E001900D928150E1F764C0809158
:10590000332857C08091402890914128A091422887
:10591000B091432832C0809119284BC0809127282C
:1059200048C0DB01E6E2F9E282E201900D9281508B
:10593000E1F749C0809148293CC0DB01E9E4F9E284
:1059400081E101900D928150E1F73DC080915A298B
:1059500030C080915B2990915C29A0915D29B09124
:105960005E290BC080915F2924C0809160299091AD
:105970006129A0916229B09163298B839C83AD83B7
:10598000BE8321C0DB01E4E6F9E288E001900D92DC
:105990008150E1F718C080914E280BC0DB01EFE485
:1059A000F8E280E101900D928150E1F70CC0809106
:1059B0005F288B8308C0DB01E0E6F8E288E0019015
:1059C0000D928150E1F790E089818A838EE188838E
:1059D00099838EE699E2B8010E948D12DF91CF91F2
:1059E0001F910F910895FF920F931F93CF93DF9311
:1059F000182FEB01F42E853509F4AFC0863508F079
:105A000040C0873409F4E4C08834F8F4823409F4DF
:105A100087C0833468F4853038F4823008F0D8C009
:105A2000882309F4D5C06CC0813409F069C080C0F6
:105A3000843409F479C0843408F4CAC0853409F484
:105A40007BC0863409F05CC080C0813598F48E3408
:105A500008F0BEC08A3409F487C08B3420F489343E
:105A600009F04EC076C08B3409F497C08C3409F02D
:105A700047C09AC0823509F49BC0823508F440C003
:105A8000A7C0843709F422C18537E8F48A3509F4C0
:105A900040C08B3550F4873509F49AC0873590F1B2
:105AA0008835A1F1893561F593C0813709F4F8C0D3
:105AB000823718F48D3521F5ECC0823709F4F9C02E
:105AC0008337F1F4FAC0803809F42BC1813860F4CF
:105AD000863709F40CC1863708F4FCC0873709F40F
:105AE0000AC18C3769F414C1823809F42AC182389A
:105AF00008F41EC1833809F42BC1803F09F468C043
:105B000004EF2FC1888180936D292AC188819981F2
:105B1000BBC0888199819093EA288093E92820C1AD
:105B20008881809397281CC188818093682818C138
:105B300088818093452814C12AEA38E24091A4283C
:105B4000C90150E00E942FB00BC188818093A42826
:105B500007C188818093A12803C18881998190938E
:105B6000A6288093A528FCC088818093ED28898190
:105B70008093EE288A818093EF288B818093F02890
:105B80008C818093F1288D818093F2288E8180937F
:105B9000F3288F818093F428E3C0888199819093C2
:105BA000DF288093DE28DCC088818093A328D8C0BA
:105BB0006881611161E060934D28662331F00E9495
:105BC000742986E00E94361BCBC00E949929C8C068
:105BD000812FBE010E943118082F813871F40E9474
:105BE000001B812FBE010E943118082F882309F065
:105BF000B8C081E08093CE1B03C0882309F0B1C0F8
:105C000080913128282F30E080913528482F50E0AE
:105C100060913828CA01861B9109281739070CF4AE
:105C2000C901A82F281B310981E090E002C0880F2C
:105C3000991F4A95E2F70197289FA001299F500DCF
:105C4000389F500D112420E030E070E0E1E0F0E0FA
:105C50000DC0C901860F971FEF0102C0CC0FDD1FD9
:105C60008A95E2F74C0F5D1F2F5F3F4F2A1788F38D
:105C700084E190E09C01429FC001439F900D529FA0
:105C8000900D1124865F9E4F9093992880939828B9
:105C900067C090E08881811191E09093722860C084
:105CA000A6E2B9E2FB0182E201900D928150E1F798
:105CB00057C088818093482953C0A9E4B9E2FB0109
:105CC00081E101900D928150E1F74AC08881809373
:105CD0005A2946C088819981AA81BB8180935B291A
:105CE00090935C29A0935D29B0935E2939C0888187
:105CF00080935F2935C088819981AA81BB81809377
:105D0000602990936129A0936229B093632928C0E8
:105D1000A4E6B9E2FB0188E001900D928150E1F721
:105D20001FC090E08881811191E090934E2818C0A7
:105D3000AFE4B8E2FB0180E101900D928150E1F700
:105D40000FC090E08881811191E090935F2808C096
:105D5000A0E6B8E2FB0188E001900D928150E1F7E6
:105D600000E0FF2049F08091CE1B882329F080E0DD
:105D70000E94121B1092CE1B802FDF91CF911F919A
:105D80000F91FF900895EF92FF920F931F937C0164
:105D9000FC0100811181B8016E5F7F4FF8018181A4
:105DA00041E00E94F32CF801918192839FE190835E
:105DB00081838EE699E2B7010E948D121F910F91A7
:105DC000FF90EF900895CF93DF93EC01E881F98184
:105DD00083E280836183662311F00E9499298EE615
:105DE00099E2BE010E948D12DF91CF9108958091BA
:105DF000F7288823E1F080E00E94180F8091F728AF
:105E0000813031F480911929882311F060E001C0BC
:105E10006BEE80919628823031F48091A828909181
:105E2000A9280E94E32E1092252910929628089501
:105E300080919628823039F48091A8289091A928E1
:105E40006BEE0E94E32E1092962810922529089559
:105E5000CF92DF92EF92FF920F931F93DF93CF9336
:105E6000CDB7DEB728970FB6F894DEBF0FBECDBF13
:105E7000D82EC92E80919628882309F03EC08091A3
:105E800024298330D1F18091A0288823B1F5809115
:105E90006C29813011F40E947429ED2CFC2CD7015F
:105EA000ED91FC9181819F012C5F3F4F823031F455
:105EB000848195819A83898342E00DC0AE014F5F52
:105EC0005F4F88E0D9010D909D01DA010D92AD017F
:105ED0008150C1F743E00281138181E060E09E01BF
:105EE0002F5F3F4F0E94C623882311F4C70107C0CC
:105EF000D092A828C092A92805C08D2D9C2D61EEB6
:105F00000E94E32E28960FB6F894DEBF0FBECDBFD9
:105F1000CF91DF911F910F91FF90EF90DF90CF9085
:105F200008955F926F927F928F929F92AF92BF92ED
:105F3000CF92DF92EF92FF920F931F93DF93CF9355
:105F4000CDB7DEB761970FB6F894DEBF0FBECDBFF9
:105F5000BC014091A028423011F0443069F4809196
:105F60009728882349F0E091A828F091A92820815A
:105F70003181D901199604C0A0E0B0E020E030E002
:105F800050910529598300910629109107291B83F7
:105F90000A83523069F41E821F82188619861A8677
:105FA0001B8680910829909109299D838C8318C0B4
:105FB000809108298C83809109298D8380910A29F9
:105FC0008E8380910B298F8380910C298887809103
:105FD0000D29898780910E298A8780910F298B87C7
:105FE000909033289C86B0902428BD8680911A29F1
:105FF00090911B299F878E87188A80911C2987FF83
:1060000002C081E0888B80911829898B423019F079
:10601000443009F06FC080919728882309F46AC042
:10602000F901F084EC81FD815C806D807E808F8041
:10603000A884C984DA84EB8440E049C011968D912C
:106040009C9112970817190709F03FC08C915817B7
:10605000E1F51B968C911B979816B9F51C968C91BF
:106060001C97B81691F5523041F413968D919C917E
:106070001497E817F90749F53DC013968C911397CB
:10608000851519F514968C9114978615F1F41596CB
:106090008C9115978715C9F416968C9116978815CB
:1060A000A1F417968C9117978A1579F418968C910C
:1060B00018978C1551F419968C9119978D1529F410
:1060C0001A968C911A978E15A9F04F5F51964F151D
:1060D00008F4B4CF59C0FD01DE01119681E10D90A5
:1060E00001928150E1F7D90118968C9118978F5F32
:1060F00018968C9390911D2980912029882321F452
:10610000809197288823E1F5DB01ED91FC9187E1EF
:1061100080838091F92881839F012E5F3F4FAE01DC
:106120004F5F5F4F81E1DA010D90AD01D9010D9212
:106130009D018150C1F780911D29838B892F877024
:1061400059F4892F90E08077907024E09595879599
:106150002A95E1F7882331F080911E2990911F291B
:10616000958B848B80912029868B80912129909119
:106170002229908F878B8EE699E20E948D1209C0AA
:10618000CB010E94561205C0E4E0EF1508F4B2CF2F
:10619000A2CF61960FB6F894DEBF0FBECDBFCF91F0
:1061A000DF911F910F91FF90EF90DF90CF90BF9004
:1061B000AF909F908F907F906F905F9008950F9316
:1061C0001F93DF93CF9300D000D0CDB7DEB78C0103
:1061D00083E693E29A838983F801818192819C838B
:1061E0008B8387E498E2BE016F5F7F4F0E942A1382
:1061F000F80141815281E3E7F8E220E030E080815C
:1062000091814817590779F4F901EE0FFF1FEE0F3E
:10621000FF1FE20FF31FED58F74D14821182108219
:106220000E94282906C02F5F3F4F35962730310541
:1062300031F7109223290F900F900F900F90CF916C
:10624000DF911F910F910895EF92FF920F931F938B
:10625000CF93DF93182FEB01109225298091A0286E
:106260008250823020F4812F0E941B34B5C0888177
:10627000883009F4A5C0893050F4823009F497C001
:10628000843009F44DC0813009F0A4C01DC08B30AA
:1062900009F446C08C3020F48A3009F09BC096C0C7
:1062A0008C3009F493C08D3009F094C0809123297B
:1062B000882319F0CB010E94DF3089819A81612FF8
:1062C0004B810E94A52586C0193E11F0113E41F474
:1062D00089819A81612F4FEF5FEF0E94841B7AC002
:1062E000809396284091E9285091EA2860E070E078
:1062F00024E0440F551F661F771F2A95D1F780E0D1
:1063000020E030E005ED1BE1EE24FF240E94241084
:10631000882309F461C080E090E00E94D51B5CC036
:1063200089819A810E94561280919628813009F4C1
:1063300053C088818430A1F4173881F0E091A828F7
:10634000F091A928A081B18183E28C9311961C93CE
:106350008EE699E2BF010E948D123CC082E005C02A
:10636000193EC1F1113EB1F183E08093962840912E
:1063700098285091992860E070E094E0440F551FF0
:10638000661F771F9A95D1F780E020E030E008E1A2
:106390001FE2EE24FF240E94241091E0909325290F
:1063A0008823D1F080E090E00E94182F15C0CB0127
:1063B0000E94DF3069817A81812F0E94A4290AC05E
:1063C00069817A81812F0E946F3404C089819A810A
:1063D0000E9456120E949929DF91CF911F910F912F
:1063E000FF90EF900895CF93DF93E091EB28F09129
:1063F000EC28C081D181DE01A656BF4FFA83E98324
:10640000882339F087E088838C9323E038E04AE0E2
:1064100013C086E088838C9318979D014AE158E267
:1064200088E0FA010190AF01F90101929F018150CA
:10643000C1F723E438EC42E1FD018FEF9FEF929327
:10644000829332979183808315978091A3288C93B0
:106450008F5F8093A3283E932E93FD014293FF8389
:10646000EE83CE0162E070E040E00E9412178823C4
:1064700011F080E003C081E080932529DF91CF9166
:106480000895CF92DF92FF920F931F93DF93CF93E4
:106490000F92CDB7DEB7F82E6B01FB0100811181A1
:1064A00084E065ED7BE10E944F2B4091A028509144
:1064B00097282091D41B66C0423011F0443039F443
:1064C000552329F0F8018085853008F05EC0322F11
:1064D0003F5FF80184819581A681B781022E04C0B7
:1064E000B695A795979587950A94D2F78170907085
:1064F000892B09F446C02093D41BF1E0FF1621F448
:1065000082E08093A02805C083E0F81611F4F09291
:10651000A02880E064ED7BE10E944F2BF82E8823B9
:10652000B9F08091EB289091EC280E9456121092BD
:10653000EC281092EB280E9499298AEEF8018183B9
:1065400010868EE699E2B6010E948D121092A02864
:106550001091A028123009F05DC0FF2061F481E0A5
:106560000E94F331882309F055C01983CE010196AA
:106570000E94E7334FC08091D41B8F5F8093D41B60
:1065800049C0232F2B3108F497CF2093D41BF1E07F
:10659000FF1609F03FC08091EB289091EC280E94F3
:1065A00056121092EC281092EB288091972888239D
:1065B00041F0F8018085853010F08AEF07C088230C
:1065C00019F0F801118203C08AEEF801818380E599
:1065D00061EE78E20E944F2B6091A8287091A92863
:1065E0008EE699E20E948D128091A7288093D41B99
:1065F00080E064ED7BE10E944F2B809171288093B5
:10660000D51B84E065ED7BE10E944F2B1092A02802
:106610000E9499290F90CF91DF911F910F91FF90C8
:10662000DF90CF900895CF92DF92EF92FF920F9379
:106630001F93DF93CF9300D0CDB7DEB7D82EC92EEE
:10664000082F192FD801ED91FC9180913328809368
:10665000A728809124288093712886818093D61B57
:1066600081818093CF1B82819381A481B5818093A6
:10667000D01B9093D11BA093D21BB093D31B278127
:106680002093D51BD092A828C092A9288BE18083A3
:106690008091CF1B82838091D01B9091D11BA091C0
:1066A000D21BB091D31B84839583A683B7832383A6
:1066B0001086118680919628882341F48091A02825
:1066C000882321F48091CF1B882341F488EE8183B5
:1066D0008EE699E2B8010E948D126EC080916C29FD
:1066E000813011F40E947429F801E080F1808BE080
:1066F0008093D41B8091CF1B8150823008F052C010
:106700008FEF9FEF9A838983809125289091262887
:106710009093E2288093E12880E5BE016F5F7F4F70
:106720000E944F2B8091CF1B813021F4D092EB2817
:10673000C092EC288DE90E945E129093A928809364
:10674000A828009729F488EED70111968C932DC0C4
:106750008091CF1B823019F4C8010E9456122091FB
:10676000A8283091A928D901ED91FC918BE1808373
:106770008091CF1B82838091D51B83838091D01B16
:106780009091D11BA091D21BB091D31B8483958390
:10679000A683B783108611868091CF1BB9010E9412
:1067A00041320AC088EEF70181838EE699E2B80192
:1067B0000E948D120E9499290F900F90CF91DF9126
:1067C0001F910F91FF90EF90DF90CF900895CF939E
:1067D000DF93C091A828D091A92898812981809120
:1067E000A0288250833020F5E92FF22F21E030E0FD
:1067F00040E050E00090D41B04C0220F331F441F20
:10680000551F0A94D2F72095309540955095848174
:106810009581A681B78182239323A423B523848302
:106820009583A683B7838091CF1BBE010E9441321E
:10683000DF91CF910895DF92EF92FF920F931F9314
:10684000DF93CF930F92CDB7DEB7982F8091A32817
:106850008F5F8093A328D090A02882E0D816B1F54E
:10686000992341F540EC53E060E070E00090D61BC6
:1068700004C0440F551F661F771F0A94D2F7405477
:106880005C4F6F4F7F4F94E0440F551F661F771F7B
:106890009A95D1F720E030E007EE13E3EE24FF24D1
:1068A0000E942410882391F0D982CE0101960E9483
:1068B000E7330CC08091D41B8F5F8093D41B609111
:1068C000A8287091A92881E00E9441320F90CF91B1
:1068D000DF911F910F91FF90EF90DF900895CF937C
:1068E000DF93EB01882391F46AED7BE10E944F2B4B
:1068F000882361F484E06BED7BE10E944F2B80E5FF
:1069000068ED7BE10E944F2B90E001C098EEE8819A
:10691000F98182E2808391838EE699E2BE010E9432
:106920008D120E949929DF91CF910895EF92FF92E5
:106930000F931F93CF93DF937C01DC01CD91DC910A
:10694000A7EDBBE1FE018AE001900D928150E1F7D5
:1069500080912828909129288F5F9F4F39F4D70183
:10696000ED91FC9182E280838CEE1FC0BE01695FD5
:106970007F4F8BE00E944F2B8091E01B8823E1F03A
:106980004091D81B5091D91B88E0B7012091DA1BA8
:106990000091DB1B0E943235882309F05CC0D701CF
:1069A000ED91FC9182E2808388EE81838EE699E20C
:1069B000B7010E948D124FC0BE016B5F7F4F87E40D
:1069C0000E944F2B8D818F3009F48E83269684E5AB
:1069D000BE010E944F2B80916C29813011F40E94DE
:1069E000742980E568ED7BE10E944F2B80E06AED21
:1069F0007BE10E944F2B182F84E06BED7BE10E941E
:106A00004F2B8BE06EED7BE10E944F2B1123A9F4FD
:106A100086E00E94361B863081F48091DE1B88233D
:106A200011F083E001C082E080932429D701ED9129
:106A3000FC9182E28083118207C0D701ED91FC9125
:106A400082E2808388EE81838EE699E2B7010E941C
:106A50008D120E949929DF91CF911F910F91FF9084
:106A6000EF900895DF92EF92FF920F931F93DF93C1
:106A7000CF93CDB7DEB72C970FB6F894DEBF0FBE1D
:106A8000CDBF182FFB01F42EE52ED22EBE016F5F75
:106A90007F4F808191819C018CE0D9010D909D01F7
:106AA000DB010D92BD018150C1F740815181DA01B6
:106AB0001C931296FC93EE931197BA016E567F4F7A
:106AC000FB0188E08193DB011196FC92DF011196B6
:106AD000E1829D012F5F3F4F8091282811968C9372
:106AE000F901319680912928D90111968C93DF0103
:106AF0001196D182FD0131969F012F5F3F4F1930D2
:106B000029F48A8511968C938B8503C08FEF11969B
:106B10008C938183F901319600839B01285030408A
:106B2000D901EAE1F8E288E001900D928150E1F7A5
:106B3000F90180912528909126289293829319300B
:106B400099F4F9013A979F01BE016E5F7F4F88E08B
:106B5000DB010D90BD01D9010D929D018150C1F75E
:106B600062E223E23CED07C08FEF9FEF92938293A6
:106B70006CE123E038ED8FEF9FEF92938293809149
:106B8000A32882938F5F8093A328329322936293EA
:106B9000DA011796FC93EE931697CA0162E070E053
:106BA00041E00E941217882311F080E003C081E0C9
:106BB000809325292C960FB6F894DEBF0FBECDBF6B
:106BC000CF91DF911F910F91FF90EF90DF9008958B
:106BD0000F931F93CF93DF93EC018DE90E945E1218
:106BE0008C010097F9F0DC01ED91FC918EE080833F
:106BF0008881818389819A81938382833496DE019F
:106C0000139688E00D9001928150E1F78AE998E2AD
:106C1000B8010E948D12882311F481E004C0C801DC
:106C20000E94561280E0DF91CF911F910F9108953D
:106C30008F929F92AF92CF92DF92EF92FF920F933B
:106C40001F93CF93DF934C01F62ED42E122F8DE994
:106C50000E945E12EC010097C9F0E881F9818DE095
:106C6000808392828182F38215830683E782C086C5
:106C7000A186D4828AE998E2BE010E948D128823FF
:106C800011F481E004C0CE010E94561280E0DF9131
:106C9000CF911F910F91FF90EF90DF90CF90AF9029
:106CA0009F908F900895BF92CF92DF92EF92FF92C4
:106CB0000F931F93CF93DF93182F6A017B01B22E9E
:106CC0008DE90E945E12EC010097B9F0E881F9812C
:106CD0008BE080831183C282D382E482F582B68204
:106CE00007838AE998E2BE010E948D12882311F47D
:106CF00081E004C0CE010E94561280E0DF91CF9166
:106D00001F910F91FF90EF90DF90CF90BF9008956B
:106D10001F93CF93DF93182F8DE90E945E12EC0131
:106D2000009789F0E881F98188E0808311838AE9FE
:106D300098E2BE010E948D12882311F481E004C004
:106D4000CE010E94561280E0DF91CF911F910895ED
:106D50001F93CF93DF93182F8DE90E945E12EC01F1
:106D6000009789F0E881F98189E0808311838AE9BD
:106D700098E2BE010E948D12882311F481E004C0C4
:106D8000CE010E94561280E0DF91CF911F910895AD
:106D90007F928F929F92AF92BF92CF92DF92EF92AB
:106DA000FF920F931F93CF93DF93F22ED32EC42E17
:106DB000B52EA62E972E882E792E8DE90E945E1272
:106DC000EC010097D9F0E881F98182E08083F182BB
:106DD000D282C382B482A58296828782708612870D
:106DE0000187E3868AE998E2BE010E948D1288231A
:106DF00011F481E004C0CE010E94561280E0DF91C0
:106E0000CF911F910F91FF90EF90DF90CF90BF90A7
:106E1000AF909F908F907F900895DF92EF92FF92B6
:106E20000F931F93CF93DF93F82ED62EEA01E22E15
:106E30008DE90E945E128C01009731F1DC01ED9129
:106E4000FC9181E08083F1828881838389819A81AA
:106E5000958384839F012A5F3F4FDE01139688E06C
:106E60000D90E90109929E018150D1F7E686D28208
:106E70008AE998E2B8010E948D12882311F481E01A
:106E800004C0C8010E94561280E0DF91CF911F918B
:106E90000F91FF90EF90DF9008955F926F927F9235
:106EA0008F929F92AF92BF92CF92DF92EF92FF921A
:106EB0000F931F93DF93CF93CDB7DEB7D82E3B014F
:106EC000F42E922E532EB02E86E7841708F455C068
:106ED0008DE90E945E128C01009709F44EC0DC011E
:106EE000ED91FC9183E08083D182D3012C912283A8
:106EF00011968D919C91129794838383CF0105966F
:106F0000A3014D5F5F4F223079F4158216821782FC
:106F10001086118612861386148613968D919C9185
:106F20001497968385830AC09C0188E0DA010D904E
:106F3000AD01D9010D929D018150C1F7B586E6865C
:106F4000C786A08A818AF28A2BE930E02F1931099D
:106F50002E0F3F1FC901692D752D4F2D50E00E9446
:106F60002FB08AE998E2B8010E948D12882311F4AB
:106F700081E004C0C8010E94561280E0CF91DF91E9
:106F80001F910F91FF90EF90DF90CF90BF90AF9047
:106F90009F908F907F906F905F900895FF920F93D6
:106FA0001F93CF93DF93182F062FF72E8DE90E94A2
:106FB0005E12EC010097E1F0812F0E94272B482FF1
:106FC000E881F98186E0808311833296CF01602FBA
:106FD0007F2D50E00E942FB08AE998E2BE010E9406
:106FE0008D12882311F481E004C0CE010E94561254
:106FF00080E0DF91CF911F910F91FF9008951F9333
:107000000E947D25182F8EE699E260E070E00E94D4
:107010002A13009719F00E94662511E00E94AE1510
:107020000E947F0D812F1F9108958EE699E26FEFE8
:107030000E9485120E94072B089581E08093E11B36
:1070400008953F924F925F926F927F928F929F929C
:10705000AF92BF92CF92DF92EF92FF920F931F9366
:10706000DF93CF93CDB7DEB762970FB6F894DEBF4C
:107070000FBECDBF4C015B013A01322ED02EFE2C4B
:107080008091E11B882321F00E94A73A1092E11B16
:107090004F2D50E09A01237030702115310511F405
:1070A000EE240AC02F5F3F4F81E090E002C0880FBE
:1070B000991F2A95E2F7E82E487F452BA1F4811409
:1070C000910489F0A114B10471F0432C552482017C
:1070D0000D0D111D8E2D90E09A8B898B800F911FC5
:1070E0008038910520F00E949D3A81E0A3C08091F4
:1070F0005A06882339F06114710409F50E949D3AFB
:1071000082E098C061147104D1F040E130E0415058
:10711000E42FF0E0D301AE0FBF1FEE51F44E8C917F
:107120002081822790E0232F30E0822B932B30E0C8
:10713000892B09F031E0442351F730935A068091AE
:107140005A06882379F0C30160E040E00E94C83A03
:10715000A2EEBBE1F30180E101900D928150E1F7D5
:1071600010925A0681E0F5018083EE2061F08E2DA9
:1071700090E002979595879523E0880F991F2A95AF
:10718000E1F781608083332021F0F5018081806404
:10719000808384E0782E7F20F50160801686CC20E5
:1071A000D1F4EE2051F0D786080D191DC401B801A5
:1071B000A501232D0D2D0E941B3A7720C1F181E0FE
:1071C000F5018083C401840D951DB5014E2D2D2D33
:1071D0000E9435392CC0772059F081E0F501808379
:1071E000C401840D951DB5014E2D2D2D0E943539FC
:1071F000EE20E9F0F5016082D786C4017E01089493
:10720000E11CF11CB701A501232D0D2D0E941B3A95
:10721000832D90E08D0D911D880D991DB701498931
:107220005A890E9422B0009711F083E003C00E94A7
:107230009D3A80E062960FB6F894DEBF0FBECDBFD8
:10724000CF91DF911F910F91FF90EF90DF90CF9042
:10725000BF90AF909F908F907F906F905F904F9076
:107260003F9008950E94813A08954F925F926F92E5
:107270007F928F929F92AF92BF92CF92DF92EF92C6
:10728000FF920F931F93DF93CF93CDB7DEB7609735
:107290000FB6F894DEBF0FBECDBF5C016B01642E4C
:1072A000122F80E090E060E040E00E94C83A77242E
:1072B000EE24FF24412E55244E010894811C911C7C
:1072C00025C07394D6011F967C92C6010E94823A13
:1072D000C4010E94943AC8010131110514F080E103
:1072E00090E0D501F401282F30E0A401420F531F94
:1072F00004C08C91919189278D93E417F507C9F704
:10730000A20EB31EE0EFFFEFEE0EFF1E8701040D8D
:10731000151D10161106ACF26620E9F0D6011F9675
:107320001C92C6010E94823A8E010F5F1F4FC80156
:107330000E94943A20E030E00CC0F801E20FF31F05
:10734000D5018C9190818927F50181935F012F5F91
:107350003F4F621691F760960FB6F894DEBF0FBEEE
:10736000CDBFCF91DF911F910F91FF90EF90DF90F4
:10737000CF90BF90AF909F908F907F906F905F90D5
:107380004F900895CF92DF92EF92FF920F931F9349
:10739000DF93CF93CDB7DEB760970FB6F894DEBF1B
:1073A0000FBECDBF6C01F62E8C01E62E07C0C801C2
:1073B0000E94823A005F1F4F80EFE80E8FE08E152B
:1073C000B0F30F2D0F70F2949FE0F9222F2D30E0D3
:1073D00084E0220F331F8A95E1F72C0D3D1D002319
:1073E000D9F010E07E010894E11CF11CC701B9013D
:1073F000402F50E00E942FB0E0E1F0E0E01BF10BE5
:107400009701200F311FC90160E070E0AF010E94B9
:107410004AB0C7010E94823A60960FB6F894DEBF68
:107420000FBECDBFCF91DF911F910F91FF90EF90D5
:10743000DF90CF9008959F92AF92BF92CF92DF924C
:10744000EF92FF920F931F93DF93CF93CDB7DEB7E9
:1074500060970FB6F894DEBF0FBECDBF6C015B0125
:107460007A01122F902EFA01078780E090E060E009
:1074700040E00E94C83AC7010E94823A80E090E052
:1074800061E040E00E94C83A112301F1012F1F3052
:1074900008F00EE019821A83E02EFF249E012D5F72
:1074A0003F4FC901B601402F50E00E942FB0602F1E
:1074B0006E5FCE0101960E94C239011738F4612F28
:1074C000601BC6018E0D9F1D0E94C239C601810F2F
:1074D000911D692D0E94C239C5010E94943A60969F
:1074E0000FB6F894DEBF0FBECDBFCF91DF911F91D5
:1074F0000F91FF90EF90DF90CF90BF90AF909F9053
:1075000008950895FC0190E0819180933E019F5F72
:107510009031D1F78091F31B806880933C0180917A
:107520003D0180FFFCCF0895FC0190E080913E0179
:1075300081939F5F9031D1F708958091141C9091B1
:10754000151C0F9719F480E00E94121B089580917A
:107550003A2890913B289093151C8093141C0F9708
:1075600011F40E94001B80915B06882319F0E4E06F
:10757000FCE102C0E4EFFBE190E0819180933F01E8
:107580009F5F9031D1F78091F31B80933C01089568
:107590000F931F93DF93CF93CDB7DEB760970FB6EE
:1075A000F894DEBF0FBECDBFDC01162F042F00976D
:1075B000F1F01092F21B82E080935B0624EF3BE136
:1075C000AD0180E1FA010190AF01F90101929F0143
:1075D0008150C1F720E030E0FD01E20FF31F808110
:1075E00080933F012F5F3F4F20313105A9F70023E2
:1075F00021F0013009F047C00EC080915B06813058
:1076000079F5E4EFFBE1819180933F018CE1E43077
:10761000F807C9F725C080915B068130A1F1809100
:10762000F21B8823A1F41092F31B10923C01CE01AF
:1076300001960E94823AE4E0FCE180913F0181934F
:107640008CE1E431F807C9F781E08093F21BE4E0B4
:10765000FCE1819180933F018CE1E431F807C9F7A7
:1076600000935B06123078F4802F880F880F880F04
:1076700088701295110F1072812B8093F31B8093E9
:107680003C0181E001C080E060960FB6F894DEBF57
:107690000FBECDBFCF91DF911F910F910895089537
:1076A00008950895089508951092752910927429E7
:1076B00010927629109277291092782910927929C0
:1076C00010927A2910927B2910927C2910927D29A0
:1076D000EEE7F9E28FEF9FEF9183808312821382AE
:1076E0001482158216821782108611863A9629E234
:1076F000E83DF20789F708950895089580EF0E9404
:1077000088368CE596E00E946CB181E08093181C6D
:1077100080E50E94883608958F929F92AF92BF9223
:10772000CF92DF92EF92FF920F931F93DF93CF934D
:10773000CDB7DEB7C65CD0400FB6F894DEBF0FBE43
:10774000CDBF282F6B015A01833309F487C18433DD
:1077500020F4823309F095C2E7C0863321F08C33E0
:1077600009F08FC282C2DA0112969C91129711968B
:107770008C91C82EDD24C90ED11CE5E0F0E0CE0EC0
:10778000DF1EC40ED51E8091FE149091FF14009749
:1077900009F0BCC000D000D0EDB7FEB731968DE641
:1077A00096E0ADB7BEB712969C938E931197DA010F
:1077B0008C91828313820E9430B1750100E010E049
:1077C0000F900F900F900F9021EA822E26E0922EBC
:1077D00022C00115110521F08AE390E00E9465B1F5
:1077E00000D000D0EDB7FEB73196ADB7BEB7129658
:1077F0009C928E921197D70115968C918283138259
:107800000E9430B10F5F1F4F0894E11CF11C0F90D4
:107810000F900F900F90F501818190E008171907E4
:10782000C0F200D084EA96E0ADB7BEB712969C9342
:107830008E9311970E9430B100E010E00F900F90EE
:1078400091EAE92E96E0F92E24C00115110521F0E8
:107850008AE390E00E9465B100D000D0ADB7BEB71A
:107860001196EDB7FEB7F282E182F5018181E00F5A
:10787000F11FE80FF11D858112968C9312971396D4
:107880001C920E9430B10F5F1F4F0F900F900F900E
:107890000F90D50112968C9190E008171907A8F265
:1078A0008E01055C1F4FB601685F7F4FC8010E94C3
:1078B000918700D000D089EA96E0EDB7FEB79283B9
:1078C0008183148303830E9430B10F900F900F9037
:1078D0000F90B601685E7F4FC8010E94918700D06B
:1078E00000D08AEB96E0ADB7BEB712969C938E930C
:1078F000119714961C930E9313970E9430B10F901A
:107900000F900F900F908DEB96E004C0029720F43B
:107910008FEB96E00E946CB1F50163817481C60122
:1079200040810E946588E5C1DA018C91853009F4B7
:107930008BC0863040F48330B9F0843028F5813034
:1079400009F0D7C10CC0873009F440C0873070F10E
:107950008B3009F442C08D3009F0CBC15FC0FA0111
:10796000818180938807C5C18A010F5F1F4F80E521
:10797000B8010E94CE3780E50E9488368EE090E004
:1079800062E070E0A8010FC0DA0111968D919C9120
:10799000129790938707809386078CE490E062E0CB
:1079A00070E046E857E00E94130DA3C1ACE1B7E2D6
:1079B000FA01319688E001900D928150E1F7B5010E
:1079C0006F5F7F4F80EF0E94CE3793C14F5F5F4F55
:1079D00088E090E066E070E0E6CF87E0E82EF12CEA
:1079E000EC0EFD1E89E0F70111928A95E9F78CE211
:1079F000888782E08F878E01075E1F4FCA0101963C
:107A0000B8010E94E886882309F473C1C801B70150
:107A100041E021E030E00E94E57F6BC18DED96E012
:107A2000BE016F5F7F4F0E940490898180931A2A64
:107A3000C501029660E820E030E040E050E003E05D
:107A400010E00E94596155C10E94BA5CFC01E95ED8
:107A5000FE4FD50111968C91878B4BC1FA01208185
:107A6000253009F4EFC0263070F4223011F12330B4
:107A700020F4213009F03DC118C02330E9F0243052
:107A800009F037C11EC0283009F45BC0293030F43A
:107A9000263029F1273009F02CC139C0293009F4EA
:107AA0008AC02A3009F025C1A9C0809188072A839D
:107AB000D2C02A832B83D0C08091890790918A07F6
:107AC00004C080918607909187072C839E838D83C5
:107AD00083E363E070E0AE014C5F5F4FC3C0FE0123
:107AE000709689E0DF011D928A95E9F7288BDE0107
:107AF0005196ECE1F7E288E001900D928150E1F7B8
:107B000083E369E070E0AE01405F5F4FABC08E0180
:107B1000005F1F4F89E0F80111928A95E9F7288BE1
:107B200080E090E068E070E046E050E09E012F5E6B
:107B30003F4F0E94450D83E369E070E0A8010E9479
:107B40002F89FE01B99682E1DF011D928A95E9F73E
:107B500088E089A70E94BA5CAC01B2E0CB16D104E0
:107B600008F4C7C0F501818190E027E131E0829FF0
:107B7000F001839FF00D929FF00D1124E40FF51F8B
:107B8000D50112968C912DE1829FC0011124499656
:107B9000DE019B96E80FF91F80E101900D92815064
:107BA000E1F7F50181818AA783E362E170E0AE012C
:107BB000475D5F4F57C0FE01ED59FF4F82E3DF0184
:107BC0001D928A95E9F721938F0181E00E944E93DF
:107BD000009741F0F801DC0181E30D9001928150A2
:107BE000E1F705C081E3D8011D928A95E9F783E3A7
:107BF00062E370E0AE014D595F4F34C0FE01EB56B9
:107C0000FF4F82E3DF011D928A95E9F789E08193B6
:107C10008F0180E00E944E93009741F0F801DC0153
:107C200081E30D9001928150E1F705C081E3D80115
:107C30001D928A95E9F783E362E370E0AE014B564B
:107C40005F4F10C01B821A822A830E94BA5CFC011B
:107C5000E95EFE4F87898B8383E362E070E0AE01CB
:107C60004E5F5F4F0E942F8944C081E0809324279C
:107C7000A5E2B7E2FA0186E001900D928150E1F7AA
:107C800038C0EDB7FEB738970FB6F894FEBF0FBEF9
:107C9000EDBF319682EE96E0ADB7BEB712969C93DB
:107CA0008E931197B382A28224831582D782C682D3
:107CB0000E9430B1750100E010E0EDB7FEB73896D4
:107CC0000FB6F894FEBF0FBEEDBF0CC06091133924
:107CD00070911439D7018D917D0190E00E9404B11B
:107CE0000F5F1F4F0C151D0588F382E197E00E947E
:107CF0006CB1C5010E942CAECA53DF4F0FB6F89489
:107D0000DEBF0FBECDBFCF91DF911F910F91FF90CE
:107D1000EF90DF90CF90BF90AF909F908F9008959D
:107D2000662341F083E197E00E946CB181E00E94FC
:107D3000A8360895909387078093860781E0809303
:107D4000E2298093181C80E50E9488360895DF930D
:107D5000CF930F92CDB7DEB7882321F081E00E9448
:107D6000A83616C021E02093171C809164039091DF
:107D70006503892B31F40E94543B83E566E877E084
:107D800005C0298382E5BE016F5F7F4F0E94CE3719
:107D90000F90CF91DF9108950F93DF93CF9300D091
:107DA0000F92CDB7DEB721E02983882321F081E04F
:107DB0000E94A83648C0663409F440C0673420F4F5
:107DC000613409F040C018C06235D9F06335D9F587
:107DD0008091640390916503892BA9F52A8381E43E
:107DE000BE016E5F7F4F0E94CE3784E18B8386E4B5
:107DF000BE016D5F7F4F25C082E5BE016F5F7F4F83
:107E000020C08091640390916503892B99F441E02F
:107E100050E060E070E00090880704C0440F551FF8
:107E2000661F771F0A94D2F781E021E000E00E94EC
:107E3000533609C080EF0E94883605C085E46BE8A0
:107E400077E00E94CE370F900F900F90CF91DF9187
:107E50000F910895EF92FF920F93DF93CF93CDB7D9
:107E6000DEB729970FB6F894DEBF0FBECDBF7A01FB
:107E7000882321F081E00E94A83667C0603F09F0A6
:107E800047C0ACE1B7E2FA0188E001900D92815061
:107E9000E1F78091640390916503892B91F041E0B3
:107EA00050E060E070E00090880704C0440F551F68
:107EB000661F771F0A94D2F781E025E000E00E9458
:107EC00053368091171C882309F43FC01092171C69
:107ED00088E08987F7018081888781818F8382810B
:107EE0008E8383818D8384818C8385818B8386813E
:107EF0008A8387818983CE0101960E94E6850E944C
:107F0000BA5CFC01E95EFE4F178A0E9459A11DC0B0
:107F10006035D9F4FA014081518150938A0740932A
:107F200089078091181C882381F01092181C809179
:107F300087078983809186078A8382E08987CA01BF
:107F4000BE016F5F7F4F0E94438529960FB6F8945C
:107F5000DEBF0FBECDBFCF91DF910F91FF90EF90AD
:107F60000895AF92CF92DF92EF920F93CF93DF936A
:107F7000282F8091640390916503892BA1F480914F
:107F8000890790918A076091880740E02FE00FE011
:107F9000EE24E394CC24AA240E94183687E297E0CA
:107FA0000E946CB17AC0222339F4E60100E034E388
:107FB000C32E37E0D32E6EC081E08093E2298093F8
:107FC000171C80E569E877E00E94CE3780E50E94C3
:107FD000883683E566E877E00E94CE375EC02B8561
:107FE000809188072817C1F58C858823A9F5898198
:107FF0009A818D5A9A4B81F58881823039F48B8130
:108000009C819093D9298093D8291FC08330C9F4CB
:108010008B818093DA298C818093DB298D818093F9
:10802000DC298E818093DD298F818093DE298885EC
:108030008093DF2989858093E0298A858093E129CF
:1080400004C081E00E94A83628C0822F60E0AE0103
:1080500020E80E940D3721C000D000D000D0EDB73D
:10806000FEB73196ADB7BEB71296DC92CE9211979D
:108070002283138289819A81958384830E9430B1FF
:1080800061960F5F8DB79EB706960FB6F8949EBFA8
:108090000FBE8DBF0E1508F4A2CFDF91CF910F91C7
:1080A000EF90DF90CF90AF9008956F927F928F9274
:1080B0009F92AF92BF92CF92DF92EF92FF920F9377
:1080C0001F93CF93DF93D22EC32EB42EA52E962EC0
:1080D000872E782E692E8DB79EB70A970FB6F89423
:1080E0009EBF0FBE8DBFEDB6FEB60894E11CF11C1D
:1080F00088E697E0EDB7FEB792838183872D962DB2
:1081000000E20E9455A2C901BA01F70122839383BC
:1081100044837583D682C782B086A1860E9430B11F
:10812000EEE7F9E2C1E0D0E08DB79EB70A960FB650
:10813000F8949EBF0FBE8DBF008111819FEF0F3F4E
:10814000190759F182818D1509F057C083818C156B
:1081500009F053C084818B1509F04FC085818A15C1
:1081600009F04BC08681891509F047C087818815C1
:1081700009F043C08085871509F03FC081858615C9
:10818000E1F52D2D3C2D4B2D5A2D692D782D872D68
:10819000962DEE240E94C83636C0FE01EE0FFF1F5A
:1081A000CE0163E0880F991F6A95E1F7E80FF91F88
:1081B000EC58F64DC08311822D2D3C2D4B2D5A2DA0
:1081C000692D782D872D962D0C2F10E0EE240E941E
:1081D000C836FE01EE0FFF1FEE0FFF1FEC0FFD1F55
:1081E000EE0FFF1FEA58F64DD082C182B282A38201
:1081F000948285827682678206C021963A96CA303A
:10820000D10509F099CFDF91CF911F910F91FF9088
:10821000EF90DF90CF90BF90AF909F908F907F9026
:108220006F900895EF920F93DF93CF93CDB7DEB7A2
:108230000E940C42CF91DF910F91EF900895FC01C5
:10824000DB0118968C911897883099F58C9192E003
:1082500089279085981709F057C0918511968C91C0
:108260001197981709F050C0928512968C91129729
:10827000981709F049C0938513968C911397981716
:1082800009F042C0948514968C9114979817E1F5E3
:10829000958515968C9115979817B1F59685169634
:1082A0008C911697981781F520E0978517968C91F9
:1082B00054C0863061F58C9192E08927908598179B
:1082C00019F5918511968C9111979817E9F492857B
:1082D00012968C9112979817B9F483858F3FA1F469
:1082E00084858E3F89F4958513968C911397981702
:1082F00059F4968514968C911497981729F420E0D8
:10830000978515968C9129C080E090E00895823081
:1083100011F080E00895208530E08091173290E0E0
:108320008D7F28173907F9F49185809118329817B5
:10833000D1F482858823B9F483858F3FA1F48485A5
:108340008E3F89F48585882371F496858C919817E2
:1083500051F420E0978511968C91981321E081E0EB
:108360002827822F089580E090E0089581E080938F
:108370003C21089591E090932E2110922F2180E2CC
:108380008093302182E0809331218DE080933221EF
:1083900088EB8093332190933C2108950F931F9392
:1083A000CF93DF93EC0110923C2110912E2101E03C
:1083B00010C0113061F480E391E2BE0148E050E06A
:1083C0000E9422B0009719F42EE231E208C0009317
:1083D0003C2180913C21882361F320E030E0C901F9
:1083E000DF91CF911F910F9108950F931F93CF931A
:1083F000DF93EC018B010E94CE41892B11F480E0C8
:1084000006C0CE01B8010E941F41811181E0DF91B9
:10841000CF911F910F910895CF92DF92EF92FF922B
:108420000F931F93DF93CF93CDB7DEB72A970FB685
:10843000F894DEBF0FBECDBF7C016B0181E080935D
:108440001A2A10921D1C10921B1C8091162A9091C2
:10845000172A8093191C90931A1C4093182A109283
:10846000192AB90150E00E942FB0D7012C91223077
:1084700081F414968C911497898313968C918A8336
:1084800089819A819093052A8093042A20930C2A4B
:10849000B2C0233009F09AC0F701238134814581AD
:1084A0005681678170858185928508E30E9455A277
:1084B0002B83D70113962C91139714963C91149704
:1084C00015964C91159716965C91169717966C9188
:1084D000179718967C91189719968C9119971A9658
:1084E0009C9100E30E9455A22C83F70123813481E3
:1084F00045815681678170858185928508E20E9459
:1085000055A22D83D70113962C91139714963C9165
:10851000149715964C91159716965C911697179689
:108520006C91179718967C91189719968C911997BA
:108530001A969C9100E20E9455A22E83F701238196
:10854000348145815681678170858185928508E1F6
:108550000E9455A22F83D70113962C91139714963E
:108560003C91149715964C91159716965C91169719
:1085700017966C91179718967C91189719968C916D
:1085800019971A969C9100E10E9455A22887F7013D
:1085900023813481458156816781708581859285EB
:1085A00008E00E9455A22987D70113968C918A87EB
:1085B000E8E1FAE27497DE01139688E00D900192EB
:1085C0008150E1F788E080930C2A15C000D000D0DC
:1085D00000D0EDB7FEB731968FE997E0ADB7BEB7E3
:1085E00012969C938E93119783EB97E093838283EB
:1085F0008BE296E0C4C0D6012C91223081F414960F
:108600008C911497898313968C918A8389819A819E
:1086100090930E2A80930D2A2093152ABDC02330F3
:1086200009F099C0F6012381348145815681678123
:1086300070858185928508E30E9455A22B83D6011F
:1086400013962C91139714963C91149715964C9170
:10865000159716965C91169717966C911797189622
:108660007C91189719968C9119971A969C9100E312
:108670000E9455A22C83F6012381348145815681C5
:10868000678170858185928508E20E9455A22D83BD
:10869000D60113962C91139714963C911497159626
:1086A0004C91159716965C91169717966C911797A3
:1086B00018967C91189719968C9119971A969C91F7
:1086C00000E20E9455A22E83F60123813481458168
:1086D0005681678170858185928508E10E9455A247
:1086E0002F83D60113962C91139714963C911497CF
:1086F00015964C91159716965C91169717966C9156
:10870000179718967C91189719968C9119971A9625
:108710009C9100E10E9455A22887F60123813481B3
:1087200045815681678170858185928508E00E9428
:1087300055A22987D60113968C918A87ADE0BAE2BB
:10874000FE01339688E001900D928150E1F788E0B8
:108750008093152A21C000D000D000D0EDB7FEB71D
:1087600031968FE997E0ADB7BEB712969C938E9382
:10877000119783EB97E09383828385E496E095835A
:1087800084830E9430B1EDB7FEB736960FB6F894E9
:10879000FEBF0FBEEDBF1DC586E291E20E941782AB
:1087A000892B41F010921F1C10921E1C1092212147
:1087B00010922021E091191CF0911A1C908180E008
:1087C0002181422F50E0482B592BCA018070987F9D
:1087D000892F9927803C910549F0803E9105C9F089
:1087E000EE24FF2410E020E030E025C07FEFE72EEC
:1087F00077E0F72EE422F522928180E0238130E0B9
:10880000282B392B80911B1C8C5F80931B1C10E044
:1088100012C01481928180E0238130E0282B392B13
:108820006FEFE62E67E0F62EE422F52280911B1C06
:108830008B5F80931B1C8091202190912121892B9B
:1088400039F1E114F10409F4C4C480911E1C909123
:108850001F1CE816F90609F0BCC4809124219091F0
:1088600025218217930709F0B4C40091032A8BEFE6
:1088700099E264E07AE2402F50E00E9422B0009733
:1088800009F0A7C480910C2A081709F0A2C422C0DD
:10889000E114F104F9F0F0921F1CE0921E1C3093D9
:1088A00025212093242186E291E240E251EA67E00B
:1088B00070E00E9440822BEF39E240910C2AE4E004
:1088C000FAE2C901BF0150E00E942FB080910C2A4A
:1088D0008093032A90911B1C953009F408C44091A1
:1088E000191C50911A1C292F30E0FA01E20FF31FD6
:1088F0006081862F807E803609F0DEC32E5F3F4F79
:10890000240F351F30933B2120933A21818187FF2B
:1089100006C02F5F3F4F30933B2120933A21809137
:108920001B1CE091191CF0911A1CE80FF11D8081AD
:1089300090E09C012071307083FD47C0E0913A21A6
:10894000F0913B21232B71F5A1E2BCE1319683E04C
:1089500001900D928150E1F7E0913A21F0913B2195
:1089600040813496F0933B21E0933A21242F30E06C
:10897000C9018F73907095958795959587958066B9
:108980008093201C46954695407396E0220F331F36
:108990009A95E1F7422B8091211C8F70482B4093D0
:1089A000211C3FC080E68093201C9081892F8695F2
:1089B000869580739F70892B8093211C8181928181
:1089C0009093231C8093221C1DC0232B09F5E0915A
:1089D0003A21F0913B218081869586958F70806643
:1089E0008093201C8081982F969596959073829500
:1089F000880F880F807C892B8093211C1092231C68
:108A00001092221C3396F0933B21E0933A2109C047
:108A100080E68093201C1092211C1092231C10923F
:108A2000221C80911B1CE091191CF0911A1CE80F6C
:108A3000F11D808182FD0BC0E0913A21F0913B2134
:108A400081918093261CF0933B21E0933A21809101
:108A50001B1CE091191CF0911A1CE80FF11D80817C
:108A600090E0837090708130910561F082309105C3
:108A70001CF4892B79F019C08230910529F00397F5
:108A8000A1F406C081E001C080E48093271C0DC0E2
:108A90008FEFFBCFE0913A21F0913B2181918093C0
:108AA000271CF0933B21E0933A21E091191CF091AF
:108AB0001A1C80911B1CE80FF11D2181822F90E070
:108AC00026FF86C027FD02C020E003C02281229538
:108AD0002F7080739070892BF1F010923C2191E0FF
:108AE0000DC080912E21813039F480912F21821781
:108AF00019F48EE291E208C090933C2180913C21D0
:108B0000882379F380E090E0909339218093382195
:108B1000892B09F4ECC280911B1CE091191CF09187
:108B20001A1CE80FF11D818190E0807390708031F4
:108B30009105A9F0813191051CF4892B41F0BFC04A
:108B40008032910531F1C09709F0B9C032C080E19F
:108B5000E8E2FCE1DF011D928A95E9F7B0C0E091FF
:108B60003821F0913921A8E2BCE1329688E00190E9
:108B70000D928150E1F7A0E3BCE180913A21909100
:108B80003B219C01F90188E001900D928150E1F7B1
:108B900061C0E0913821F0913921A8E2BCE1329620
:108BA00088E001900D928150E1F786E0E0E3FCE17E
:108BB00060C0E0913821F0913921A8E2BCE1329601
:108BC00088E001900D928150E1F788E29CE173C04A
:108BD000807390708031910521F1813191051CF4F1
:108BE000892B41F06CC080329105D1F1C09709F01A
:108BF00066C052C0A8E2BCE180913A2190913B212D
:108C00009C01F90180E101900D928150E1F7809182
:108C10003A2190913B21409690933B2180933A21B9
:108C20004EC08EEF8093281C80E88093291CEAE2D6
:108C3000FCE186E0DF011D928A95E9F736962091E6
:108C40003A2130913B21C901DC0188E00D9001926D
:108C50008150E1F780913A2190913B210896DCCF39
:108C60008EEF8093281C80E88093291C8CE0EAE238
:108C7000FCE1DF011D928A95E9F7E0913A21F0913C
:108C80003B21819191919093371C8093361CF093F6
:108C90003B21E0933A2113C08EEF8093281C80E89B
:108CA0008093291CEAE2FCE186E0DF011D928A95AF
:108CB000E9F7CF01029764E07AE20E940E61E09149
:108CC000191CF0911A1C80911B1CE80FF11D4181A9
:108CD000842F90E09C012470307043FF78C0232BD8
:108CE00009F055C18370907081309105D9F08230C0
:108CF00091051CF4892B41F04AC182309105A1F104
:108D0000039709F044C14EC0A8E3BCE180913A2129
:108D100090913B219C01F90180E101900D928150DD
:108D2000E1F7E1C08FEF8093381CE0913A21F09198
:108D30003B2181918093391C2AE33CE189E0D901F0
:108D40001D928A95E9F7D901199685E001900D9257
:108D50008150E1F780913A2190913B2106969093C2
:108D60003B2180933A2113C18FEF8093381CE0910F
:108D70003A21F0913B2181918093391C2AE33CE117
:108D80008BE0D9011D928A95E9F7D901199683E004
:108D900001900D928150E1F780913A2190913B2111
:108DA0000496DDCF8FEF8093381C82E08093391CCE
:108DB0008DE0EAE3FCE1DF011D928A95E9F7E0919D
:108DC0003A21F0913B2181918093471CC8C0232B0D
:108DD00009F46AC047FD02C090E002C092819F7012
:108DE00010923C2121E00DC080912E21813039F478
:108DF00080912F21891719F42EE231E208C02093C7
:108E00003C2180913C21882379F320E030E03093AD
:108E10003921209338212115310509F468C1809149
:108E20001B1CE091191CF0911A1CE80FF11D8181A7
:108E300090E08370907082309105E9F08330910565
:108E400039F1019709F0A3C0A8E3BCE1F90132961A
:108E500088E001900D928150E1F7A0E4BCE180919F
:108E60003A2190913B219C01F90188E001900D92FB
:108E70008150E1F757C0A8E3BCE1F901329688E0E0
:108E800001900D928150E1F786E0E0E4FCE159C0E9
:108E9000A8E3BCE1F901329688E001900D9281507F
:108EA000E1F788E39CE16FC0837090708130910599
:108EB00001F1823091051CF4892B41F068C08230A9
:108EC0009105B1F1039709F062C04EC0A8E3BCE17F
:108ED00080913A2190913B219C01F90180E1019020
:108EE0000D928150E1F780913A2190913B2140967B
:108EF00036CF8EEF8093381C80E88093391CEAE3EC
:108F0000FCE186E0DF011D928A95E9F73696209113
:108F10003A2130913B21C901DC0188E00D9001929A
:108F20008150E1F780913A2190913B21089617CF2B
:108F30008EEF8093381C80E88093391C8CE0EAE344
:108F4000FCE1DF011D928A95E9F7E0913A21F09169
:108F50003B21819191919093471C8093461CF09303
:108F60003B21E0933A2113C08EEF8093381C80E8B8
:108F70008093391CEAE3FCE186E0DF011D928A95CB
:108F8000E9F7CF0102976DE07AE20E940E618091CD
:108F90001D1C885D80931D1C80911B1CE091191C79
:108FA000F0911A1CE80FF11D808182FF56C0A0913C
:108FB0003A21B0913B218C91887F803F09F04DC0D0
:108FC00081E18093261C8C91803F29F1833F09F039
:108FD0008EC0E0E2FCE1B89611968C9111978295D3
:108FE0008F7090E080559F409093481C818311962C
:108FF0008C91119790E08F70907080559F40928374
:10900000838312968D919C91139790934F1C80931C
:109010004E1C149619C011968D919C9112979093A5
:10902000491C8093481C13968D919C9114979093A2
:109030004B1C80934A1C15968D919C91169790938A
:109040004F1C80934E1C1796B0933B21A0933A215E
:1090500080911D1C885F80931D1C90913A21809106
:10906000191C981B90931B1CE114F10451F41092ED
:10907000241C80911D1C8852891B9091182A890FED
:109080000CC0E8EDFFEFEE0EFF1EF092241C88E20C
:1090900090E0E80EF91E8E2D88528093251C809159
:1090A000261C813121F58091241C9091251C9093E0
:1090B0004D1C80934C1C1BC0613409F08AC0892F61
:1090C0008F5F80931B1CA0E2BCE1FA01E80FF11D49
:1090D00088E201900D928150E1F780911B1C885D20
:1090E00080931B1C80911D1C885D80931D1C4091EA
:1090F000182A90911B1C491B40931C1C212F30E007
:1091000083E0220F331F8A95E1F780911D1C280F01
:10911000311D205E334EE091191CF0911A1CE90FAD
:10912000F11DC901BF0150E00E942FB0EF28C9F026
:109130008091202190912121892B31F480911D1C57
:10914000809320211092212120911C1C80912021AC
:1091500090912121820F911D9093212180932021B4
:109160000BC020911D1C80911C1C90E0820F911D52
:1091700090931F1C80931E1C20912021309121214F
:109180002115310539F080911E1C90911F1C281764
:109190003907F9F40AE91AE220E23CE140911E1C89
:1091A00050911F1CC801B9010E942FB060911E1C74
:1091B00070911F1C10921F1C10921E1C10922121D6
:1091C0001092202110921C2A10921B2AC8010E9482
:1091D0008E642A960FB6F894DEBF0FBECDBFCF9136
:1091E000DF911F910F91FF90EF90DF90CF90089546
:1091F0006F927F928F929F92AF92BF92CF92DF92A7
:10920000EF92FF920F931F93DF93CF93CDB7DEB70B
:109210002B970FB6F894DEBF0FBECDBF3C01FE0109
:1092200031968BE0DF011D928A95E9F782E0898310
:109230002091890730918A076114710439F48FEF06
:109240009FEF9D838C833B832A8313C03B832A83B8
:10925000F3014085423079F4308120E0818190E053
:10926000822B932B9D838C8349838F5F9F4F09F0C3
:10927000B8C050E0B7C0483009F09EC0D3012C916F
:1092800030E040E050E060E070E080E090E008E333
:109290000E94D4A2122FF32EE42ED52EC62EB72E66
:1092A000A82E992EF301218130E040E050E060E0EB
:1092B00070E080E090E000E30E94D4A2122BF32A39
:1092C000E42AD52AC62AB72AA82A992AD3011796AA
:1092D0008C911797182B12962C9130E040E050E0BB
:1092E00060E070E080E090E008E20E94D4A2122BDF
:1092F000F32AE42AD52AC62AB72AA82A992AF301EA
:10930000238130E040E050E060E070E080E090E0F9
:1093100000E20E94D4A2122BF32AE42AD52AC62AFC
:10932000B72AA82A992AD30114962C9130E040E05C
:1093300050E060E070E080E090E008E10E94D4A29C
:10934000122BF32AE42AD52AC62AB72AA82A992A50
:10935000F301258130E040E050E060E070E080E023
:1093600090E000E10E94D4A2122BF32AE42AD52A2D
:10937000C62AB72AA82A992AD30116962C9130E03A
:1093800040E050E060E070E080E090E008E00E94A3
:10939000D4A2122BF32AE42AD52AC62AB72AA82A4D
:1093A000992A1C83FD82EE82DF82C886B986AA864E
:1093B0009B8683E0898315C000D000D000D0EDB734
:1093C000FEB7319687ED97E0ADB7BEB712969C9386
:1093D0008E93119783EB97E09383828380E395E0EC
:1093E00029C051E080911A2A90E0FC01B3E0EE0F11
:1093F000FF1FBA95E1F7E80FF91FED5DF54D808588
:10940000823029F1883011F483E022C000D000D0EE
:1094100000D0EDB7FEB7319687ED97E0ADB7BEB798
:1094200012969C938E93119783EB97E0938382839C
:109430008BE395E0958384830E9430B1EDB7FEB74E
:1094400036960FB6F894FEBF0FBEEDBF1BC082E08C
:109450002091162A3091172ABE016F5F7F4F4091ED
:10946000182A00E2E52ECC24AA2488240E944D3735
:109470001092192A1092182A882321F485E098E086
:109480000E946CB12B960FB6F894DEBF0FBECDBF15
:10949000CF91DF911F910F91FF90EF90DF90CF90D0
:1094A000BF90AF909F908F907F906F9008951F9383
:1094B000CF93DF93EC0110921D1C10921B1C109295
:1094C000192A1092182AE091162AF091172AF0937F
:1094D0001A1CE093191C3296F0933B21E0933A2139
:1094E000329780E6808380911B1CE091191CF091DB
:1094F0001A1CE80FF11D118280911B1CE091191CB0
:10950000F0911A1CE80FF11D128282EB9AE20E9480
:10951000CE41892B31F482EA9AE20E94CE41892B16
:10952000B1F080911B1C90E00196E091191CF09124
:109530001A1CE80FF91F80818068808380913A218E
:1095400090913B21019690933B2180933A21809109
:109550009A2A482F50E090919B2A9A0184E0220F8A
:10956000331F8A95E1F7892F82958F70822B282FE0
:10957000269526958295880F880F807C282B692F49
:1095800070E0CB018F709070892B99F580919C2AA7
:1095900090919D2A892B69F580911B1CE091191CE3
:1095A000F0911A1CE80FF11D808188608083809102
:1095B0009A2A90E08F709070892B81F480919B2A79
:1095C000807F61F480911B1CE091191CF0911A1CA2
:1095D000E80FF11D80818061808355C0E0913A21C0
:1095E000F0913B21208380913A2190913B2101967B
:1095F00046C04F705070452B41F5862F807F29F56E
:1096000080911B1CE091191CF0911A1CE80FF11DB0
:10961000808180618083E0913A21F0913B21207C20
:1096200080919B2A8F70282B2083E0913A21F09122
:109630003B2180919C2A90919D2A928381838091E5
:109640003A2190913B2103961AC0E0913A21F09182
:109650003B2180919A2A90919B2AA0919C2AB091BB
:109660009D2A80839183A283B383E0913A21F09174
:109670003B21208380913A2190913B210496909345
:109680003B2180933A218091A02A813161F480911D
:109690001B1CE091191CF0911A1CE80FF11D808130
:1096A000846080830EC0E0913A21F0913B21808359
:1096B00080913A2190913B21019690933B21809398
:1096C0003A218091A12A803479F08F3FC9F081300E
:1096D00011F580911B1CE091191CF0911A1CE80FE8
:1096E000F11D808181600AC080911B1CE091191CD2
:1096F000F0911A1CE80FF11D80818260808319C0EF
:1097000080911B1CE091191CF0911A1CE80FF11DAF
:1097100080818360F3CFE0913A21F0913B218083F7
:1097200080913A2190913B21019690933B21809327
:109730003A218091A22A9091A32A892BB9F5809190
:10974000A42A9091A52A892B89F58091A62A909127
:10975000A72A892B59F58091A82A9091A92A892BAB
:1097600029F58091AA2A9091AB2A892BF9F480914E
:10977000AC2A9091AD2A892BC9F48091AE2A9091A0
:10978000AF2A892B99F48091B02A9091B12A892B24
:1097900069F480911B1C90E00196E091191CF091F6
:1097A0001A1CE80FF91F8081806446C082EA9AE2A1
:1097B0000E94CE419093392180933821892B09F45E
:1097C0006EC080911B1C90E00196E091191CF091F5
:1097D0001A1CE80FF91F8081806C808380911B1C0C
:1097E00090E00296A091191CB0911A1CA80FB91F05
:1097F000E0913821F091392181818295807F9C917F
:10980000892B8C9360911A2A89E0689FB0011124FA
:109810006D5D754D82EA9AE20E941F41882371F0C6
:1098200080911B1C90E00196E091191CF0911A1C8C
:10983000E80FF91F808180638083B3C08091AA2ADA
:109840009091AB2A892B81F48091AC2A9091AD2A1A
:10985000892B51F48091AE2A9091AF2A892B21F463
:109860008091B02A87FF4AC080911B1C90E001962E
:10987000E091191CF0911A1CE80FF91F808180619A
:10988000808320913A2130913B21C901DC01EAEA31
:10989000FAE288E001900D928150E1F766C0809174
:1098A000A22A8E3F09F067C08091A32A803809F070
:1098B00062C060911A2A89E0689FB00111246D5D31
:1098C000754D82EA9AE20E941F41882309F0A8CFD1
:1098D0008091AA2A9091AB2A892B69F58091AC2AB4
:1098E0009091AD2A892B39F58091AE2A9091AF2ABB
:1098F000892B09F58091B02A87FD1DC080911B1C22
:1099000090E00196E091191CF0911A1CE80FF91FE4
:10991000808180628083E0913A21F0913B218091A7
:10992000B02A9091B12A9183808380913A219091BD
:109930003B21029632C080911B1C90E00196E09181
:10994000191CF0911A1CE80FF91F80818061808337
:1099500020913A2130913B21C901DC01EAEAFAE287
:1099600088E001900D928150E1F780913A21909129
:109970003B21089612C080913A2190913B219C0195
:10998000D901E2EAFAE280E101900D928150E1F71B
:1099900080913A2190913B21409690933B21809376
:1099A0003A218091B22A8F3F09F0DDC080911B1CC3
:1099B00090E00196E091191CF0911A1CE80FF91F34
:1099C0008081886080838091B32A823009F042C010
:1099D0008091B42A9091B52A892BE1F58091B62A1D
:1099E0009091B72A892BB1F58091B82A9091B92A24
:1099F000892B81F58091BA2A9091BB2A892B51F548
:109A00008091BC2A9091BD2A892B21F58091BE2A94
:109A10009091BF2A892BF1F48091C02A8823D1F438
:109A200080911B1C90E00196E091191CF0911A1C8A
:109A3000E80FF91F808183608083E0913A21F091E3
:109A40003B218091C12A808380913A2190913B21D2
:109A5000019671C18091B42A9091B52A892B09F0A1
:109A600074C08091B62A9091B72A892B09F06DC0F5
:109A70008091B82A9091B92A892B09F066C080910B
:109A8000BA2A9091BB2A892B81F58091BC2A9091AA
:109A9000BD2A892B51F58091BE2A882331F580910A
:109AA0001B1C90E00196E091191CF0911A1CE80F24
:109AB000F91F808182608083E0913A21F0913B21FF
:109AC0008091B32A8083E0913A21F0913B21319635
:109AD000AFEBBAE283E00D9001928150E1F7809103
:109AE0003A2190913B21049626C18091BA2A909107
:109AF000BB2A892B51F58091BC2A882331F58091AE
:109B00001B1C90E00196E091191CF0911A1CE80FC3
:109B1000F91F808181608083E0913A21F0913B219F
:109B20008091B32A8083E0913A21F0913B213196D4
:109B3000ADEBBAE285E00D9001928150E1F78091A2
:109B40003A2190913B210696F6C080913A2190915E
:109B50003B219C01D901E2EBFAE280E101900D92F8
:109B60008150E1F7E3C082EB9AE20E94CE419093EC
:109B7000392180933821892B09F459C080911B1C0D
:109B800090E00196E091191CF0911A1CE80FF91F62
:109B900080818460808380911B1C90E00296E0911C
:109BA000191CF0911A1CE80FF91FA0913821B091EF
:109BB0003921808111969C91892B808382EB9AE2D6
:109BC000BE010E941F41882309F042C08091BA2A39
:109BD0009091BB2A892B81F48091BC2A9091BD2A57
:109BE000892B51F48091BE2A9091BF2A892B21F4B0
:109BF0008091C02A87FF50C080911B1C90E0019685
:109C0000E091191CF0911A1CE80FF91F8081816006
:109C1000808320913A2130913B21C901DC01EAEB9C
:109C2000FAE288E001900D928150E1F76CC08091DA
:109C3000B22A8E3F09F06DC08091B32A803809F0B6
:109C400068C082EB9AE2BE010E941F41882371F036
:109C500080911B1C90E00196E091191CF0911A1C58
:109C6000E80FF91F80818360808369C08091BA2AE0
:109C70009091BB2A892B69F58091BC2A9091BD2ACD
:109C8000892B39F58091BE2A9091BF2A892B09F53D
:109C90008091C02A87FD1DC080911B1C90E0019619
:109CA000E091191CF0911A1CE80FF91F8081826065
:109CB0008083E0913A21F0913B218091C02A9091DC
:109CC000C12A9183808380913A2190913B21029611
:109CD00032C080911B1C90E00196E091191CF0911C
:109CE0001A1CE80FF91F80818160808320913A213E
:109CF00030913B21C901DC01EAEBFAE288E00190F6
:109D00000D928150E1F780913A2190913B21089684
:109D100012C080913A2190913B219C01D901E2EB44
:109D2000FAE280E101900D928150E1F780913A21B1
:109D300090913B21409690933B2180933A2188E279
:109D400080931D1C8091A02A813109F064C09091FC
:109D5000C22A8091C32A805B904F0F9770F5909133
:109D6000C42A8091C52A20EF803B920730F18F5B97
:109D7000904F18F5E0913A21F0913B2183EF8083D9
:109D8000E0913A21F0913B219091C52A905B80911E
:109D9000C32A8295807F980F9183E0913A21F091B8
:109DA0003B218091C82A9091C92A93838283809114
:109DB0003A2190913B21049625C0E0913A21F091FF
:109DC0003B2180EF8083E0913A21F0913B2180910B
:109DD000C22A9091C32AA091C42AB091C52A818336
:109DE0009283A383B483E0913A21F0913B21809147
:109DF000C82A9091C92A9683858380913A219091AF
:109E00003B21079690933B2180933A2180911D1C22
:109E1000885F80931D1CA0913A218091191CA81B7A
:109E2000A0931B1C80911D1C482F50E0E0911B2A21
:109E3000F0911C2AE41BF50B2A2F30E086E490E019
:109E4000821B930B6091191C70911A1C8E179F072F
:109E500008F0E3C0CB0104964A2F50E00E9438B0CE
:109E6000E091191CF0911A1C80911B2A90911C2AD8
:109E7000906C9083E091191CF0911A1C80911B2A20
:109E80008183E091191CF0911A1C80912321828317
:109E9000E091191CF0911A1C8091222183838091FA
:109EA0001B1C8C5F80931B1C16E4412F481B487FB2
:109EB00040931C1C6091191C70911A1C680F711D35
:109EC00020911D1C30E02656354DCB01B90150E0E4
:109ED0000E942FB020911B1C80911C1C90E0820FCF
:109EE000911D9093192A8093182ACE010E94F84858
:109EF00020911D1C80911C1C90E0820F911D90935D
:109F000021218093202185E080931B1CE091191C66
:109F1000F0911A1C80911B2A90911C2A906E9083BC
:109F2000E091191CF0911A1C80911B2A8183809169
:109F30001B1C181B187F10931C1C55C0E091191C8A
:109F4000F0911A1C13E0369527951A95E1F72483B2
:109F500060911B2A70911C2A40912021509121214F
:109F60009B01241B350B80911C1C90E0281739079E
:109F700020F4862F841B80931C1C80911B1C6091F5
:109F8000191C70911A1C680F711D40911C1C2091A6
:109F90002021309121212656354DCB01B90150E0C9
:109FA0000E942FB020911B1C80911C1C90E0820FFE
:109FB000911D9093192A8093182ACE010E94F84887
:109FC00002C00E94FF37809141018231D1F320917C
:109FD0001C1C8091202190912121820F911D909332
:109FE00021218093202120912021309121218091D5
:109FF0001B2A90911C2A2817390708F49FCF8091BB
:10A000002221909123210196909323218093222154
:10A0100010922121109220211CC0260F371F465676
:10A02000554DC901BA01AF010E942FB020911B1CF0
:10A0300080911B2A90911C2A820F911D20911D1C3A
:10A04000821B91099093192A8093182ACE010E94AD
:10A05000F84881E0DF91CF911F910895FC01538171
:10A06000560F5093222A272F33274281420F4093C5
:10A07000212AA181A093202AE081E0931F2A842F26
:10A0800090E08217930748F48A2F8F5F8093202AED
:10A09000882319F4EF5FE0931F2A852F90E07070FA
:10A0A0008617970790F4842F8F5F8093212A882347
:10A0B00061F48091202A8F5F8093202A882329F4DD
:10A0C00080911F2A8F5F80931F2A08959C01415021
:10A0D0005040460F571FFB010EC0708160E0818128
:10A0E000DB01A80FB11D2A0F3B1F2A173B0710F4F5
:10A0F0002F5F3F4F3296E417F50778F3E417F50723
:10A1000049F4908180E0280F391F2817390710F48F
:10A110002F5F3F4FC90108959C01AB0180E090E0A3
:10A12000B9010E946650282F892F922F089580E050
:10A1300090E06AE97AE248E250E00E9466500097B7
:10A1400019F42FEF3FEF02C0382F292FC9010895CE
:10A150000F931F9310919E2A00E090913E21091BBE
:10A16000110990919F2A090F111D9801280F311D87
:10A17000C90162EA7AE240E250E00E9466506091D2
:10A180003E2170E06E53754DA8010E946650009705
:10A1900019F42FEF3FEF02C0382F292FC9011F916B
:10A1A0000F9108958AE30E94A850089586E00E94C6
:10A1B000A850089581E10E94A85008950F931F931D
:10A1C000CF93DF93182F092F4091412150914221C5
:10A1D000BCE24F5F5F4F8DE74030580710F040E022
:10A1E00050E1342F252FA0E00EC0AB9FF0011124C9
:10A1F000E25CF54D85A1882329F080899189821739
:10A20000930739F3AF5FA23081F740934121509318
:10A21000422110924021E0E0F0E020E03CE21AC050
:10A22000239FD0011124A25CB54D95968C919597F2
:10A23000882321F420934021FD0110C0873049F488
:10A24000309731F096969C91969786A1891708F4DD
:10A25000FD012F5F223020F320934021309771F1D0
:10A2600082E085A380914321808F80914421818F5A
:10A2700080914521828F80914621838F84EC94E0E8
:10A28000978F868F91A380A381E090E0958F848F34
:10A2900017A281E086A383E084A312A280E183A3B6
:10A2A000508B418B738B628BEF01212F302FC901B3
:10A2B000DC0180E10D9009928150E1F7CF01DF913F
:10A2C000CF911F910F910895AC011092402120E091
:10A2D00013C0E22FF0E0322F3F5FEE0FFF1FEA5670
:10A2E000F54D808191818417950729F420934021B1
:10A2F000118210820895232F223058F32093402199
:10A300000895AC011092402120E012C0E22FF0E04D
:10A31000322F3F5FEE0FFF1FEA56F54D808191818E
:10A32000892B29F420934021518340830895232FC2
:10A33000223060F3209340210895BC0180913C2A93
:10A3400090913D2A44960E942E50E0913C2AF09133
:10A350003D2A80911F2A848B8091202A858B8091B1
:10A36000212A868B8091222A878B0895282F892F76
:10A37000922F0895EF92FF920F931F939C01442711
:10A380005527F22EE32E00E010E0362F272F40E075
:10A3900050E0A90133272227E22AF32A042B152BA8
:10A3A000B701C8011F910F91FF90EF900895FC0134
:10A3B00040911D2A50911E2A2AE93FE2241B350BA9
:10A3C000621773070CF49B011216130664F42093B2
:10A3D0009C2F30939D2FE417F50729F0CA01BF0188
:10A3E000A9010E942FB0089582E080933F21A0919F
:10A3F0003E212A2F30E0F901EE53F54D8181682F7F
:10A4000070E0F3E0660F771FFA95E1F7695F7F4F21
:10A4100042E0285D3F4F3CC0F901E80FF91FE656C6
:10A42000F54D8081882319F0813019F42EC04F5FDB
:10A430002FC090E0807C90708038910549F0803C7E
:10A44000910549F08034910501F540933F2109C001
:10A4500040933F2108C040933F218091B22A8F3F13
:10A4600011F481E00895242F30E040E050E02A0FFD
:10A47000311D411D511D285D3F4F4F4F5F4F84E0FF
:10A4800062E00E94D36882E0089581818E5F480F68
:10A49000842F90E0681779070CF0BECF40933F21DE
:10A4A00080E008950F931F93CF93DF93C0913C2AD0
:10A4B000D0913D2A843009F4C5C206ED1AE210930A
:10A4C0003B2A00933A2A10931E2A00931D2A8330B8
:10A4D00069F48DA18F70833011F00C94F75A8C8D34
:10A4E0009D8D892B11F00C94F75A93C0823009F09E
:10A4F00094C010921C2A10921B2A10929D2F109229
:10A500009C2F809146218F5F80934621882399F468
:10A51000809145218F5F80934521882361F480914C
:10A5200044218F5F80934421882329F48091432123
:10A530008F5F809343212DA1273011F0253051F4F6
:10A540008EA18F5F8EA3883711F00C94F75A1DA24D
:10A550000C94F75A222311F40C94F75A8C8D9D8D8C
:10A56000892B09F452C08EA181508EA38F5F11F008
:10A570000C94F75A3FA1383029F02150223048F48A
:10A58000353039F41DA280E88093352A0E94B86ADC
:10A59000D0C6353010F080E307C083E090E002C001
:10A5A000880F991F3A95E2F78EA38FA18F5F8FA333
:10A5B0008DA190E08F7090708330910501F184300F
:10A5C00091054CF48130910509F461C4029711F0B2
:10A5D0000C94F75A0DC08630910509F4BEC6883038
:10A5E000910509F4BAC6049711F00C94F75AB5C650
:10A5F000E0913E21F0E0EE53F54D15864FC484E026
:10A600008093352A0E94B86AD6C62F70233009F08D
:10A61000EEC788E08093352A80C6853019F5E09131
:10A62000382AF091392A80899189892B09F4DFC76A
:10A6300010923D2A10923C2AC8010C9790933B2A15
:10A6400080933A2A90931E2A80931D2A10929D2F60
:10A6500010929C2F10921C2A10921B2A88E0809343
:10A66000352AEEC180919A2A807F803609F0BFC7D3
:10A6700090919E2A80E020919F2AAC01420F511DAB
:10A680009A0180911B2A90911C2A8417950708F43F
:10A69000AEC7285D3F4F30931C2A20931B2A809120
:10A6A000A22A8F3F09F4A3C7C801849760E840E05D
:10A6B00050E00E94B55E892B09F067C0C8018497FD
:10A6C0000E942A5C882309F060C08091B22A8F3FE3
:10A6D00009F058C08091B32A823009F053C08091AC
:10A6E000B42A9091B52A892B09F04CC08091B62AE2
:10A6F0009091B72A892B01F58091B82A9091B92AB7
:10A70000892BD1F48091BA2A9091BB2A892BA1F48C
:10A710008091BC2A9091BD2A892B71F48091BE2A28
:10A720009091BF2A892B41F48091C02A882321F47B
:10A730008091C12A813049F18091B62A9091B72A3F
:10A74000892B01F58091B82A9091B92A892BD1F4EF
:10A750008091BA2A9091BB2A892BA1F48091BC2ABE
:10A760009091BD2A892B71F48091BE2A9091BF2AC5
:10A77000892B41F48091C02A882321F48091C12A39
:10A78000823019F00E94065B3AC780EA9AE2909301
:10A79000372A8093362A10923E2110923D21E09173
:10A7A000362AF091372A80818B3209F44BC08C32E3
:10A7B00048F4863009F4B1C1813109F4B5C0882369
:10A7C00089F06BC08A3309F474C08B3320F48C3267
:10A7D00009F063C00CC78B3309F409C78C3309F047
:10A7E0005CC006C080913D2180FD57C0816009C0DA
:10A7F00080913D2181FF04C086FD4FC0806401C06F
:10A80000826080933D210E94F451813009F4EFC6AB
:10A81000813018F0823019F6F2C620913E21E22FE5
:10A82000F0E0CF018E53954D9093372A8093362ACE
:10A83000285FFC018181880F880F880F280F2093E3
:10A840003E21ADCF80913D2182FD27C08460809361
:10A850003D2190913E21E92FF0E0DF01AE53B54D4F
:10A8600013968C911397882349F0BA969F01442739
:10A8700037FD4095542F84E060E018C0B093372A2C
:10A88000A093362A985FEE53F54D8181880F880F8B
:10A89000880F980F90933E2182CFEA59FA429F0188
:10A8A000442737FD4095542F84E061E00E94D3682F
:10A8B000A6C60E94D2508F5F9F4F09F098C6E091C4
:10A8C0003E21F0E0EE53F54DE081E538B9F0E63891
:10A8D00028F4E038B1F0E138D9F418C0E73829F0AD
:10A8E000E73848F0E838A1F403C00E941D7414C092
:10A8F0000E94397211C00E94FA6B0EC00E94257925
:10A900000BC00E944F030E94B26906C00E942D989E
:10A9100010921C2A10921B2A80911B2A90911C2AAB
:10A92000892B09F464C66BC680911B2A90911C2A5E
:10A93000C09790931C2A80931B2A8AEC9AE29093EA
:10A940003B2A80933A2AE0913E21F0E0EE53F54D08
:10A9500086819781892B31F00E94DA508F5F9F4F5B
:10A9600009F045C68EE99FE29093392A8093382AF0
:10A9700048C02889398921153105F1F180913E219E
:10A98000E82FF0E0EE53F54D828193818217930713
:10A9900099F52A893B892115310529F0808191811A
:10A9A0008217930749F588819981892BE1F48A817F
:10A9B0009B81892BC1F48C819D81892BA1F48E818F
:10A9C0009F81892B81F488859985892B61F48A85FB
:10A9D0009B85892B41F48C859D85892B21F48E855F
:10A9E0009F85892BC1F082EA9AE2BE0140E150E0E6
:10A9F0000E9422B0009779F06996D093392AC093CB
:10AA0000382AC091382AD091392ABFE2C03DDB07ED
:10AA100008F4AFCFECC510923D2A10923C2A82E098
:10AA20008093352A8AEC9AE290933B2A80933A2AC3
:10AA300090931E2A80931D2A10929D2F10929C2F76
:10AA40000E94786820919C2F30919D2F211531050F
:10AA500009F4CDC5C901C09690931C2A80931B2A86
:10AA6000285F3F4F30939E2A885280939F2AA0915F
:10AA7000382AB091392A54968C9154978093A12A00
:10AA800081E18093A02AE0913E21F0E0EE53F54D64
:10AA9000348325831782168250968D919C9151970D
:10AAA0009183808352968D919C9153979383828357
:10AAB000A2EBBAE22091382A3091392AC901FC016F
:10AAC00080E101900D928150E1F782EA9AE262EB17
:10AAD0007AE20E94166086ED9AE290933B2A809378
:10AAE0003A2A80913E21C82FD0E0CE53D54D0E9406
:10AAF000DA50809590959F838E8380913E21E82F38
:10AB0000F0E0EE53F54D86819781892B09F065C5FC
:10AB10008FEF9FEF9783868360C50E94D6508F5F2B
:10AB20009F4F09F064C580913E21082F10E00E531D
:10AB3000154DCEE3DAE28DA18823D9F0D801129623
:10AB40002D913C911397888999892817390789F4A1
:10AB50002D913C918A899B892817390751F482EA03
:10AB60009AE2BE0140E150E00E9422B0009709F451
:10AB7000B2C1AC96BAE2CA36DB07E9F2E0F2F801FC
:10AB800085858F73823001F582819381909349216D
:10AB9000809348211092402113C0E42FF0E0EE0F83
:10ABA000FF1FEA56F54D20914821309149218081BF
:10ABB00091812817390709F489C04F5F40934021DC
:10ABC00040914021423048F380913E21E82FF0E04F
:10ABD000DF01AE53B54D1D968C911D9782FD07C5C3
:10ABE00084E11D968C931D978CE390E090931C2A32
:10ABF00080931B2AFD0180E5848797811B968C91A9
:10AC00001B9717968C931797938796811A968C911A
:10AC10001A9716968C9316979287958119968C9110
:10AC2000199715968C93159791879481909340214D
:10AC300018968C91189714968C93149790871B965E
:10AC40008C911B978F5F1B968C931B978823C1F465
:10AC50001A968C911A978F5F1A968C931A9788235D
:10AC600079F419968C9119978F5F19968C9319978F
:10AC7000882331F418968C9118978F5F18968C93CF
:10AC8000E0913E21F0E0DF01AE53B54D2D913C91B6
:10AC900011973093492120934821FD0182819381AE
:10ACA0009183808313963C932E931297E2EBFAE202
:10ACB000DF01509780E10D9001928150E1F782EA27
:10ACC0009AE262EB7AE20E94166054C4109240212C
:10ACD000C0E0D0E04CE250E03CE225C0822F90E0A2
:10ACE000849FF001859FF00D949FF00D1124E25C8C
:10ACF000F54D85A1882339F48CE2289FE0011124C9
:10AD0000C25CD54D14C0873059F4209721F096A12C
:10AD10008EA1891728F4239FE0011124C25CD54D30
:10AD20002F5F20934021209140212230B8F22097BC
:10AD300009F45DC4D0933D2AC0933C2A83E08EA3DE
:10AD40008CA31AA284E08BA31FA2E0913E21F0E025
:10AD5000EE53F54D82819381998B888B808191810F
:10AD60009B8B8A8BDE01E2EAFAE280E101900D9290
:10AD70008150E1F781E08DA380914321888F8091FC
:10AD80004421898F809145218A8F809146218B8F24
:10AD900081E090E09D8F8C8FE0913E21F0E0EE53BA
:10ADA000F54D87818F8BE0913E21F0E0EE53F54D1C
:10ADB00086818E8BE0913E21F0E0EE53F54D85814A
:10ADC0008D8BE0913E21F0E0EE53F54D84818C8B2C
:10ADD00081E090E00E949D51E0913E21F0E0EE5331
:10ADE000F54D848590E0807F9070813591050CF45D
:10ADF0004EC01092402135C0F901E656F54D84ADA4
:10AE000080934721882309F442C0813021F44F5FA9
:10AE10004093402126C08230C1F485AD8430A9F42E
:10AE200036AD20E087AD90E0822B932B90934921A3
:10AE300080934821F4E0853C9F0710F084EC94E077
:10AE40009F8F8E8F99A388A322C080914021E82FE5
:10AE5000F0E0E952F54DE081EE23C9F0E80FE09310
:10AE6000402140914021242F30E0E0913E21F0E04C
:10AE7000EE53F54D848582958F7090E00597880F8D
:10AE8000991F880F991F281739070CF4B5CFE09147
:10AE90003E21F0E0EE53F54D80E18587E0913E21C3
:10AEA000F0E0DF01AE53B54D1D968C911D97826089
:10AEB0001D968C931D97FD0182E0848B84E0858B29
:10AEC000868B84EC878B80E490E090931C2A80939F
:10AED0001B2A80E60EC3D0933D2AC0933C2A1092D1
:10AEE000352A80913E21A82FB0E0FD01EE53F54DAB
:10AEF000858582FF03C01DA280E293C2848582956E
:10AF00008F70880F880F8093402120911B2A3091E9
:10AF10001C2A28523040281B310930931C2A2093C8
:10AF20001B2A8DA18F70823039F4AE53B54D1D961A
:10AF30008C918F73823139F1232B59F4E0913E21AA
:10AF4000F0E0EE53F54D858590E083709070892B8D
:10AF5000D1F080913E21E82FF0E0EE53F54D948141
:10AF60008C89981709F0B2C295818D89981709F0DC
:10AF7000ADC296818E89981709F0A8C297818F89F2
:10AF8000981709F0A3C2E0913E21F0E0EE53F54D91
:10AF9000858584FF52C06C8D7D8D6115710509F426
:10AFA0004CC0CE0148960E942E5080913E21E82F41
:10AFB000F0E0EE53F54D208580911F2A2817E9F522
:10AFC00091858091202A9817C1F592858091212A38
:10AFD000981799F593858091222A981771F5288FF3
:10AFE0008091202A898F8091212A8A8F8091222A1C
:10AFF0008B8F8FA18823D1F42AA19CA18EA1981BAD
:10B00000822F869586958695981B392F320F3AA305
:10B010008BA1282F26952695821B97FD9195890F48
:10B020008BA3369536953695830F8CA381E080935C
:10B03000352A8CA18EA31D8E1C8E8DA1282F30E069
:10B04000C9018F7090708430910509F4EFC185308B
:10B0500091055CF48230910591F1833091050CF0FB
:10B06000CAC0019709F0C3C210C08630910509F427
:10B0700025C2863091050CF4FDC18730910509F495
:10B0800025C2089709F0B3C2C6C18091352A80FF56
:10B09000AEC283E08DA380E48093352A1D8E1C8E82
:10B0A00020911B2A30911C2A2115310509F431C148
:10B0B00082E48093352AC9010E949D512AC1809162
:10B0C000352A80FF8DC080913E21E82FF0E0EE53BD
:10B0D000F54D85858F73823109F082C0848590E0BB
:10B0E000807F9070813591050CF44EC01092402104
:10B0F00035C0F901E656F54D84AD8093472188238C
:10B1000009F442C0813021F44F5F4093402126C0B2
:10B110008230C1F485AD8430A9F436AD20E087AD2E
:10B1200090E0822B932B909349218093482124E037
:10B13000853C920710F084EC94E09F8F8E8F99A34A
:10B1400088A322C080914021E82FF0E0E952F54D1C
:10B15000E081EE23C9F0E80FE093402140914021C7
:10B16000242F30E0E0913E21F0E0EE53F54D848550
:10B1700082958F7090E00597880F991F880F991F0F
:10B18000281739070CF4B5CF83E08DA3E0913E2159
:10B19000F0E0EE53F54D84818C8BE0913E21F0E0A0
:10B1A000EE53F54D85818D8BE0913E21F0E0EE531D
:10B1B000F54D86818E8BE0913E21F0E0EE53F54D0A
:10B1C00087818F8B81E090E00E949D5182E4809383
:10B1D000352A1D8E1C8E10921C2A10921B2A99C093
:10B1E00080E28093352A0E94B86AE0913C2AF0916F
:10B1F0003D2A15A2E9CC80913E21E82FF0E0EE53E4
:10B20000F54D858580FF25C024FD23C08C8D9D8D47
:10B21000892B09F0ECC180911B2A90911C2A019680
:10B220000E949D512091352A822F80618093352A7A
:10B2300080911B2A90911C2A892B19F0226120935E
:10B24000352A0E94B86A81E090E09D8F8C8F88E05B
:10B2500082C085FF25C0328920E0838990E0282BB9
:10B26000392B80913A2A90913B2A820F931F909319
:10B270003B2A80933A2AE0913E21F0E0EE53F54DCF
:10B28000328920E0838990E0282B392B80911B2A7A
:10B2900090911C2A821B930B90931C2A80931B2A4B
:10B2A00020911B2A30911C2A2115310559F08DA1BE
:10B2B00084FD08C08091352A82608093352AC901B7
:10B2C0000E949D51E0913E21F0E0EE53F54D9685B0
:10B2D00080E02785820F911D90934921809348211A
:10B2E00028A139A12817390710F0892B21F43093B0
:10B2F00049212093482180914821909149219F8F95
:10B300008E8F8091352A90E083709070892B09F49C
:10B310006EC110929D2F10929C2F0E94B86A80914E
:10B32000352A282F85FF0CC010929D2F10929C2F3C
:10B330001DA2E0913E21F0E0EE53F54D84E1CCC03A
:10B3400084FF12C010929D2F10929C2F81E090E0FC
:10B350009D8F8C8F84E08DA31FA2E0913E21F0E0B1
:10B36000EE53F54D81E1B8C080919C2F90919D2FB7
:10B37000892B01F120FF02C01D8E1C8E8C8D9D8DAE
:10B380000097A1F42E8D3F8D80919C2F90919D2F41
:10B390002817390720F430939D2F20939C2F8091FC
:10B3A0009C2F90919D2F9D8F8C8F04C090939D2FEB
:10B3B00080939C2F1FA280911D2A90911E2A90930A
:10B3C0003B2A80933A2A80919C2F90919D2F892B24
:10B3D00081F08C8D9D8D009761F0CC9690931C2A06
:10B3E00080931B2AE0913E21F0E0EE53F54D88E179
:10B3F00010C08091352A81FFFAC08CE390E09093D1
:10B400001C2A80931B2AE0913E21F0E0EE53F54D7B
:10B4100080E1858768C08091352A80FFE8C01DA241
:10B4200080E18093352A0E94B86AE1C080911B2A8E
:10B4300090911C2A009711F00E949D51E0913E21AD
:10B44000F0E0EE53F54D85859091352A80FF0BC0D5
:10B4500090FF06C087E08DA31EA21D8E1C8E1DC00E
:10B4600086E08DA31AC090FF22C085E08DA31D8EBB
:10B470001C8EBDC080911B2A90911C2A009711F050
:10B480000E949D51E0913E21F0E0EE53F54D8585FF
:10B4900080FF0DC087E08DA31EA281E090E00E9496
:10B4A0009D5180E18093352A0E94B86A0FC0809137
:10B4B0001B2A90911C2A892B49F499C08091352A26
:10B4C00080FF95C087E08DA31EA291C0E0913E2130
:10B4D000F0E0EE53F54D80E185878CE390E09093AA
:10B4E0001C2A80931B2AE0913E21F0E0EE53F54D9B
:10B4F00080E58487E0913E21F0E0EE53F54D8C89A4
:10B5000080878D8981878E8982878F898387888DBF
:10B510008483898D85838A8D86838B8D878386E05E
:10B520008093A02A88899989918380838A899B89BD
:10B5300093838283A2EBBAE2FE0180E101900D9237
:10B540008150E1F782EA9AE262EB7AE20E941660A9
:10B550008DA1E0913E2184FF06C0F0E0EE53F54D51
:10B560001786168607C0F0E0EE53F54D84E0868717
:10B5700084EC878780911A2A90E027E131E0829F4E
:10B58000F001839FF00D929FF00D1124E751F04DD3
:10B5900084818093A12A80911B2A90911C2A8897EC
:10B5A00090939E2A80911B2A885280939F2AE09133
:10B5B0003E21F0E08F010E53154DD80153961C9299
:10B5C000539752961C92F801118A108A0E94D65005
:10B5D00080959095F801918B808B80E680939A2AD4
:10B5E00010929B2A10929D2A10929C2A08C01092B9
:10B5F0001C2A10921B2A10923E2110923D2110927B
:10B60000352ADF91CF911F910F9108951F931091CB
:10B610001A2A212F30E087E191E0289FF001299F2D
:10B62000F00D389FF00D1124E751F04D83898823E8
:10B6300041F110921A2A0BC082EB9AE20E94B27E6C
:10B640008823C1F480911A2A8F5F80931A2A8091EF
:10B650001A2A823088F328C00E94D27A892B51F4AA
:10B6600080911A2A8F5F80931A2A80911A2A823039
:10B6700098F31DC08091A12A81508093A12A88232C
:10B6800029F410921C2A10921B2A17C08AE99AE208
:10B69000489660E840E050E00E94B55E892B69F072
:10B6A00081E00E94525209C010921A2ADECF1092F5
:10B6B0001C2A10921B2A10931A2A1F9108950F9387
:10B6C0001F93CF93DF938C014091412150914221F0
:10B6D0004F5F5F4F8DE74030580710F040E050E17A
:10B6E000342F252F8091AE2F9091AF2F8217930783
:10B6F00079F38091C72F9091C82F8217930741F358
:10B7000040934121509342211092402120E0A9E131
:10B71000B0E01CC0322F3F5F822F90E08A9FF00183
:10B720008B9FF00D9A9FF00D1124E256F04D808909
:10B730009189892B51F42093402189E1289FD001E0
:10B740001124A256B04D49F434C0232F223010F3F7
:10B7500020934021A0E0B0E02CC050965C9350971D
:10B7600051964C93519753967C936E935297011533
:10B77000110531F480E1ED0119928A95E9F707C0CE
:10B78000ED01F80180E1019009928150E1F780918B
:10B790001A2A90E027E131E0829FF001839FF00DAB
:10B7A000929FF00D1124E751F04D848154968C93B3
:10B7B0005497CD01DF91CF911F910F910895CF92B2
:10B7C000DF92EF92FF920F930E943F630E94B68038
:10B7D00080E009C0E82FF0E0EE0FFF1FEA56F54DBC
:10B7E000118210828F5F8230A8F320E04CE250E09B
:10B7F0000DC0822F90E0849FF001859FF00D949FF3
:10B80000F00D1124E25CF54D15A22F5F223088F374
:10B8100080E094E0909342218093412120E049E12F
:10B8200050E00EC0822F90E0849FF001859FF00DC4
:10B83000949FF00D1124E256F04D118A108A2F5F6B
:10B84000223080F3209340210F91FF90EF90DF9002
:10B85000CF900895CF93DF93DC018C918F3F09F057
:10B8600066C011968C911197823009F060C01296D3
:10B870008D919C911397892B09F059C014968D9145
:10B880009C911597892B09F052C016968D919C9129
:10B890001797892B09F04BC018968D919C91199799
:10B8A000892B09F044C01B968C911B97813009F0BD
:10B8B0003EC01C968C911C978F3FC9F51092542165
:10B8C00020911A2A30E040E0CDE1D0E087E191E01C
:10B8D000289FB001299F700D389F700D112423C03F
:10B8E000842F90E08C9FF0018D9FF00D9C9FF00DB8
:10B8F0001124E60FF71FE751F04D81A592A58F5F48
:10B900009F4F81F01D969C911D9786A1981751F429
:10B9100017969C91179780A1981721F44093542172
:10B9200081E006C04F5F4830D8F24093542180E058
:10B93000DF91CF91089540E020E030E0FC01E20F7C
:10B94000F31F5081FB01E20FF31FE0815E1731F41A
:10B95000485F2F5F3F4F403889F70AC0E527842FA3
:10B96000885FE7FD05C04F5F481711F0EE0FF9CF74
:10B97000842F089589EE9FE20895E0911A2AF0E05D
:10B98000DF01AB5ABE4D1C92EE0FFF1FDF01A55A1F
:10B99000BE4D6D917C91E95AFE4D808191810E944E
:10B9A000CF7608950E94DFAEAA2797FDA095BA2F03
:10B9B000BC01CD0120E838E046EF57E10E940BAD15
:10B9C0009B01AC012058324C4243544FB901CA018B
:10B9D00008954F925F926F927F928F929F92BF9243
:10B9E000CF92DF92EF92FF920F931F9380911A2ACA
:10B9F00090E039EEC32E3FE2D32E27E1422E21E024
:10BA0000522E849DF001859DF00D949DF00D112422
:10BA1000EC0DFD1D65817681878190850E94A7A62A
:10BA200020E030E040E05FE30E9429A50E9453A39C
:10BA30003B014C010E94DFAEB82E0E94DFAEFB2C12
:10BA4000EE24E80EF91E00E010E080911A2A90E042
:10BA50009C01249DC001259D900D349D900D1124C5
:10BA6000C80ED91EF60165817681878190850E9476
:10BA7000A7A60E9453A39B01AC01C801B7010E9475
:10BA80000BAD9B01AC01260D371D481D591DB90199
:10BA9000CA011F910F91FF90EF90DF90CF90BF9060
:10BAA0009F908F907F906F905F904F9008951F931D
:10BAB000CF93DF939C0110911A2AA12FB0E0FD01D2
:10BAC000EB5AFE4D8081882309F04AC021153105CB
:10BAD00091F0CFE5D1E2F90180E101900992815026
:10BAE000E1F7FD01EE0FFF1FE95AFE4D8FE591E2F0
:10BAF0009183808307C0FD01EE0FFF1FE95AFE4DC1
:10BB0000118210826115710591F0CFE6D1E2FB013F
:10BB100080E1019009928150E1F7FD01EE0FFF1FD6
:10BB2000E55AFE4D8FE691E29183808307C0FD01C7
:10BB3000EE0FFF1FE55AFE4D11821082AB5ABE4D2B
:10BB400081E08C930E94DFAE6FEF7FE70E94F8AC3C
:10BB5000AC01662757FD6095762F812F0E94B48235
:10BB6000DF91CF911F910895EF92FF920F931F9352
:10BB70000E94D25C7B018C01E0911A2AF0E0EE5A1F
:10BB8000FE4D8081833078F481E0E81684E2F80687
:10BB900084EF080780E0180730F0E12C24E2F22E51
:10BBA00024EF022F112D80E090E060E070E00E9411
:10BBB000CF7680911A2AE82FF0E0EE5AFE4D908160
:10BBC0009F5F9083B801A7010E94F1821F910F919E
:10BBD000FF90EF90089580911A2AA82FB0E087E196
:10BBE00091E0A89FF001A99FF00DB89FF00D1124DE
:10BBF000E751F04D84898823E1F0AE5ABE4D8C9117
:10BC00008823B9F40E94D25CAC01CB01DA01AC010B
:10BC1000BD01413084E2580784EF680780E078076F
:10BC200020F040E054E264EF70E080911A2A0E9414
:10BC3000F18208951F9310911A2AE12FF0E0E05B42
:10BC4000FE4D8081882399F40E94DFAEAA2797FDDC
:10BC5000A095BA2FBC01CD0120E834E84EE150E0B8
:10BC60000E942DADAB01BC01812F0E942E831F913C
:10BC700008950E94D27A892BD1F4E0911A2AF0E03B
:10BC8000E05BFE4D8081843090F40E94E56F8091EE
:10BC90001A2AE82FF0E0E05BFE4D90819F5F9083D1
:10BCA00040E45BE46CE470E00E942E830895809190
:10BCB0001A2A0E947182E0911A2AF0E0E05BFE4DA0
:10BCC00010820E9478670895AF92BF92CF92DF9260
:10BCD000EF92FF921F93CF93DF936C011092542148
:10BCE00080911A2A90E03DE1A32EB12C27E131E0AA
:10BCF000829F7001839FF00C929FF00C112427C04B
:10BD0000812F90E08A9D90018B9D300D9A9D300D82
:10BD100011242E0D3F1DF901E751F04DEF01A996B9
:10BD200081A592A58F5F9F4F79F0C9018E5F9F4CCF
:10BD3000B60140E150E00E9422B0009729F48FEF55
:10BD40009FEF9983888307C01F5F10935421109140
:10BD500054211830A8F2DF91CF911F91FF90EF90FE
:10BD6000DF90CF90BF90AF900895AF92BF92CF92E7
:10BD7000DF92EF92FF920F931F93CF93DF936C01AB
:10BD8000062F7A011092542120911A2A30E006954C
:10BD9000069506954DE1A42EB12C87E191E0289FF0
:10BDA000E001299FD00D389FD00D112438C0212FDC
:10BDB00030E02A9DF0012B9DF00D3A9DF00D1124ED
:10BDC000EC0FFD1FE751F04D81A592A58F5F9F4FAE
:10BDD00019F184A995A98E159F0519F0E114F104B4
:10BDE000D9F42A9DC0012B9D900D3A9D900D1124F0
:10BDF0008C0F9D1F8E5F9F4CB601402F50E00E941C
:10BE000022B0009749F48DE1189F900111242C0F66
:10BE10003D1F2E5F3F4C09C01F5F109354211091AE
:10BE20005421183020F220E030E0C901DF91CF9199
:10BE30001F910F91FF90EF90DF90CF90BF90AF9048
:10BE400008951F93CF93DF93BC0110911A2AE12F1D
:10BE5000F0E0EE0FFF1FE65BFE4D8081918140E137
:10BE600050E00E9422B00097B9F4812F0E947D8299
:10BE7000A0911A2AB0E0FD01EE0FFF1FE65BFE4D18
:10BE8000208131818FEF9FEFE901998B888B11829F
:10BE90001082A25BBE4D1C92DF91CF911F9108953D
:10BEA0001F93DC0150968D919C915197892B09F538
:10BEB00010911A2AE12FF0E0EE0FFF1FE65BFE4D16
:10BEC00080819181892BA9F4B183A0830E94DFAE88
:10BED000AA2797FDA095BA2FBC01CD0120E834E830
:10BEE0004EE150E00E942DADAB01BC01812F0E94BC
:10BEF000C4831F9108951F93CF93DF9320911A2A33
:10BF0000A22FB0E0FD01EE0FFF1FE65BFE4D40816A
:10BF100051814115510509F485C0C7E1D1E0AC9FBD
:10BF2000F001AD9FF00DBC9FF00D1124E751F04DD5
:10BF3000A25BBE4D9C91808D981748F580E090E003
:10BF400060E070E00E94067110911A2A212F30E003
:10BF5000F901E25BFE4D80818F5F80832C9FF001B1
:10BF60002D9FF00D3C9FF00D1124E751F04D65859C
:10BF700076858785908928EE33E040E050E00E9486
:10BF8000C5ACAB01BC01812F0E94C4834BC0822F82
:10BF90000E947D8220911A2A30E0F901EE0FFF1FE6
:10BFA000E65BFE4DA081B18181E090E051969C93CB
:10BFB0008E93509711821082F901E25BFE4D108240
:10BFC0001092542140E0ADE1B0E02C9FB0012D9FD4
:10BFD000700D3C9F700D112421C0242F2F5F842FE2
:10BFE00090E08A9FF0018B9FF00D9A9FF00D112435
:10BFF000E60FF71FE751F04D81A592A5892B69F453
:10C00000409354218DE1489FC0011124860F971F52
:10C010008E5F9F4C0E94505F05C0422F4830E8F26F
:10C0200040935421DF91CF911F9108955F926F92B9
:10C030007F928F929F92AF92BF92CF92DF92EF92B8
:10C04000FF920F931F93CF93DF93682E592E7B019E
:10C05000FB0180818E3F21F48181803821F465C00D
:10C060008F3F09F462C081E080935421CC2400E02A
:10C07000EDE18E2E912C77E1A72E71E0B72E69E0CD
:10C08000762E4CC080911A2A90E02D2D30E0289D0C
:10C09000E001299DD00D389DD00D11248A9DB0015D
:10C0A0008B9D700D9A9D700D11246C0F7D1FFB01EF
:10C0B000E751F04D81A592A5019759F56E5F7F4C30
:10C0C000C7010E949B5C182F8C1518F160911A2AE9
:10C0D000862F90E09C012A9DC0012B9D900D3A9DDA
:10C0E000900D11248C0F9D1F679DB00111246D5D73
:10C0F000754D8E5F9F4C0E941F41882341F08091B7
:10C100001A2A813021F458E0C52EC10E01C0C12E7B
:10C110000D2D809154218F5F80935421D090542114
:10C1200037E03D1508F0AECF44C0109254210DE128
:10C1300010E0C7E1D1E049E0F42E36C060911A2A40
:10C14000262F30E090E0809FA001819F500D909FAE
:10C15000500D11242C9FC0012D9F900D3C9F900DE0
:10C160001124480F591FFA01E751F04D818D8E3F80
:10C17000B1F4828D803899F46F9DB00111246D5D0A
:10C18000754DCA018E5F9F4C0E941F41882339F074
:10C1900080911A2A813019F4009154210AC08091AB
:10C1A00054218F5F8093542180915421883030F244
:10C1B00000E0402F50E020911A2A30E08DE190E01D
:10C1C000489FF001499FF00D589FF00D112487E121
:10C1D00091E0AC01249FC001259F900D349F900DEC
:10C1E0001124E80FF91F262D352DC901DC01EE5F62
:10C1F000FF4C80E101900D928150E1F7DF91CF91EA
:10C200001F910F91FF90EF90DF90CF90BF90AF9074
:10C210009F908F907F906F905F900895CF93DF9362
:10C22000FC01DB0118968C911897883039F4EF01E6
:10C2300028960D9009928150E1F71BC08630E9F4F1
:10C240009F01285F3F4FAB0183E0EA010990AE01F7
:10C25000E90109929E018150C1F78FEF83878EEF2C
:10C260008487EF012D96139683E00D9009928150FB
:10C27000E1F7808592E0892714C08230B1F41196ED
:10C280008C91119787878C91868715868EEF84878E
:10C290008FEF8387128680911832818780911732C1
:10C2A0008D7F8087DF91CF9108958FEF9FEF0E9460
:10C2B000DD647F928F929F92AF92BF92CF92DF9276
:10C2C000EF92FF920F931F93CF93DF93882E792ED7
:10C2D00069017A010130110519F4603409F0C6C012
:10C2E0001092542190901A2AA92CBB2440E0ADE171
:10C2F000B0E087E191E0A89EB001A99E700DB89EC4
:10C30000700D1124AEC0C42FD0E0542F5F5FCA9FC0
:10C310009001CB9F300DDA9F300D1124260F371F6F
:10C32000F901E751F04D81A592A58F5F9F4F09F06C
:10C3300097C040935421F901EE5FFF4C882D972D53
:10C340009C01D90180E10D9001928150E1F701300B
:10C35000110501F58DE190E09C01C29FC001C39FD2
:10C36000900DD29F900D112427E131E0A901A49EE8
:10C370009001A59E300DB49E300D1124820F931FA5
:10C3800069E0969EB00111246D5D754D8E5F9F4CE6
:10C390000E940E6180911A2A90E02091542130E091
:10C3A000FDE1AF2EB12C2A9DA0012B9D500D3A9D91
:10C3B000500D1124C7E1D1E0BC016C9FC0016D9FFD
:10C3C000900D7C9F900D1124480F591FFA01E751E1
:10C3D000F04D12A611A615AB04ABC114D104E104B3
:10C3E000F10411F1CA018C5E9F4CB701A6010E94B5
:10C3F00040822091542130E080911A2A90E02A9DB9
:10C40000F0012B9DF00D3A9DF00D11249C012C9F05
:10C41000C0012D9F900D3C9F900D1124E80FF91F36
:10C42000E751F04D13AA02C081E083AB8091542103
:10C430002DE1829FC001112420911A2A30E047E1AA
:10C4400051E0B901649F9001659F300D749F300DDC
:10C450001124820F931F8E5F9F4C0E94505F06C075
:10C46000452F483008F44FCF40935421DF91CF91AE
:10C470001F910F91FF90EF90DF90CF90BF90AF9002
:10C480009F908F907F900895EF92FF920F931F934C
:10C49000CF93DF9381E0809354210DE110E0C7E159
:10C4A000D1E0EE24EA94FE2C47C080911A2A90E055
:10C4B00030E0209FA001219F500D309F500D11248E
:10C4C0009C012C9FC0012D9F900D3C9F900D11242D
:10C4D000480F591FFA01E751F04D81A592A58F5FD2
:10C4E0009F4F29F183A9813011F1CA018C5E9F4CC5
:10C4F0000E941782892BD9F02091542130E080913D
:10C500001A2A90E0209FF001219FF00D309FF00D3E
:10C5100011249C012C9FC0012D9F900D3C9F900DDC
:10C520001124E80FF91FE751F04DF2A6E1A6809122
:10C5300054218F5F8093542120915421283008F496
:10C54000B4CFDF91CF911F910F91FF90EF9008959D
:10C550009F92AF92BF92CF92DF92EF92FF920F9392
:10C560001F93DF93CF93CDB7DEB7E2970FB6F89462
:10C57000DEBF0FBECDBF109254210DE1A02EB12C15
:10C5800017E1E12E11E0F12E8E010F5F1F4FB8E28F
:10C59000CB2EB8E0DB2EADE19A2E5AC02E2F30E024
:10C5A00080911A2A90E02A9DF0012B9DF00D3A9D72
:10C5B000F00D1124AC014E9DC0014F9D900D5E9D6C
:10C5C000900D1124E80FF91FE751F04D81A592A5B8
:10C5D0005FEF8F3F9507B9F1ADB7BEB718970FB6AC
:10C5E000F894BEBF0FBEADBFEDB7FEB73196129641
:10C5F0001C930E931197D382C28235832483978331
:10C6000086830E94A1B12DB73EB7285F3F4F0FB67A
:10C61000F8943EBF0FBE2DBF60915421699DB001BB
:10C62000112480911A2A90E0AC014E9DC0014F9DCB
:10C63000900D5E9D900D1124680F791F6E5F7F4CE9
:10C64000C8010E949187809154218F5F809354216B
:10C65000E0915421E83008F4A1CFE2960FB6F894A7
:10C66000DEBF0FBECDBFCF91DF911F910F91FF9025
:10C67000EF90DF90CF90BF90AF909F9008955F9222
:10C680006F927F928F929F92AF92BF92CF92DF92E2
:10C69000EF92FF920F931F93CF93DF933B014C01D7
:10C6A000142F522EE60180911A2A90E027E1A22E43
:10C6B00021E0B22E8A9D60018B9DD00C9A9DD00CFA
:10C6C000112429EE3FE2C20ED31E80E095E0A0E0E7
:10C6D000B0E0F60180839183A283B38380E48483F6
:10C6E00080E395E7A0E0B0E085839683A783B087D9
:10C6F0000E94E95CF6016187728783879487809145
:10C700001A2A90E09C012A9DC0012B9D900D3A9D14
:10C71000900D1124FC01E751F04D28EE33E040E08C
:10C7200050E0258736874787508B21E0208F728A1B
:10C73000618A138A148B558A068B278B86509F4CEF
:10C74000B70146E050E00E946FB0F0901A2A6F2DBA
:10C7500070E020E00DE110E06A9DA0016B9D500D9E
:10C760007A9D500D1124AFEFBFEF10C0822F90E0E3
:10C77000809FF001819FF00D909FF00D1124E40F38
:10C78000F51FE751F04DB2A7A1A72F5F283070F336
:10C790009B0183E0220F331F8A95E1F7A901460F21
:10C7A000571FFA01ED5DF54D88858087E0E00BC0ED
:10C7B000F0E0DA01AE0FBF1FAD5DB54DEC0FFD1F10
:10C7C00080818C93E92F9E2F9F5F8885E81780F3E7
:10C7D000E0935421C7E1D1E06C9FA0016D9F500D03
:10C7E0007C9F500D1124DA01A751B04DAF5FBE4FB1
:10C7F0009FEF9D9382E08D931D921D921D921D923D
:10C800001D921D921D921D921D9211E01D939D93EC
:10C81000F901E60FF71FED5DF54D8085E80FF11D7D
:10C82000339781918D9381918D9380818C93A051C9
:10C83000B140552009F45AC08EEF90E85A969C9367
:10C840008E9359975C961C921E925B975E961C92F3
:10C850001E925D9790961C921E925F9792961C92E4
:10C860001E92919794961C921E92939796961C9264
:10C870001E92959798961C921E92979769E0F69E45
:10C88000B00111246D5D754DCA018E5F9F4C0E94F1
:10C890000E6180911A2A90E0FC01EC9FC001ED9F8F
:10C8A000900DFC9F900D1124FC01E751F04D12A654
:10C8B00011A623E030E035AB24AB13AB8E5F9F4C69
:10C8C0000E94505F0E941A5E6114710481049104F9
:10C8D00069F080911A2A90E08C9FF0018D9FF00DF5
:10C8E0009C9FF00D1124E751F04D138B80911A2A73
:10C8F00040E452E46FE070E00E946B83DF91CF91DF
:10C900001F910F91FF90EF90DF90CF90BF90AF906D
:10C910009F908F907F906F905F90089541E00E946C
:10C9200065880895CF93DF93EC018881833319F4F0
:10C930008981833389F020E030E0FE01E20FF31FAC
:10C94000D901AD5DB54D90818C91981799F42F5F09
:10C950003F4F2630310589F78C859D8586589D4D42
:10C9600049F410921A2A6E507040CE010E9640E0A3
:10C970000E946588DF91CF910895CF93DF93209136
:10C980001A2AE22FF0E0DF0124E0AA0FBB1F2A954C
:10C99000E1F7AC57B84CEC0180E109900D92815061
:10C9A000E1F784E0EE0FFF1F8A95E1F7EC57F84CB2
:10C9B0008FEF8787DF91CF910895FFCF0F931F935C
:10C9C000CF93DF9380911B2A90911C2A009709F442
:10C9D00058C18150954008F045C18091B22A90918C
:10C9E000B32A892B59F58091B42A9091B52A892BC5
:10C9F00029F58091B62A9091B72A892BF9F4809174
:10CA0000B82A9091B92A892BC9F48091BA2A9091B9
:10CA1000BB2A892B99F48091BC2A9091BD2A892B3D
:10CA200069F48091BE2A9091BF2A892B39F48091B4
:10CA3000C02A9091C12A892B09F414C18091B22A8D
:10CA40008F3F09F414C180911A2A813071F48091CA
:10CA5000640390916503892B41F482EB9AE20E9472
:10CA6000B27E882311F410921A2A82EB9AE20E9475
:10CA7000B27E882331F082EB9AE20E94807FEC0143
:10CA800014C080911A2A813041F4809164039091FE
:10CA90006503892B11F410921A2A0E94D27AFC01A4
:10CAA000009709F4DFC0C081D181209739F08A8DC9
:10CAB0009B8D8530910509F065C00BC082EB9AE231
:10CAC00060E070E040E020E030E00E94E57FEC01B3
:10CAD00002C01B8E1A8E88A9882329F010921B325F
:10CAE00010921A3218AA80911A3290911B32892B17
:10CAF000A9F42EE132E33FA72EA740911B2A5091C3
:10CB00001C2A40931A3250931B32EAE9FAE2C90117
:10CB1000BF010E942FB080911B2A88AB82EA9AE263
:10CB200060E840E050E00E94B55E892B19F082EA8F
:10CB30009AE202C080E090E060E070E0AE010E9406
:10CB4000067180911A2A90E027E131E0829FF0017E
:10CB5000839FF00D929FF00D1124E751F04D6585F4
:10CB600076858785908928EE33E040E050E00E948A
:10CB7000C5ACAB01BC01CE0184960E94408281E02D
:10CB80008CA775C0009729F588A9882329F01092F1
:10CB90001B3210921A3218AA80911A3290911B32CD
:10CBA000892B09F06EC02EE132E33FA72EA74091FA
:10CBB0001B2A50911C2A40931A3250931B32EAE9E7
:10CBC000FAE2C901BF010E942FB080911B2A88ABF5
:10CBD00058C0029761F483E090E09B8F8A8FCE016A
:10CBE0004C9640E45BE46CE470E00E9440828091EB
:10CBF0001A2A90E027E131E0829FF001839FF00D37
:10CC0000929FF00D1124E751F04D6585768587855B
:10CC1000908928EE33E040E050E00E94C5ACAB01C3
:10CC2000BC01CE0184960E9440828E01005F1F4F9E
:10CC3000C8010E94918148A94423A1F040931B2A76
:10CC400010921C2A2AE93AE26EA57FA5C90150E09C
:10CC50000E942FB010921B3210921A3218AAC801EB
:10CC60000E94918110921C2A10921B2A0AC080E017
:10CC700090E00E94918110921C2A10921B2A10921F
:10CC80003E21DF91CF911F910F9108950F931F9334
:10CC9000DF93CF93CDB7DEB760970FB6F894DEBFC2
:10CCA0000FBECDBF8C016436710520F0FC011082EF
:10CCB00080E035C0FB01EC55F84C8081882319F4E5
:10CCC000F80110822CC04091463150914731DE016D
:10CCD000119620E030E04130510519F4EDE1F0E02B
:10CCE00002C0E0E0F0E0C901880F991FE80FF91FCA
:10CCF000E75EFE4C808191818D939D932F5F3F4F26
:10CD00002730310541F7CB010E94B651988B8F87B0
:10CD1000C801BE016F5F7F4F0E94918781E06096DE
:10CD20000FB6F894DEBF0FBECDBFCF91DF911F913C
:10CD30000F910895CF92DF92EF92FF920F931F937E
:10CD4000DF93CF9300D0CDB7DEB710921A2A02EB53
:10CD50001AE28FEF92E09093B32A8093B22A109256
:10CD6000B52A1092B42A1092B72A1092B62A1092BD
:10CD7000B92A1092B82A1092BB2A1092BA2A10929D
:10CD8000BD2A1092BC2A1092BF2A1092BE2A80E0BF
:10CD900092E09093C12A8093C02A98EEE92E9FEFEB
:10CDA000F92EE00EF11E89E0D70197968C93C80109
:10CDB0004097B8010E94166010923E2180E6809351
:10CDC0009A2AF70111821382128281E186832FEF62
:10CDD000278380E1C82ED12CC00ED11E82E099E0BD
:10CDE000D60113969C938E9312979093C32A8093A7
:10CDF000C22A80E094E315969C938E93149717961D
:10CE00001C921E921697085E1F4F82E08093CA2ADA
:10CE100081E0F801818313821282278B158A148A9C
:10CE2000168A80911A2A90E027E131E0829FA001C2
:10CE3000839F500D929F500D1124FA01E751F04D40
:10CE400084A995A9892BB1F0D701D496FA01EE5F98
:10CE5000FF4C80E101900D928150E1F781E08093D9
:10CE60001A2A0E944B7B10921A2AFC01B29681A1C9
:10CE700081FD05C010921C2A10921B2A2EC022EEA2
:10CE80003AE2AF0180E1DA010D90AD01D9010D92D6
:10CE90009D018150C1F78089F80182A711A610A6D3
:10CEA00081E083A78CE590E090931C2A80931B2A55
:10CEB00084E390E09A8389838A81D70114968C93C6
:10CEC0001497898115968C930E94DA5080959095DD
:10CED000F601978386830E94DE640F900F90CF91B6
:10CEE000DF911F910F91FF90EF90DF90CF90089509
:10CEF0000F931F930E94D27A892B59F580911A2A99
:10CF0000E82FF0E034E0EE0FFF1F3A95E1F7EC5721
:10CF1000F84C87858823E9F01786CF0160E420E08C
:10CF200030E040E050E001E00E94E97C80911A2A64
:10CF300090E024E0880F991F2A95E1F78C57984CD0
:10CF400060E420E030E040E050E001E010E00E94CA
:10CF5000596180911A2A90E007E111E0809FF00169
:10CF6000819FF00D909FF00D1124E751F04D8389C2
:10CF70008823A1F00E94D27A892B71F080911A2A1D
:10CF800090E0809FF001819FF00D909FF00D1124A3
:10CF9000E751F04D128A118A0E94EB5D0E94A8624F
:10CFA0001F910F91089580911A2A813071F4809118
:10CFB0004631909147318F5F9F4F09F186E391E3AE
:10CFC0000E94B6410E945003089580911331882336
:10CFD000B1F480914631909147318F5F9F4F79F442
:10CFE00080912F30909130308F5F9F4F41F0809132
:10CFF000FE2F882321F08FE190E30E94B64108952F
:10D000008091632A882359F08EE39AE290933D2A17
:10D0100080933C2A82E00E9452520E94DE648091FA
:10D020008F2A882359F08AE69AE290933D2A8093CA
:10D030003C2A82E00E9452520E94DE6408950F93BF
:10D040001F93DF93CF93CDB7DEB769970FB6F894F0
:10D05000DEBF0FBECDBF8C01E62F623708F03DC0AA
:10D0600080914631909147310197B9F580911C32FA
:10D0700090911D32892B89F580917F21882369F554
:10D0800060931C3210921D3220E237E3C901BA01CD
:10D090004E2F50E00E942FB081E080931A2A80EF3B
:10D0A00093EB9A8B898B9C8B8B8B80E48D8BDE0131
:10D0B0001196E6E3F1E380E101900D928150E1F7F2
:10D0C0001F87088BCE0101969093392A8093382AC6
:10D0D00085E00E9452520E94DE6469960FB6F89471
:10D0E000DEBF0FBECDBFCF91DF911F910F9108958D
:10D0F0008091352A883081F5E0911C32F0911D3203
:10D10000309709F44FC020E237E380911D2A9091B7
:10D110001E2AB901AF010E942FB080911C3290915C
:10D120001D32E0911D2AF0911E2AE80FF91F2DE013
:10D1300020830196E0911D2AF0911E2AE80FF91F25
:10D140002AE02083019690939D2F80939C2F10922C
:10D150001D3210921C320895823021F581E08093B7
:10D160007F21E0911D2AF0911E2A80911B2A909127
:10D170001C2AE80FF91F108200D000D088E398E045
:10D18000EDB7FEB79283818380911D2A90911E2A6C
:10D19000948383830E9430B110927F210F900F906F
:10D1A0000F900F900895CF92DF92EF92FF920F931E
:10D1B0001F93CF93DF93D82EC62E79018A01109248
:10D1C0003E21A2E8B1E2E2EBFAE280E101900D92A9
:10D1D0008150E1F780911B2A90911C2AC096909370
:10D1E0001C2A80931B2A8150954030F080E095E006
:10D1F00090931C2A80931B2A6AE97AE240911B2AA9
:10D2000050911C2A40535040CB01C0960E9438B028
:10D2100080E680939A2A10929B2A10929D2A10925F
:10D220009C2A8AE38093A02A80911A2A90E027E121
:10D2300031E0829FF001839FF00D929FF00D112449
:10D24000E751F04D84818093A12A8091A22A909188
:10D25000A32A892B51F58091A42A9091A52A892B84
:10D2600021F58091A62A9091A72A892BF1F480912B
:10D27000A82A9091A92A892BC1F48091AA2A909179
:10D28000AB2A892B91F48091AC2A9091AD2A892BFD
:10D2900061F48091AE2A9091AF2A892B31F480916C
:10D2A000B02A9091B12A892BD1F0E2EBFAE2DF01AA
:10D2B000509780E10D9001928150E1F78091822199
:10D2C0008F3F91F484E0D81651F422E0C21639F46D
:10D2D00082EA9AE262E871E20E9416600EC0109241
:10D2E0001C2A10921B2A35C0A2EABAE2E2E8F1E257
:10D2F00080E101900D928150E1F7E0913E21CE2F27
:10D30000D0E0FE01EE53F54DD082C182C801B701D5
:10D310000E94BA51CA53D54D688379838A839B830F
:10D3200080911B2A90911C2A889790939E2A889618
:10D33000885280939F2A80913E21C82FD0E0CE53FF
:10D34000D54D1B821A820E94D250809590959B8366
:10D350008A83DF91CF911F910F91FF90EF90DF9023
:10D36000CF9008954AE95AE280911A2A90E027E185
:10D3700031E0829FF001839FF00D929FF00D112408
:10D38000E751F04D84818093A12A8091B22A8F3F8A
:10D3900081F4DA015896FA01389680E101900D92F5
:10D3A0008150E1F782EA9AE262EB7AE20E9416602B
:10D3B0001BC0A2E8B1E2FA01389680E101900D921B
:10D3C0008150E1F7E2EAFAE2DF01509680E10D9048
:10D3D00001928150E1F7A2EBBAE2E2E8F1E280E1EA
:10D3E00001900D928150E1F760913E21662301F199
:10D3F0008AE38093A02A70E040911B2A50911C2A56
:10D40000461B570B50931C2A40931B2A48525040EE
:10D4100050939E2A485D5F4F842F885280939F2AA5
:10D420006A53754D4C52504086EC9AE20E9438B0D7
:10D4300010923E2181E88093C22A1092C32A109252
:10D44000C52A1092C42A0E94D2508095909590933C
:10D45000C52A8093C42A08950F931F93CF93DF9317
:10D4600020E620939A2A10929B2A10929D2A1092CD
:10D470009C2A2AE32093A02A20911A2A30E047E12F
:10D4800051E0249FF001259FF00D349FF00D1124F1
:10D49000E751F04D24812093A12AA2EBBAE2FC01CE
:10D4A00080E101900D928150E1F782EA9AE262EB0D
:10D4B0007AE20E9416608AE38093A02A80E390E0DB
:10D4C00090931C2A80931B2A809180219091812126
:10D4D0000196909381218093802120913E21C22F3B
:10D4E000D0E0CA53D54D198218820E94B6519B8351
:10D4F0008A8380913E21482F50E020911B2A309151
:10D500001C2AFA01EA53F54D81E6848331968F5F38
:10D510008138D9F7C901809690931C2A80931B2AE1
:10D520002850304030939E2A885280939F2A8A0147
:10D530000E53154D80E8F801808311821382128208
:10D540000E94D25080959095F801938382838091B8
:10D55000802190918121DF91CF911F910F910895AA
:10D56000FC0171A760A70895FC01768B658B089577
:10D57000A0913C2AB0913D2A109719F0FD01B89670
:10D5800005C0E091382AF091392A75968091352AA4
:10D5900086FF22C050962D913C9151978091942105
:10D5A000909195218217930731F480919621909163
:10D5B0009721009769F48091982190919921821781
:10D5C000930751F480919A2190919B21009721F02B
:10D5D000918380831382128220813181211531054C
:10D5E00021F082819381F90109950895009749F00E
:10D5F00090933D2A80933C2A83E00E9452520E94DD
:10D60000DE640895009749F09093392A8093382A70
:10D6100085E00E9452520E94DE640895CF93DF930A
:10D62000EC0180919621909197218C179D0771F4C0
:10D6300080919421909195210E946451109295219E
:10D6400010929421109297211092962180919A2104
:10D6500090919B218C179D0771F480919821909156
:10D6600099210E9464511092992110929821109250
:10D670009B2110929A21E3E6FAE2838194818C1730
:10D680009D0719F4148213821082BC96CF018597EE
:10D6900086599A4290F3EEE9FFE2858996898C17C4
:10D6A0009D0711F4118A108A79968FE2E03DF80700
:10D6B000A0F3DF91CF910895AC0110929321E4E99A
:10D6C000F1E220E014C0808191818417950769F40C
:10D6D000828193818617970741F4209393211182C9
:10D6E0001082CA010E946451089534962F5F22303F
:10D6F00050F3209393210895CF93DF93EA010E9482
:10D700005F5BFC01009711F0D68BC58BCF01DF91D9
:10D71000CF910895EF92FF920F931F93DF93CF93D2
:10D72000CDB7DEB760970FB6F894DEBF0FBECDBFA2
:10D730008C017B018FEF92E09A8389831C821B828C
:10D740001E821D8218861F821A8619861C861B86D9
:10D750001E861D8680E091E0988B8F87CE01019612
:10D76000B8010E945F5BFC01009721F0F68AE58A10
:10D77000118B008BCF0160960FB6F894DEBF0FBE01
:10D78000CDBFCF91DF911F910F91FF90EF90089542
:10D79000AC0110929221E4E9F1E220E012C0322FB4
:10D7A0003F5F80819181892B51F420939221518395
:10D7B000408373836283CA010E9481510895349625
:10D7C000232F223060F32093922108950F931F930B
:10D7D000CF93DF938A010E94DE50EC01009721F085
:10D7E00019A708A70E94F66ACE01DF91CF911F9179
:10D7F0000F9108959F92AF92BF92CF92DF92EF92D6
:10D80000FF920F931F93CF93DF9380911A2A90E09A
:10D8100027E131E0829FE001839FD00D929FD00DE0
:10D820001124C751D04D8F89882309F4C2C3809138
:10D83000A12A8F3F09F0B3C38091A22A8E3F09F03D
:10D84000AEC38091A32A803809F0A9C380913E21FC
:10D85000A82FB0E0FD01EE53F54D8181882309F03A
:10D860009EC3AA53B54D8C9181118C83E0913E21CA
:10D87000F0E0EA53F54D2481358146815781211529
:10D8800031054105510509F448C080911A2A90E0FC
:10D89000C7E1D1E08C9FF0018D9FF00D9C9FF00DB2
:10D8A0001124E751F04DE580F68007811085CA010B
:10D8B000B9010E94BA51E616F7060807190769F17F
:10D8C00000911A2A10E0E0913E21F0E0EA53F54D74
:10D8D00064817581868197810E94BA510C9FF00105
:10D8E0000D9FF00D1C9FF00D1124E751F04D658345
:10D8F00076838783908700911A2A10E00E94E95C62
:10D900000C9FF0010D9FF00D1C9FF00D1124E751AD
:10D91000F04D6187728783879487E0913E21F0E024
:10D92000EA53F54D60857185828593856115710592
:10D9300081059105A1F000911A2A10E00E94BA51C8
:10D9400027E131E0029FF001039FF00D129FF00DDF
:10D950001124E751F04D658776878787908B109269
:10D96000A02110929F211092A2211092A12140E0AB
:10D9700009C0E42FF0E0EE0FFF1FED55FE4D1182C0
:10D9800010824F5F4430A8F34093B3218CE0809322
:10D990009E2160911B2A70911C2A3AC0F901E6561B
:10D9A000F54D8181882309F4F8C28081833071F0BC
:10D9B000853039F08130E1F4F093A021E0939F218C
:10D9C00017C0F093A221E093A12112C040E044309F
:10D9D00079F0542F5F5FE42FF0E0EE0FFF1FED555D
:10D9E000FE4D80819181892B09F4DEC2452FEFCF56
:10D9F00080919E21E0913E21F0E0E656F54DE80F42
:10DA0000F11D95A5990F990F990F980F90939E214D
:10DA100090913E2180919E21282F30E0290F311DC9
:10DA2000245D3F4F2617370708F4B8CF4093B32142
:10DA3000E091A121F091A2213097C1F000911A2A22
:10DA400010E064817581868197810E94BA5127E137
:10DA500031E0029FF001039FF00D129FF00D1124A1
:10DA6000E751F04D60837183828393831092B321D9
:10DA70009924939480C164817581868197810E94E5
:10DA8000BA517B018C01E091B321F0E0EE0FFF1F52
:10DA9000ED55FE4D0190F081E02D60857185828508
:10DAA00093850E94BA51E616F7060807190708F48D
:10DAB0005DC1E091B321F0E0EE0FFF1FED55FE4D8B
:10DAC0000190F081E02D80898E3F21F4818980389A
:10DAD00009F44CC1838187FF7CC0CF0140960E942E
:10DAE000497EEC019093AE218093AD21E091B3216A
:10DAF0000097C1F5F0E0EE0FFF1FED55FE4D0190D0
:10DB0000F081E02D648175818681978161157105B1
:10DB10008105910509F45DC0EF0160966F3F2FEF1D
:10DB200072072FEF82072FEF920771F012810E9488
:10DB3000BA5120E432E44FE050E00E94C5AC9B01B2
:10DB4000AC01CE01612F06C0CE01628120E030E041
:10DB500040E050E000E00E94E97C9093AE21809389
:10DB6000AD2137C0F0E0EE0FFF1FED55FE4D0190E7
:10DB7000F081E02D64817581868197816115710541
:10DB80008105910549F06F3FEFEF7E07EFEF8E07BC
:10DB9000EFEF9E0749F404C0CE010E94467B19C0F6
:10DBA00089A1816089A315C00E94BA5120E432E4A2
:10DBB0004FE050E00E94C5ACAB01BC01CE014196E4
:10DBC0000E944082E091AD21F091AE2181A18E7F33
:10DBD00081A3E091B321F0E0EE0FFF1FED55FE4D64
:10DBE0000190F081E02D838186FFC0C08481958102
:10DBF000A681B7810097A105B10509F4B7C0CF018F
:10DC00004096628141E050E00E94B55EDC01909355
:10DC1000B2218093B121E091B321009709F478C03B
:10DC2000F0E0EE0FFF1FED55FE4D0190F081E02D6D
:10DC300064817581868197816F3FFFEF7F07FFEFDA
:10DC40008F07FFEF9F0709F460C00E94BA5161522D
:10DC50007C418040904040F5E091B321F0E0EE0F30
:10DC6000FF1FED55FE4D0190F081E02D648175811F
:10DC7000868197810E94BA517B018C018091B121EC
:10DC80009091B22142960E94F2815B016C01C80121
:10DC9000B70120E432E44FE050E00E94C5ACA61684
:10DCA000B706C806D90600F50091B1211091B2213E
:10DCB0000E5E1F4FE091B321F0E0EE0FFF1FED5518
:10DCC000FE4D0190F081E02D648175818681978100
:10DCD0000E94BA5120E432E44FE050E00E94C5AC0B
:10DCE000AB01BC01C80109C08091B1219091B22162
:10DCF000429640E058E467E27DEA0E944082E0916B
:10DD0000B121F091B221128E31C05A969C922EC050
:10DD1000F0E0EE0FFF1FED55FE4D0190F081E02D7C
:10DD20006481758186819781EF0160966F3F2FEF47
:10DD300072072FEF82072FEF920771F012810E9476
:10DD4000BA5120E432E44FE050E00E94C5AC9B01A0
:10DD5000AC01CE01612F06C0CE01628120E030E02F
:10DD600040E050E001E010E00E9459618091B32151
:10DD70008F5F8093B321E091B321E43058F4F0E059
:10DD8000EE0FFF1FED55FE4D0190F081E02D309715
:10DD900009F071CE82EA9AE20E94807FFC019093A2
:10DDA000AC218093AB2160919F217091A0216115DE
:10DDB000710509F461C0009771F46E5F7F4F82EACC
:10DDC0009AE241E022E030E00E94E57F9093AC21AE
:10DDD0008093AB2151C0828D938D892B21F482E0F9
:10DDE00090E0938F828F20911A2A822F90E0FC017D
:10DDF00033E0EE0FFF1F3A95E1F7E80FF91FED5DF5
:10DE0000F54DA084213061F4E0919F21F091A02193
:10DE10008181813019F098E0A92E02C082E0A82EFD
:10DE200000919F211091A0210E5F1F4FE090AB2128
:10DE3000F090AC21E7016096C801BE014A2D50E088
:10DE40000E9422B0009721F4F701808DA81671F08E
:10DE5000CE01B8014A2D50E00E942FB0E091AB21D5
:10DE6000F091AC2182E090E0938F828FE091AB2122
:10DE7000F091AC2181E0818FE0913E21F0E0EA5306
:10DE8000F54D82819381E091AB21F091AC21892BFA
:10DE900009F454C0309771F482EA9AE260E070E0CD
:10DEA00041E025E030E00E94E57F9093AC21809333
:10DEB000AB2102C081E0818F8091AB219091AC2198
:10DEC0000E94847A8C019093B0218093AF21E091DD
:10DED0003E210097D9F40091AB211091AC21F0E0E4
:10DEE000EA53F54D828193810E94B651A0E0B0E0E3
:10DEF000BC01CD0120E432E44FE050E00E94C5AC0B
:10DF0000AB01BC01C8010E94C17D25C0F0E0EA530D
:10DF1000F54D828193810E94B651A0E0B0E0BC0132
:10DF2000CD0120E432E44FE050E00E94C5ACAB01EB
:10DF3000BC01C80102960E9440820DC0309759F082
:10DF4000CF010E94847A9093B0218093AF210097F3
:10DF500011F00E943B7BE091AB21F091AC21309716
:10DF6000C9F040A94423B1F040931B2A10921C2A07
:10DF70002AE93AE266A577A5C90150E00E942FB0D0
:10DF800010921B3210921A32E091AB21F091AC2129
:10DF900010AA0FC00E94D36702C04093B321109211
:10DFA0001C2A10921B2A05C02656354D318320832A
:10DFB0001FCDDF91CF911F910F91FF90EF90DF90D8
:10DFC000CF90BF90AF909F900895EF92FF920F93E4
:10DFD0001F93DF93CF9300D0CDB7DEB780911A2A7D
:10DFE000282F30E087E191E0289FF001299FF00D74
:10DFF000389FF00D1124E751F04D8789882309F4EB
:10E00000FCC0F90183E0EE0FFF1F8A95E1F7E20FF4
:10E01000F31FED5DF54D2085822F90E00296022FD3
:10E020000E5F87709070081B892B09F0085F8AE9E2
:10E030009AE220E620939A2A10929B2A10929D2A17
:10E0400010929C2A2AE32093A02A2FEF2093A12A42
:10E05000FC0178962FEF32E03093B32A2093B22A56
:10E0600013821282158214821782168211861086FC
:10E07000138612861586148620E032E037872687BD
:10E080000896BF010E94166020913E21A22FB0E0A9
:10E09000FD01EE53F54D85E880831182FD01EA53C1
:10E0A000F54D108211821282138210929E2A809165
:10E0B000A22A9091A32A892B99F58091A42A909164
:10E0C000A52A892B69F58091A62A9091A72A892BE8
:10E0D00039F58091A82A9091A92A892B09F5809178
:10E0E000AA2A9091AB2A892BD9F48091AC2A9091DD
:10E0F000AD2A892BA9F48091AE2A9091AF2A892B61
:10E1000079F48091B02A9091B12A892B49F488E062
:10E1100080939F2AD096B0931C2AA0931B2A5DC09F
:10E12000E02EFF24822F90E0C0968E0D9F1D9093CD
:10E130001C2A80931B2A085F00939F2A0850A6532D
:10E14000B54DB093A021A0939F2181E08C930695BB
:10E150000695069511960C93119720911A2A1296FE
:10E16000822F90E0FC0103E0EE0FFF1F0A95E1F71C
:10E17000E80FF91FED5DF54D408589E0289F90017E
:10E1800011242D5D354DCD01B90150E00E942FB015
:10E1900080911A2A90E0FC0113E0EE0FFF1F1A9500
:10E1A000E1F7E80FF91FED5DF54D808590E09701EF
:10E1B000281B390B225030403A83298320919F211C
:10E1C0003091A0212E5F3F4F280F391FC90160E019
:10E1D00070E049815A810E944AB080913E21082F07
:10E1E00010E00E53154DF801138212820E94D25096
:10E1F00080959095F801938382830F900F90CF9133
:10E20000DF911F910F91FF90EF900895FF920F9370
:10E210001F93CF93DF938C01EA0180911A2A282F54
:10E2200030E087E191E0289FF001299FF00D389FB1
:10E23000F00D1124E751F04D8789882309F413C1AB
:10E24000F90153E0EE0FFF1F5A95E1F7E20FF31FBC
:10E25000ED5DF54D2085822F90E0029642E0F42E90
:10E26000F20E87709070F81A892B11F088E0F80E82
:10E2700010923E2180E680939A2A10929B2A109257
:10E280009D2A10929C2A8AE38093A02A9FEF909364
:10E29000A12AE2EBFAE261157105B9F49093B22A72
:10E2A00082E0818313821282158214821782168281
:10E2B00011861086128681E0838794878D858587F5
:10E2C0008E859F859787868707C0DF01FB0180E1E8
:10E2D00001900D928150E1F787E88093C22A109255
:10E2E000C32A1092C62A1092C72A1092C82A1092E6
:10E2F000C92AAAECBAE2FE0180E101900D92815098
:10E30000E1F710929E2ACE0160E840E050E00E94C2
:10E31000B55E892B09F070C00115110549F0A2EA1C
:10E32000BAE2F80180E101900D928150E1F706C058
:10E3300082EA9AE262EB7AE20E94166088E1F80EC5
:10E34000F0929F2A88EEF80E0F2D10E0005C1F4F10
:10E3500010931C2A00931B2A00541040A0913E21C8
:10E36000B0E0A652B54DB093A021A0939F2181E0CB
:10E370008C93F694F694F6941196FC921197209152
:10E380001A2A1296822F90E0FC0133E0EE0FFF1F55
:10E390003A95E1F7E80FF91FED5DF54D408589E00D
:10E3A000289F900111242D5D354DCD01B90150E01C
:10E3B0000E942FB080911A2A90E0FC0123E0EE0F1A
:10E3C000FF1F2A95E1F7E80FF91FED5DF54D8085F8
:10E3D00090E0081B190B0250104020919F213091B2
:10E3E000A0212E5F3F4F280F391FC90160E070E068
:10E3F000A8010E944AB029C01092A32A1092A22A12
:10E400001092A52A1092A42A1092A72A1092A62A46
:10E410001092A92A1092A82A1092AB2A1092AA2A26
:10E420001092AD2A1092AC2A1092AF2A1092AE2A06
:10E430001092B12A1092B02A88E180939F2A80E43A
:10E4400090E090931C2A80931B2A80913E21C82F34
:10E45000D0E0CE53D54D1B821A820E94D2508095B7
:10E4600090959B838A83DF91CF911F910F91FF90AD
:10E470000895BF92CF92DF92EF92FF920F931F9376
:10E48000DF93CF93CDB7DEB72B970FB6F894DEBFEF
:10E490000FBECDBF80911A2A90E027E131E0829F24
:10E4A000F001839FF00D929FF00D1124E751F04D84
:10E4B0008789882309F4B1C190913E21E92FF0E0CA
:10E4C000DF01AA53B54DDC908091A12A8F3F09F05E
:10E4D000A0C1EE53F54D8181882309F09AC11496AD
:10E4E0008C9114978F3F09F494C1E0E4BE2EBD20B7
:10E4F000D6FE05C08091B22A8F3F09F48AC184E11B
:10E5000080939E211092A02110929F2160911B2A3E
:10E5100070911C2A292F30E0245D3F4FA9014656F7
:10E52000554D1AC0FC01E656F54D8181882309F44A
:10E5300070C18081823021F4F093A021E0939F216B
:10E5400080919E21FA01E80FF11D9181990F990F99
:10E55000990F980F90939E2180919E21F901E80FC9
:10E56000F11DCF01E617F707E8F2CD01049660E848
:10E5700040E050E00E94B55EFC019093B221809390
:10E58000B121009769F080899189892B09F041C1F7
:10E5900080913E2190E08653954D0E94215F39C1C4
:10E5A00080913E2190E08653954D0E94807F90930C
:10E5B000AC218093AB21892B09F42BC120911A2A1D
:10E5C000822F90E0FC0173E0EE0FFF1F7A95E1F7D8
:10E5D000E80FF91FED5DF54D0085213051F4E09114
:10E5E0009F21F091A0218181813011F008E001C0CC
:10E5F00002E020919F213091A0212E5F3F4FCE015C
:10E600000196B901402F50E00E942FB00987E09099
:10E610009F21F090A021E114F10411F410E018C042
:10E620008091AB219091AC219B878A87BC01605F70
:10E630007F4FC7010296402F50E00E9422B0982FD2
:10E64000EA85FB85808D081711F011E001C0192FB4
:10E6500060E8C62ECD20E091AB21F091AC21828DF7
:10E66000938D009709F045C0E114F10409F4D1C07D
:10E670009F01205F3F4FA7014E5F5F4FC901BA0165
:10E68000402F50E00E942FB0E091AB21F091AC21DF
:10E69000008FE090AB21F090AC21BB2021F181E014
:10E6A00090E0F701938F828F80911A2A90E027E102
:10E6B00031E0829FF001839FF00D929FF00D1124B5
:10E6C000E751F04D618572858385948528EE33E0AE
:10E6D00040E050E00E94C5ACAB01BC01C7014C96C4
:10E6E0000E94408274C082E090E0F701938F828F95
:10E6F0006EC0D5FC0AC0112341F0019709F089C012
:10E7000082E090E0938F828F84C0E114F10489F05D
:10E710009F01205F3F4FA7014E5F5F4FC901BA01C4
:10E72000402F50E00E942FB0E091AB21F091AC213E
:10E73000008FBB2041F1E090AB21F090AC2181E053
:10E7400090E0F701938F828F80911A2A90E027E161
:10E7500031E0829FF001839FF00D929FF00D112414
:10E76000E751F04D618572858385948528EE33E00D
:10E7700040E050E00E94C5ACAB01BC01C7014C9623
:10E780000E94408210C080919F219091A021892BEE
:10E7900051F0112341F0E091AB21F091AC2182E0E6
:10E7A00090E0938F828FE091AB21F091AC21818D2D
:10E7B000882369F0CC2059F4CF010E94847A909389
:10E7C000B0218093AF21009711F00E943B7BE09134
:10E7D000AB21F091AC21C18EE091AB21F091AC2145
:10E7E00040A94423B1F040931B2A10921C2A2AE925
:10E7F0003AE266A577A5C90150E00E942FB01092B9
:10E800001B3210921A32E091AB21F091AC2110AA88
:10E8100004C010921C2A10921B2A2B960FB6F89453
:10E82000DEBF0FBECDBFCF91DF911F910F91FF9043
:10E83000EF90DF90CF90BF900895BF92CF92DF927C
:10E84000EF92FF920F931F93DF93CF93CDB7DEB775
:10E8500029970FB6F894DEBF0FBECDBF50911A2A8C
:10E86000652F70E087E191E0689FF001699FF00DEE
:10E87000789FF00D1124E751F04D8789882309F422
:10E880007EC28091A12A8F3F09F075C280913E21FE
:10E89000282F30E0F901EA53F54D84818F3F09F4C8
:10E8A0006AC2F901EE53F54D8181882309F063C2F4
:10E8B0001092A02110929F2184E180939E210091CB
:10E8C0001B2A10911C2A44E1F901BC9616C0DC01F8
:10E8D000A656B54D11968C911197882309F449C21B
:10E8E0008C91813021F4B093A021A0939F211196A7
:10E8F0008C91880F880F880F480FCF01840F911DCE
:10E900008017910720F340939E21A0919F21B09101
:10E91000A021109709F499C08091A22A9091A32A6E
:10E92000892B59F58091A42A9091A52A892B29F544
:10E930008091A62A9091A72A892BF9F48091A82A80
:10E940009091A92A892BC9F48091AA2A9091AB2A87
:10E95000892B99F48091AC2A9091AD2A892B69F486
:10E960008091AE2A9091AF2A892B39F48091B02AF8
:10E970009091B12A892B09F4FEC1FB0113E0EE0F3F
:10E98000FF1F1A95E1F7E60FF71FED5DF54DB08417
:10E99000513051F411968C911197813019F078E033
:10E9A000B72E02C062E0B62E9D012E5F3F4F8E0152
:10E9B0000F5F1F4FC801B9014B2D50E00E942FB0CF
:10E9C000B98682EA9AE20E94807F7C019093AC2112
:10E9D0008093AB21009749F482EA9AE2B80140E0C3
:10E9E00022E030E00E94E57F30C000919F2110912D
:10E9F000A0210E5F1F4F50E1C52ED12CC80ED91E8D
:10EA0000C801B6014B2D50E00E9422B0009721F4BE
:10EA1000F701808DB81681F0C601B8014B2D50E08A
:10EA20000E942FB0E091AB21F091AC21B08EE0912B
:10EA3000AB21F091AC2105C0F701828D938D892B1C
:10EA400021F482E090E0938F828F80913E2190E0CC
:10EA50008653954D60E840E050E00E94B55E90938B
:10EA6000B2218093B121892B09F485C18091A22A1A
:10EA70009091A32A892B09F074C08091A42A9091C7
:10EA8000A52A892B09F06DC08091A62A9091A72A0A
:10EA9000892B09F066C08091A82A9091A92A892B18
:10EAA00009F05FC08091AA2A9091AB2A892B09F0C6
:10EAB00058C08091AC2A9091AD2A892B09F051C0A1
:10EAC0008091AE2A9091AF2A892B09F04AC080919B
:10EAD000B02A9091B12A892B09F043C082EB9AE2C7
:10EAE0000E942A5C882309F446C1E091B121F0918B
:10EAF000B22180899189892B61F18FEF92E0909307
:10EB0000B32A8093B22A1092B52A1092B42A109296
:10EB1000B72A1092B62A1092B92A1092B82A1092E7
:10EB2000BB2A1092BA2A1092BD2A1092BC2A1092C7
:10EB3000BF2A1092BE2A80E091E09093C12A809370
:10EB4000C02A82EA9AE262EB7AE20E94166050E200
:10EB500055C080913E2190E08653954D0E94215FE3
:10EB60000AC182EA9AE260E840E050E00E94B55EA5
:10EB7000892B09F000C182EB9AE20E942A5C88236B
:10EB8000B9F0E2EBFAE2DF01509780E10D900192DB
:10EB90008150E1F780913E21E82FF0E0A2EABAE24D
:10EBA000E653F54D80E101900D928150E1F725C0CB
:10EBB00082EB9AE260E840E050E00E94B55E20916E
:10EBC000B1213091B2212817390709F0D4C0E2EB06
:10EBD000FAE2DF01509780E10D9001928150E1F758
:10EBE00080913E21E82FF0E0A2EABAE2E653F54D2B
:10EBF00080E101900D928150E1F750E610923E21A4
:10EC000080911A2A282F30E087E191E0289FF001B7
:10EC1000299FF00D389FF00D1124E751F04D8389A5
:10EC200081115068F90143E0EE0FFF1F4A95E1F7AB
:10EC3000E20FF31FED5DF54D2085822F90E00296E7
:10EC4000422F4E5F87709070481B892B09F0485FF8
:10EC500080E680939A2A10929B2A10929D2A109205
:10EC60009C2A10929E2A485E40939F2A48518AE32C
:10EC70008093A02A8FEF8093A12A88E88093C22AEC
:10EC80001092C32A5093C62AAAECBAE22091B1216D
:10EC90003091B221C901FC0180E101900D928150B7
:10ECA000E1F7042F10E0005C1F4F10931C2A009323
:10ECB0001B2A00541040A0913E21B0E0A652B54D51
:10ECC000B093A021A0939F2182E08C934695469516
:10ECD000469511964C93119720911A2A1296822FDD
:10ECE00090E0FC0133E0EE0FFF1F3A95E1F7E80FEB
:10ECF000F91FED5DF54D408589E0289F90011124B5
:10ED00002D5D354DCD01B90150E00E942FB08091AD
:10ED10001A2A90E0FC01A3E0EE0FFF1FAA95E1F78D
:10ED2000E80FF91FED5DF54D808590E0081B190B8C
:10ED30000250104020919F213091A0212E5F3F4F23
:10ED4000280F391FC90160E070E0A8010E944AB095
:10ED500080913E21082F10E00E53154DF8011382CB
:10ED600012820E94D25080959095F80193838283FD
:10ED700006C040939E2110921C2A10921B2A2996AD
:10ED80000FB6F894DEBF0FBECDBFCF91DF911F91BC
:10ED90000F91FF90EF90DF90CF90BF9008956F920A
:10EDA0007F928F929F92AF92BF92CF92DF92EF921B
:10EDB000FF920F931F93DF93CF9300D0CDB7DEB7B1
:10EDC000AC0180911A2A282F30E087E191E0289F3A
:10EDD000F001299FF00D389FF00D1124E751F04DFF
:10EDE0008789882309F420C2F901A3E0EE0FFF1FF1
:10EDF000AA95E1F7E20FF31FED5DF54D2085822F17
:10EE000090E00296E2E0DE2ED20E87709070D81A63
:10EE1000892B11F088E0D80E6115710529F58FEF67
:10EE200092E09093B32A8093B22A1092B52A10925E
:10EE3000B42A1092B72A1092B62A1092B92A1092C8
:10EE4000B82A1092BB2A1092BA2A1092BD2A1092A8
:10EE5000BC2A1092BF2A1092BE2A80E091E09093C3
:10EE6000C12A8093C02A08C0A2EBBAE2FB0180E16C
:10EE700001900D928150E1F74115510549F0A2EA48
:10EE8000BAE2FA0180E101900D928150E1F706C0EB
:10EE900082EA9AE262EB7AE20E94166010923E21C8
:10EEA00080E680939A2A10929B2A10929D2A1092B3
:10EEB0009C2A8AE38093A02A8FEF8093A12A86E878
:10EEC0008093C22AEAE9FAE211A680911A2A90E018
:10EED00007E111E0809FF001819FF00D909FF00D00
:10EEE0001124E751F04D84818093C62A818992894B
:10EEF0000E94B6519093C92A8093C82A80913E21DE
:10EF0000E82EFF24E6ECFAE2EE0EFF1E80911A2AAC
:10EF100090E0809FF001819FF00D909FF00D1124F3
:10EF2000E751F04D65817681878190850E94BA51C5
:10EF3000F701648375838683978380913E21E82E51
:10EF4000FF2486EC9AE2E80EF91E80911A2A90E0DE
:10EF5000809FF001819FF00D909FF00D1124E751EB
:10EF6000F04D65857685878590890E94BA51F701B5
:10EF700060877187828793870D2D10E0085C1F4F93
:10EF800010931C2A00931B2A08531040A0913E2185
:10EF9000B0E0AE52B54DB093A021A0939F2181E087
:10EFA0008C938D2D86958695869511968C931197C9
:10EFB00020911A2A1296822F90E0FC0133E0EE0F86
:10EFC000FF1F3A95E1F7E80FF91FED5DF54D40851C
:10EFD00089E0289F900111242D5D354DCD01B901A7
:10EFE00050E00E942FB080911A2A90E0FC0123E0AB
:10EFF000EE0FFF1F2A95E1F7E80FF91FED5DF54DC4
:10F00000808590E0081B190B0250104020919F2131
:10F010003091A0212E5F3F4F280F391FC90160E0BA
:10F0200070E0A8010E944AB0FCE0DF0ED0929E2161
:10F030000E944B7B7C011092B321B2E29B2EA3E095
:10F040006A2EF0EC7F2EE4E08E2EAA24AA94BA2C2D
:10F050006501C8C0899DF0011124EE0DFF1D81A13D
:10F060008670863009F0B9C080818E3F21F481819D
:10F07000803809F4B2C080913E21082F10E0045D71
:10F080001F4F80919E21482F50E0D801A656B54DC4
:10F09000A40FB51F6C9213967C92139711968C92C5
:10F0A00011972091B321822F90E0FC0175E0EE0FC3
:10F0B000FF1F7A95E1F7880F991FE80FF91FEE0DF2
:10F0C000FF1D808912968C931297299DF0011124BF
:10F0D000EE0DFF1D81A180FF0DC01496AD92BD9273
:10F0E000CD92DC9217971896AD92BD92CD92DC929C
:10F0F0001B9743C0040F151F0656154D6589768969
:10F100008789908D20E432E44FE050E00E940BADFF
:10F11000CA01B9010E94BA51F801648375838683DC
:10F12000978380913E2190919E21092F10E0080F36
:10F13000111D0A53154D8091B32190E0FC0145E06B
:10F14000EE0FFF1F4A95E1F7880F991FE80FF91F8F
:10F15000EE0DFF1D658D768D878D90A120E432E444
:10F160004FE050E00E940BADCA01B9010E94BA51B4
:10F17000F8016087718782879387E0913E21F0E0F4
:10F1800080919E21EA53F54DE80FF11D14861586F6
:10F19000168617868091B32190E0DC0125E0AA0F46
:10F1A000BB1F2A95E1F7880F991FA80FB91F70960A
:10F1B000AE0DBF1D80E10D9001928150E1F780916D
:10F1C0009E21805E80939E2180911B2A90911C2A13
:10F1D000809690931C2A80931B2A8091B3218F5F85
:10F1E0008093B3218091B321843008F433CF809190
:10F1F0001B2A90911C2A88979A8389838A818093FD
:10F200009E2A898180939F2A80913E21082F10E0B9
:10F210000E53154DF801138212820E94D250809530
:10F220009095F801938382830F900F90CF91DF9197
:10F230001F910F91FF90EF90DF90CF90BF90AF9014
:10F240009F908F907F906F900895BF92CF92DF92A2
:10F25000EF92FF920F931F93DF93CF93CDB7DEB75B
:10F2600069970FB6F894DEBF0FBECDBF50911A2A32
:10F27000052F10E087E191E0089FF001099FF00D54
:10F28000189FF00D1124E751F04D8789882309F468
:10F29000F8C08389882309F4F0C08091A12A8F3FA8
:10F2A00009F0EBC080913E21682F70E0FB01EE5326
:10F2B000F54D8181882309F0E0C01092A0211092C1
:10F2C0009F2184E080939E21E0901B2AF0901C2ACD
:10F2D00020E030E044E0FB01BC9611C0DC01A65602
:10F2E000B54D11969C911197992309F4C0C08C914A
:10F2F000813009F49D01990F990F990F490FCF01A2
:10F30000840F911D8E159F0548F320939F21309304
:10F31000A02140939E212115310509F493C08091CD
:10F32000A22A9091A32A892B59F58091A42A909121
:10F33000A52A892B29F58091A62A9091A72A892BA5
:10F34000F9F48091A82A9091A92A892BC9F4809177
:10F35000AA2A9091AB2A892B99F48091AC2A90919A
:10F36000AD2A892B69F48091AE2A9091AF2A892B1E
:10F3700039F48091B02A9091B12A892B09F47DC08B
:10F38000F80183E0EE0FFF1F8A95E1F7E00FF11F10
:10F39000ED5DF54DB084513049F4F9018181813042
:10F3A00019F008E0B02E02C012E0B12E2E5F3F4FE0
:10F3B0008E010F5F1F4FC801B9014B2D50E00E9415
:10F3C0002FB0B98682EA9AE20E94807F7C019093F6
:10F3D000AC218093AB21009749F482EA9AE2B8010C
:10F3E00040E022E030E00E94E57F2CC000919F21A8
:10F3F0001091A0210E5F1F4FB0E1CB2ED12CC80E73
:10F40000D91EC801B6014B2D50E00E9422B00097D2
:10F4100021F4F701808DB81661F0C601B8014B2DBB
:10F4200050E00E942FB0E091AB21F091AC21B08E62
:10F4300005C0F701828D938D892B21F482E090E045
:10F44000938F828F10921C2A10921B2ADE011A962B
:10F45000E2EAFAE280E101900D928150E1F780E06A
:10F4600090E0BE01665F7F4F0E94575D0AC03093F7
:10F47000A02120939F2140939E2110921C2A10923C
:10F480001B2A69960FB6F894DEBF0FBECDBFCF9191
:10F49000DF911F910F91FF90EF90DF90CF90BF9081
:10F4A000089520911A2A30E040E0ABE0B0E086E118
:10F4B00090E0289FB001299F700D389F700D112496
:10F4C0000FC0842F90E08A9FF0018B9FF00D9A9FD0
:10F4D000F00D1124E60FF71FEC53FB4D12864F5F22
:10F4E000423078F340930026089590E028E831E018
:10F4F000A901849F9001859F300D949F300D1124A8
:10F500002C543E4DC9010895CF93DF93DC01109236
:10F510000626109205261092002650911A2A252FB1
:10F5200030E040E0CBE0D0E086E190E0289FB00101
:10F53000299F700D389F700D112429C0842F90E0F1
:10F540008C9FF0018D9FF00D9C9FF00D1124E60F14
:10F55000F71FEC53FB4D82858823C1F08081918198
:10F560008A179B0799F4409300268BE0489FC001BF
:10F57000112426E1529F90011124820F931F8C5376
:10F580009B4D909306268093052605C04F5F423021
:10F59000A8F2409300268091052690910626DF91DF
:10F5A000CF9108950F931F93CF93DF931092062668
:10F5B000109205261092002690911A2A292F30E0E9
:10F5C00086E1989FD001112440E050E060E00BE01C
:10F5D00010E086E190E0289FE001299FD00D389F40
:10F5E000D00D11242BE036C0862F90E0809FF001D3
:10F5F000819FF00D909FF00D1124EC0FFD1FEC5337
:10F60000FB4D8285882329F10190F081E02D309710
:10F6100001F1828D938D009711F0059759F44115F2
:10F620005105B9F4629FA00111244A0F5B1F4C538E
:10F630005B4D0FC0609300268BE0689FC0011124D2
:10F640008A0F9B1F8C539B4D909306268093052613
:10F6500009C06F5F623040F2509306264093052642
:10F66000609300268091052690910626DF91CF9128
:10F670001F910F910895FC0112860190F081E02DF9
:10F68000828D938D059709F415A60895FC0181A13B
:10F690008D7F81A3089520911A2A88E8289F9001E0
:10F6A000112420513B4DC90108957F928F929F9262
:10F6B000AF92BF92CF92DF92EF92FF920F931F9380
:10F6C000CF93DF9390911A2AA92FB0E086E1989FFB
:10F6D000E001112420E030E040E00BE010E086E1A2
:10F6E00090E0A89FB001A99F700DB89F700D1124E4
:10F6F0005BE018C0842F90E0809FF001819FF00DA7
:10F70000909FF00D1124E60FF71FEC53FB4D8285FF
:10F71000813039F4459F900111242C0F3D1F2C534B
:10F720003B4D4F5F423030F3309306262093052641
:10F7300040930026109204261092032687E191E060
:10F74000A89FF001A99FF00DB89FF00D1124E7517B
:10F75000F04D8789882309F4DCC01092002611E35C
:10F76000812E912CB8E8AB2EB1E0BB2EA1E37A2E0E
:10F77000F2E0CF2ED12CC7E1D1E0E4E0EE2EF12C67
:10F78000C3C080911A2A90E0242F30E0289DD00138
:10F79000299DB00D389DB00D11248A9D90018B9D3F
:10F7A000300D9A9D300D1124A20FB31FAC54BE4DE5
:10F7B0009D968C919D97813009F0A1C0479DF001E5
:10F7C0001124E20FF31FEC54FE4DF0930426E09356
:10F7D0000326828D938D8130910501F18130910551
:10F7E00038F08330910549F1049709F088C034C09E
:10F7F00084A5833018F09D961C9281C0CF01849619
:10F800000E941782892B09F47AC0409103265091F7
:10F81000042680E090E060E070E048C0CF014C96A4
:10F820000E941782892B09F46AC0E0910326F091A7
:10F830000426D38EC28E14A662C0CF014C960E94BD
:10F840001782892B09F45BC0E0910326F09104260E
:10F85000F38EE28E14A623C084A58330D0F014A6C4
:10F86000CF010E94847AFC0190930626809305269E
:10F87000009749F012860190F081E02D828D938DE2
:10F88000059709F415A6E0910326F091042615A624
:10F8900036C0CF0184960E941782892B81F1409156
:10F8A00003265091042680E090E0BA010E94067180
:10F8B000009103261091042680911A2A90E08C9FD3
:10F8C000F0018D9FF00D9C9FF00D1124E751F04D3C
:10F8D000658576858785908928EE33E040E050E0A5
:10F8E0000E94C5ACAB01BC01C80184960E94408255
:10F8F000E0910326F091042684A58F5F84A7809170
:10F9000000268F5F8093002640910026483008F43F
:10F9100038CF109202261092012681E080930026B3
:10F92000C8E8D0E002E218E841C050911A2A252F19
:10F9300030E0842F90E0FC0175E0EE0FFF1F7A9518
:10F94000E1F7880F991FE80FF91F2C9FC0012D9F29
:10F95000900D3C9F900D1124E80FF91FEF5EFA4DBA
:10F96000808181FF1EC0409FF0011124519FC00182
:10F970001124E80FF91FE051FB4DF0930226E093AC
:10F98000012681A180FD0DC0CF0141960E94178202
:10F99000892B39F0E0910126F091022681A18D7F1B
:10F9A00081A3809100268F5F8093002640910026DE
:10F9B000443008F4BACFDF91CF911F910F91FF909F
:10F9C000EF90DF90CF90BF90AF909F908F907F90FF
:10F9D0000895AF92BF92CF92DF92EF92FF920F9372
:10F9E0001F93CF93DF93182FB92EA62E69017A01AA
:10F9F000109202261092012681E0809300268091C9
:10FA00001A2A90E041E028E830E0829FB001839F0D
:10FA1000700D929F700D112419C0242F2F5F842F19
:10FA200090E0FC0135E0EE0FFF1F3A95E1F7880FFB
:10FA3000991FE80FF91FE60FF71FEF5EFA4D80815F
:10FA400081FD03C04093002610C0422F443028F3AC
:10FA500040930026443049F40E94DFAE63E070E03A
:10FA60000E94F8AC8F5F809300269091002682E27E
:10FA7000989FF001112480911A2A28E8829FC001E2
:10FA80001124E80FF91FE051FB4DF0930226E0939B
:10FA90000126EF01212F3B2DC901DC0180E10D90F2
:10FAA00009928150E1F7A08AC114D104E104F10464
:10FAB00069F0CF014196B701A6010E944082E09112
:10FAC0000126F091022681A18E7F02C081A1816072
:10FAD00081A320911A2A30E060910026862F90E0C1
:10FAE000FC01A5E0EE0FFF1FAA95E1F7880F991F13
:10FAF000E80FF91F88E890E0289FA001299F500D8A
:10FB0000389F500D1124E40FF51FEF5EFA4D8081F0
:10FB10008260808300FF13C0862F90E0FC0165E0C7
:10FB2000EE0FFF1F6A95E1F7880F991FE80FF91F85
:10FB3000E40FF51FEF5EFA4D8081846012C0862FBE
:10FB400090E0FC0125E0EE0FFF1F2A95E1F7880FFA
:10FB5000991FE80FF91FE40FF51FEF5EFA4D808142
:10FB60008B7F80838091012690910226DF91CF9137
:10FB70001F910F91FF90EF90DF90CF90BF90AF90CB
:10FB80000895EF92FF920F931F93CF93DF93EC01B1
:10FB90007A018B01109206261092052610920026FB
:10FBA00020911A2A30E040E0ABE0B0E086E190E03E
:10FBB000289FB001299F700D389F700D112416C029
:10FBC000242F2F5F842F90E08A9FF0018B9FF00DF0
:10FBD0009A9FF00D1124E60FF71FEC53FB4D828521
:10FBE000882319F4409300260FC0422F423040F37F
:10FBF00040930026423041F40E94DFAE62E070E0A4
:10FC00000E94F8AC80930026E09100268BE0E89FEC
:10FC1000F001112480911A2A26E1829FC00111244B
:10FC2000E80FF91FEC53FB4DF0930626E0930526F1
:10FC3000C193D193CF01B801A7010E9440822091C6
:10FC4000002630E040911A2A50E08BE090E0289F97
:10FC5000F001299FF00D389FF00D112486E190E00E
:10FC60009C01429FC001439F900D529F900D112413
:10FC7000E80FF91FEC53FB4D81E082878091052648
:10FC800090910626DF91CF911F910F91FF90EF90F9
:10FC90000895EF92FF920F931F93CF93DF937C0110
:10FCA00010920226109201261092002600911A2A24
:10FCB000202F30E088E890E0289FE001299FD00DB8
:10FCC000389FD00D11243EC0812F90E0FC0175E0DB
:10FCD000EE0FFF1F7A95E1F7880F991FE80FF91FC4
:10FCE000EC0FFD1FEF5EFA4D808181FF28C0212FB0
:10FCF00030E0C90155E0880F991F5A95E1F7220FAE
:10FD0000331F820F931F8C0F9D1F80519B4DB70196
:10FD100040E150E00E9422B0009789F482E2189FEF
:10FD2000C001112428E8029F90011124820F931F23
:10FD300080519B4D909302268093012608C01F5F3F
:10FD40001093002610910026143008F4BDCF809146
:10FD5000012690910226DF91CF911F910F91FF9084
:10FD6000EF900895EF92FF921F93CF93DF937C0162
:10FD70001092002680911A2A90E028E830E0829FB5
:10FD8000E001839FD00D929FD00D112442C0812F9E
:10FD900090E0FC0175E0EE0FFF1F7A95E1F7880F08
:10FDA000991FE80FF91FEC0FFD1FEF5EFA4D8081E0
:10FDB00081FF2CC0212F30E0C90155E0880F991F29
:10FDC0005A95E1F7220F331F820F931F8C0F9D1F4F
:10FDD000212F30E0F901B5E0EE0FFF1FBA95E1F7F2
:10FDE000220F331FE20FF31FEC0FFD1FE051FB4DFD
:10FDF000408946954695469580519B4DB70150E008
:10FE00000E9422B0009711F481E009C01F5F109397
:10FE1000002610910026143008F4B9CF80E0DF915D
:10FE2000CF911F91FF90EF900895CF92DF92EF92C4
:10FE3000FF920F931F93CF93DF93EC011092042650
:10FE4000109203261092002600911A2A202F30E0EB
:10FE5000E1E3CE2ED12C88E891E0289F7001299F04
:10FE6000F00C389FF00C11243AC0812F90E08C9D4B
:10FE700090018D9D300D9C9D300D11242E0D3F1D48
:10FE8000F901EC54FE4D85A5882331F1408D88851C
:10FE9000481711F5C9018C539E4DBE0150E00E94D8
:10FEA00022B00097C9F481E3189FC0011124402FAC
:10FEB00050E028E831E0B901469F9001479F300D9E
:10FEC000569F300D1124820F931F8C549E4D90939A
:10FED00004268093032607C01F5F1093002610910D
:10FEE0000026183010F28091032690910426DF91AD
:10FEF000CF911F910F91FF90EF90DF90CF900895D9
:10FF0000CF92DF92EF92FF920F931F93CF93DF93E5
:10FF10007C01109204261092032610920026009174
:10FF20001A2A202F30E0F1E3CF2ED12C88E891E07F
:10FF3000289FE001299FD00D389FD00D112434C097
:10FF4000812F90E08C9DF0018D9DF00D9C9DF00D1A
:10FF50001124EC0FFD1FEC54FE4D85A5882309F1FB
:10FF6000CF01B70140E150E00E9422B00097C9F4F0
:10FF700081E3189FC0011124402F50E028E831E0B0
:10FF8000B901469F9001479F300D569F300D1124B7
:10FF9000820F931F8C549E4D9093042680930326CA
:10FFA00007C01F5F1093002610910026183040F202
:10FFB0008091032690910426DF91CF911F910F919C
:10FFC000FF90EF90DF90CF900895BF92CF92DF9295
:10FFD000EF92FF920F931F93CF93DF93D82EC92EEA
:10FFE0008B01B42E790110920426109203261092F0
:10FFF000002620911A2A30E040E0A1E3B0E088E832
:020000021000EC
:1000000091E0289FB001299F700D389F700D112439
:1000100016C0242F2F5F842F90E08A9FF0018B9FC2
:10002000F00D9A9FF00D1124E60FF71FEC54FE4DD2
:1000300085A5882319F4409300260FC0422F48302D
:1000400040F340930026483041F40E94DFAE68E060
:1000500070E00E94F8AC8093002640911A2A90919B
:10006000002681E3989FE0011124242F30E088E8E6
:1000700091E0BC01269FC001279F900D369F900DF7
:100080001124C80FD91FCC54DE4DD0930426C09341
:100090000326DE012D2D3C2DC901FC0180E10190DC
:1000A0000D928150E1F701151105C9F0109200265B
:1000B000E0E00AC0F0E0DE01AE0FBF1FE00FF11F6D
:1000C000808150968C93E92FD80118968C919E2FA1
:1000D0009F5FE81778F3E0930026888F1BC0842F7A
:1000E00090E0FC01A3E0EE0FFF1FAA95E1F7E80FF7
:1000F000F91FED5DF54D40859E01205F3F4FC90121
:1001000060E070E050E00E944AB0E0910326F09178
:100110000426108EE0910326F0910426B18EF38E12
:10012000E28ECF014C9640E050E060E070E00E942B
:1001300040828091032690910426849640E050E00E
:1001400060E070E00E944082E0910326F091042676
:1001500014A681E085A7CF01DF91CF911F910F9168
:10016000FF90EF90DF90CF90BF9008951F93109174
:100170001A2A412F50E020E0A1E3B0E088E891E0A6
:10018000489FB001499F700D589F700D11240FC0FA
:10019000822F90E08A9FF0018B9FF00D9A9FF00DC7
:1001A0001124E60FF71FEC54FE4D15A62F5F2830E3
:1001B00078F320E0ABE0B0E086E190E0489FB0014A
:1001C000499F700D589F700D11240FC0822F90E031
:1001D0008A9FF0018B9FF00D9A9FF00D1124E60F7E
:1001E000F71FEC53FB4D12862F5F223078F320E08F
:1001F00088E890E0489FB001499F700D589F700DAE
:10020000112414C0822F90E0FC01A5E0EE0FFF1F27
:10021000AA95E1F7880F991FE80FF91FE60FF71F5E
:10022000EF5EFA4D80818D7F80832F5F243050F305
:100230002093002687E191E0489FF001499FF00D4F
:10024000589FF00D1124E751F04D8589882309F45A
:1002500064C088E890E0489F9001499F300D589F06
:10026000300D1124D901A051BB4D8EEF90E81196AD
:100270009C938E9384E490E0489FF001499FF00D99
:10028000589FF00D1124EE0FFF1FEE50FB4D118211
:100290001082FA01EE0FFF1FCA0175E0880F991F47
:1002A0007A95E1F7E80FF91FEE0FFF1FEE0FFF1F22
:1002B000EC50FB4D1182108217961C921E921697DD
:1002C000FA0194E0EE0FFF1F9A95E1F7E40FF51F96
:1002D00083E0EE0FFF1F8A95E1F7E850FB4D118296
:1002E00010821B961C921E921A971D961C921E92AB
:1002F0001C971F961C921E921E9780E450968C931A
:100300002F5E3A4DF901808183608083812F40EA1E
:1003100056E861E070E00E9401841F910895FFCFCC
:100320000895CF92DF92EF92FF920F931F93DF9386
:10033000CF93CDB7DEB729970FB6F894DEBF0FBEC7
:10034000CDBF8C0180911A2A882339F5011511053A
:10035000A1F483E389838A838091BE2A8B83809171
:10036000BF2A8C838091C02A8D838091C12A8E837D
:1003700086E089878E010F5F1F4FE0901B2AF09067
:100380001C2A80E060E040E050E026E09AE9C92EB7
:100390009AE2D92E0E94628A10C0813091F4011530
:1003A000110541F48FEF89838A8382E089878E016A
:1003B0000F5F1F4FC8010E94574A10921C2A1092CB
:1003C0001B2A80E090E029960FB6F894DEBF0FBE9E
:1003D000CDBFCF91DF911F910F91FF90EF90DF90F4
:1003E000CF9008950F931F93DF93CF9300D000D049
:1003F000CDB7DEB78C01CE0101960E94DA0DF8016F
:10040000208131814281538189819A81AB81BC8174
:10041000281B390B4A0B5B0BB901CA010F900F90D7
:100420000F900F90CF91DF911F910F9108950F932F
:100430001F93DF93CF9300D000D0CDB7DEB78C01F0
:10044000CE0101960E94DA0D60E070E0F801208193
:1004500031814281538189819A81AB81BC81281786
:1004600039074A075B0710F461E070E0CB010F9099
:100470000F900F900F90CF91DF911F910F910895E2
:10048000CF92DF92EF92FF920F931F93DF93CF9360
:1004900000D000D0CDB7DEB76C017A018B01CE0160
:1004A00001960E94DA0DF601E482F5820683178335
:1004B00089819A81AB81BC818E0D9F1DA01FB11FC8
:1004C00080839183A283B3830F900F900F900F903E
:1004D000CF91DF911F910F91FF90EF90DF90CF9020
:1004E0000895882321F48DE00E94180F089581302B
:1004F00019F48CE00E94180F0895882321F489E0F4
:100500000E94180F0895813019F488E00E94180F96
:10051000089584E00E94180F85E00E94180F86E07D
:100520000E94180F87E00E94180F88E00E94180FA1
:1005300089E00E94180F8AE00E94180F8BE00E9449
:10054000180F8CE00E94180F8DE00E94180F8EE0AB
:100550000E94180F8FE00E94180F80E10E94180F70
:1005600081E10E94180F0895AF92BF92CF92DF925F
:10057000EF92FF920F931F935A016B01813031F478
:1005800080E120E030E00AEB14E805C081E120E0E2
:1005900030E003EB14E8EE24FF240E9424108823AB
:1005A000B9F0A114B104C104D10491F000D000D07D
:1005B0008BE398E0EDB7FEB7928381838EEE91E0F6
:1005C000948383830E9430B10F900F900F900F900F
:1005D0001F910F91FF90EF90DF90CF90BF90AF9061
:1005E0000895AF92BF92CF92DF92EF92FF920F9356
:1005F0001F935A016B01813031F48EE020E030E02E
:1006000009EC14E805C08FE020E030E002EC14E8CB
:10061000EE24FF240E9424108823B9F0A114B10411
:10062000C104D10491F000D000D08BE398E0EDB785
:10063000FEB79283818388ED91E0948383830E9447
:1006400030B10F900F900F900F901F910F91FF906E
:10065000EF90DF90CF90BF90AF900895AF92BF9290
:10066000CF92DF92EF92FF920F931F935A016B018B
:10067000813031F48CE020E030E008ED14E805C072
:100680008DE020E030E001ED14E8EE24FF240E942C
:1006900024108823B9F0A114B104C104D10491F04D
:1006A00000D000D08BE398E0EDB7FEB79283818352
:1006B00081EC91E0948383830E9430B10F900F907E
:1006C0000F900F901F910F91FF90EF90DF90CF90C0
:1006D000BF90AF900895AF92BF92CF92DF92EF920A
:1006E000FF920F931F93282F5A016B01E82FF0E020
:1006F000411551056105710551F4EE0FFF1FE95FCA
:10070000F94D808191815C01CC24DD2406C0EE0F7F
:10071000FF1FE95FF94D51834083213041F48AE0A6
:10072000B601A50120E030E00EEE14E807C08BE032
:10073000B601A50120E030E000EE14E8EE24FF242D
:100740000E9424108823B9F0A114B104C104D1047B
:1007500091F000D000D08BE398E0EDB7FEB7928324
:1007600081838AEA91E0948383830E9430B10F9061
:100770000F900F900F901F910F91FF90EF90DF90CF
:10078000CF90BF90AF900895AF92BF92CF92DF927B
:10079000EF92FF920F931F935A016B01813031F456
:1007A00088E020E030E003E015E805C089E020E0C3
:1007B00030E00CEF14E8EE24FF240E94241088237C
:1007C000B9F0A114B104C104D10491F000D000D05B
:1007D0008BE398E0EDB7FEB7928381838DE891E0DB
:1007E000948383830E9430B10F900F900F900F90ED
:1007F0001F910F91FF90EF90DF90CF90BF90AF903F
:100800000895AF92BF92CF92DF92EF92FF920F9333
:100810001F93282F5A016B01E82FF0E04115510575
:100820006105710551F4EE0FFF1FE55FF94D808101
:1008300091815C01CC24DD2406C0EE0FFF1FE55F33
:10084000F94DB182A082213041F486E0B601A501C4
:1008500020E030E009E115E807C087E0B601A50116
:1008600020E030E00BE015E8EE24FF240E94241085
:100870008823B9F0A114B104C104D10491F000D0CF
:1008800000D08BE398E0EDB7FEB79283818387E7D2
:1008900091E0948383830E9430B10F900F900F906A
:1008A0000F901F910F91FF90EF90DF90CF90BF902E
:1008B000AF900895AF92BF92CF92DF92EF92FF92E6
:1008C0000F931F93282F5A016B01E82FF0E0411579
:1008D00051056105710551F4EE0FFF1FE15FF94D00
:1008E000808191815C01CC24DD2406C0EE0FFF1FC6
:1008F000E15FF94DB182A082213041F484E0B6017C
:10090000A50120E030E005E315E807C085E0B60169
:10091000A50120E030E007E215E8EE24FF240E9464
:1009200024108823B9F0A114B104C104D10491F0BA
:1009300000D000D08BE398E0EDB7FEB792838183BF
:100940008AE591E0948383830E9430B10F900F90E9
:100950000F900F901F910F91FF90EF90DF90CF902D
:10096000BF90AF90089510921A2A0E94BD5C0E9419
:10097000DE64089581E080931A2A0E94BD5C0E9483
:10098000DE64089510921A2A0E94B45D0E94DE640B
:10099000089581E080931A2A0E94B45D0E94DE646B
:1009A000089510921A2A0E94395E0E94DE6408950A
:1009B00081E080931A2A0E94395E0E94DE640895C5
:1009C00010921A2A80E040E050E060E070E00E945F
:1009D0006B830E9444620E94DE64089581E08093EC
:1009E0001A2A40E050E060E070E00E946B830E94B1
:1009F00044620E94DE64089510921A2A0E947B5F6E
:100A00000E94DE64089581E080931A2A0E947B5F31
:100A10000E94DE64089510921A2A80E040E050E0BF
:100A200060E070E00E9401840E94557B0E94DE64B9
:100A3000089581E080931A2A40E050E060E070E081
:100A40000E9401840E94557B0E94DE6408951092EA
:100A50001A2A80E040E050E060E070E00E945A8492
:100A60000E9400680E94DE64089581E080931A2A43
:100A700040E050E060E070E00E945A840E9400680C
:100A80000E94DE6408950F931F93DF93CF93CDB739
:100A9000DEB762970FB6F894DEBF0FBECDBF9A8B5C
:100AA000898BFB0181E080931A2A8A89809317320F
:100AB00089898093183282E08093342A80818093E0
:100AC0002C2A818180932D2A8EEF90E89A83898346
:100AD0001C821B821E821D8218861F821A8619861E
:100AE0001C861B861E861D86188A1F86CE010196CF
:100AF00060E420E030E040E050E001E010E00E94DF
:100B0000596162960FB6F894DEBF0FBECDBFCF918C
:100B1000DF911F910F910895CF92DF92EF92FF9294
:100B20000F93DF93CF93CDB7DEB729970FB6F89425
:100B3000DEBF0FBECDBFAC01FE01319689E0DF0103
:100B40001D928A95E9F786E0898710921A2A411545
:100B5000510581F020E030E0BF01FB01E20FF31FFF
:100B6000DA01A20FB31F8C9180832F5F3F4F263095
:100B7000310599F786E0898789E698E00E94BD648F
:100B800068E077E080E090E041E021E000E0B0E55F
:100B9000EB2EB8E0FB2E6E010894C11CD11C0E9404
:100BA000DF5B80E040E251EA67E070E00E945A8437
:100BB00029960FB6F894DEBF0FBECDBFCF91DF915F
:100BC0000F91FF90EF90DF90CF900895CF92DF923A
:100BD000EF92FF920F936C0101E000931A2A80912B
:100BE000640390916503892BC1F489E598E00E9424
:100BF000BD6400931A2A68EE73E080E090E041E063
:100C000021E000E054E5E52E58E0F52E0E94DF5B80
:100C100089E598E00E94B6410DC060E070E080E098
:100C200090E040E021E000E034E5E32E38E0F32EF0
:100C30000E94DF5B81E040E251EA67E070E00E94E1
:100C40005A840F91FF90EF90DF90CF90089583E149
:100C500096E29093172A8093162A0E9489820E9416
:100C6000BA410895FC0120E09081818180839183C5
:100C70002E5F32962031C1F70895992787FD909510
:100C80000E9401B08A3314F0875308958053089569
:100C9000FF920F931F938C01FC0180810E943D867F
:100CA000F82EF29480EFF822F80181810E943D86AF
:100CB0008F0D1F910F91FF900895992787FD9095B3
:100CC0000E94F9AF8833A1F1893384F4843341F170
:100CD00085333CF4823301F1833304F58133D1F45D
:100CE00017C0863309F187330CF51CC0833641F1F8
:100CF00084363CF4813601F1823604F5893351F4AF
:100D000019C0853609F18536ECF0863619F41EC017
:100D100081E0089580E0089582E0089583E00895D9
:100D200084E0089585E0089586E0089587E00895B9
:100D300088E0089589E008958AE008958BE0089599
:100D40008CE008958DE008958EE008958FE0089579
:100D5000EF92FF921F93CF93DF937C01EC0110E0A1
:100D600001C01F5F8881992787FD90950E94E5AF9C
:100D7000892B19F4C0E0D0E022C02196143089F705
:100D8000F9CFF70180810E945D8690E0143029F44C
:100D9000982F88279295907F0CC0133019F4982FC4
:100DA000882707C0123029F424E0880F991F2A955C
:100DB000E1F7C80FD91F11500894E11CF11C112351
:100DC00001F7CE01DF91CF911F91FF90EF90089531
:100DD0005F926F927F928F929F92AF92BF92CF92CB
:100DE000DF92EF92FF920F931F93DF93CF9300D088
:100DF00000D00F92CDB7DEB74C016B018C019C0186
:100E0000A8E0EA2EFF24F8E05F2E5E010894A11C02
:100E1000B11CE5E06E2E712C6C0E7D1E02C00F5FC2
:100E20001F4FF80140814A3311F04423C1F7C80134
:100E3000821B930B059714F080E05EC0F80182914D
:100E40008F010F5F1F4F8A3319F0D501F9012FC0B1
:100E5000442319F0F40190E00EC0EF2DF0E0EE0F06
:100E6000FF1FEC0DFD1D11821082F39440C08A33E8
:100E700009F49F5F319680818823C9F7252D291BAE
:100E8000922F8F2D0AC0E82FF0E0EE0FFF1FEC0D20
:100E9000FD1D1182108291508F5F9923A1F7F20EF0
:100EA000E21A0F5F1F4F98011FC08D9331969E2F3E
:100EB000921B80818A3319F0A615B705B1F7F501A9
:100EC000E90FF11D1082C5010E94A886EF2DF0E008
:100ED000EE0FFF1FEC0DFD1D9183808398012F5FA6
:100EE0003F4FF394EA948901EE2009F09ACF80E015
:100EF000F8E0FF1609F481E00F900F900F900F902B
:100F00000F90CF91DF911F910F91FF90EF90DF90A5
:100F1000CF90BF90AF909F908F907F906F905F9099
:100F20000895AF92BF92CF92DF92EF92FF920F930C
:100F30001F93CF93DF938C01EB016115710509F4C9
:100F40006BC0EE24FF2439E7C32E38E0D32E20E314
:100F5000A22E9AE3B92E88819981009779F5EE2027
:100F600069F540E06F2D70E001C04F5F242F30E045
:100F7000F901EE0FFF1FEC0FFD1F80819181892B7E
:100F800029F4260F371F283031057CF3413039F41E
:100F9000D801AD928D01F394229640E030C08F2DA0
:100FA00090E0840F911D089709F44150842F90E040
:100FB000880F991FC80FD91FF40E21C00E94B65187
:100FC00000D000D000D0EDB7FEB73196ADB7BEB7B8
:100FD00012961C930E931197D382C28295838483B9
:100FE0000E94A1B1080F191F2296F3944E2DEDB760
:100FF000FEB736960FB6F894FEBF0FBEEDBFF8E011
:10100000FF1641F0D801BD928D01B7E0BF1510F079
:10101000E42EA1CFF8011082DF91CF911F910F91A3
:10102000FF90EF90DF90CF90BF90AF900895AF9278
:10103000BF92CF92DF92EF92FF920F931F93DF93B5
:10104000CF9300D000D000D0CDB7DEB77C0100E058
:1010500010E05E010894A11CB11C4CE7C42E48E0CE
:10106000D42E00D000D000D0EDB7FEB73196ADB78A
:10107000BEB71296BC92AE921197D382C282D701AC
:10108000A00FB11F8C91848315820E94A1B10F5FC4
:101090001F4F8DB79EB706960FB6F8949EBF0FBE32
:1010A0008DBF00311105E9F626960FB6F894DEBF24
:1010B0000FBECDBFCF91DF911F910F91FF90EF90A9
:1010C000DF90CF90BF90AF9008951F93CF93DF93A1
:1010D0009C01EB01142F80911B2A90911C2A892BD3
:1010E00019F02FEF3FEF13C08AE99AE2B901AE0180
:1010F0000E9438B010931A2AD0931C2AC0931B2A3E
:1011000081E00E9452520E94DE6420E030E0C9017A
:10111000DF91CF911F910895DC019C9111968C91E4
:1011200011979F5F983728F090E003C06B9A639AFD
:1011300008959817D9F38C91FD01E80FF11D628392
:101140009C930895DC0111969C911197FD01E90F84
:10115000F11D22818C918C91981711F42FEF07C00B
:10116000892F8F5F883708F080E011968C93822F4B
:101170000895FC019081818120E0981321E0822F65
:101180000895FC018081282F30E08181281B3109DE
:1011900037FF02C028583F4F822F089510920B3816
:1011A00080910B3880930A38109285388091853869
:1011B0008093843888E98093C10086E08093C200E0
:1011C0001092C50083E08093C400109224270895F4
:1011D0001092C1000895682F789484E898E30E94E3
:1011E0008C888091C10085FD21C08091C00085FF61
:1011F000FCCF90918538E92FF0E0EC57F74C228135
:101200008091843880918438981711F42FEF07C0AB
:10121000E92FEF5FE83708F0E0E0E09385382093AE
:10122000C6008091C10080628093C1000895833A16
:1012300029F0843A41F08B3179F40AC08BE10E94A5
:10124000EB8881E009C08BE10E94EB8882E004C05A
:101250008BE10E94EB8883E00E94EB880895EF9277
:10126000FF921F93CF93DF93182FEB017A0183EA4C
:101270000E94EB888C2F0E9417898D2F0E9417895E
:10128000812F0E94178906C0F70181917F010E947A
:10129000178921972097C1F784EA0E94EB88DF9194
:1012A000CF911F91FF90EF900895CF93DF93EC01C2
:1012B00003C00E94EB88219688818823D1F7DF91B3
:1012C000CF91089580910A38282F30E080910B3813
:1012D000281B310937FF02C028583F4F822F08953D
:1012E00080910A38282F30E080910B38281B310973
:1012F00037FF02C028583F4F822F089580918438CD
:10130000282F30E080918538281B310937FF02C033
:1013100028583F4F822F089590918538E92FF0E0AB
:10132000EC57F74C2281809184388091843898174B
:1013300011F42FEF07C0E92FEF5FE83708F0E0E086
:10134000E0938538822F0895789480910A38282F69
:1013500030E080910B38281B310937FF02C0285834
:101360003F4F222391F390910B38E92FF0E0E65F95
:10137000F74C228180910A3880910A38981711F42D
:101380002FEF07C0E92FEF5FE83708F0E0E0E093C8
:101390000B38822F0895682F8AE098E30E948C888A
:1013A0001092972608951F920F920FB60F920BB6C8
:1013B0000F9211242F933F934F935F936F937F93DB
:1013C0008F939F93AF93BF93EF93FF936091C6006A
:1013D0008AE098E30E948C8810929726FF91EF9103
:1013E000BF91AF919F918F917F916F915F914F913D
:1013F0003F912F910F900BBE0F900FBE0F901F903B
:1014000018951F920F920FB60F920BB60F921124E0
:101410002F938F939F93EF93FF93909184388091B4
:1014200085389817C9F090918538E92FF0E0EC578E
:10143000F74C22818091843880918438981711F478
:101440002FEF07C0E92FEF5FE83708F0E0E0E09307
:1014500085382093C60005C08091C1008F7D8093A0
:10146000C100FF91EF919F918F912F910F900BBE33
:101470000F900FBE0F901F901895DF93CF93CDB7AD
:10148000DEB767970FB6F894DEBF0FBECDBF8E30C4
:1014900008F080E08983CE01029646E150E00E9488
:1014A0006FB08BE367E170E0AE014F5F5F4F0E946A
:1014B0002F8967960FB6F894DEBF0FBECDBFCF91D0
:1014C000DF9108952F923F924F925F926F927F9299
:1014D0008F929F92AF92BF92CF92DF92EF92FF9244
:1014E0000F931F93DF93CF93CDB7DEB7AA970FB6B5
:1014F000F894DEBF0FBECDBF8AA7662E1A01722EEA
:10150000480156018091FE149091FF14009709F054
:101510005CC0680110E081E8482E88E0582E1DC0AC
:10152000112321F08AE390E00E9465B100D000D041
:10153000EDB7FEB73196ADB7BEB712965C924E923C
:101540001197D6018D916D01828313820E9430B173
:101550001F5F0F900F900F900F90171508F38E01DB
:101560000E5F1F4FB501685F7F4FC8010E949187D2
:1015700000D000D084E898E0EDB7FEB79283818375
:10158000148303830E9430B10F900F900F900F903F
:10159000B501685E7F4FC8010E94918700D000D0DE
:1015A00085E998E0ADB7BEB712969C938E931197DC
:1015B00014961C930E9313970E9430B10F900F90C6
:1015C0000F900F9088E998E004C0029720F48AE910
:1015D00098E00E946CB1062D10E00B5F1F4F070DC5
:1015E000111D0E0D1F1D83EA0E94EB88802F0E94A3
:1015F0001789812F0E94178986E30E9417898AA57F
:101600000E941789862D0E941789872D0E941789AD
:101610008E2D0E9417898F2D0E94178906C0F10117
:1016200081911F010E9417896A946620C1F706C044
:10163000D4018D914D010E9417897A947720C1F7CA
:1016400012C0F50180810E941789198203C0898127
:101650008F5F89838981883CD0F30894A11CB11CD9
:101660000894E108F108E114F10459F784EA0E94B2
:10167000EB88AA960FB6F894DEBF0FBECDBFCF9110
:10168000DF911F910F91FF90EF90DF90CF90BF906F
:10169000AF909F908F907F906F905F904F903F9012
:1016A0002F9008954F925F926F927F928F929F92A8
:1016B000AF92BF92CF92DF92EF92FF920F931F9360
:1016C000CF93DF9363E0462E512C55E0E52EF12CAD
:1016D00044E0642E712C31E0832E912C2AE9A22E55
:1016E00026E2B22E92E0C92ED12C01E0DDC00E948C
:1016F000A489182F833A99F410929626109299266D
:101700001092982680919D2690919E26009761F0D8
:101710000E942CAE10929E2610929D2605C08B3101
:1017200019F400939626C0C0809196268823F9F07C
:10173000123029F0133039F0113039F402C014EAB4
:1017400014C013EA12C01BE110C080919D26909135
:101750009E26009731F00E942CAE10929E26109289
:101760009D26109299261092982610929626809186
:101770009826909199268230910531F18330910518
:1017800030F4009781F0019709F08EC014C08430C6
:10179000910509F453C08430910508F444C00597BD
:1017A00009F082C064C0133A09F07EC09092992675
:1017B0008092982679C010939A26F5011182D092D2
:1017C0009926C092982670C0D12FC0E080919A26A9
:1017D00090919B268C0F9D1F90939B2680939A2619
:1017E000509299264092982690939526809394261D
:1017F0001092932610929226009761F00E947FAD7E
:101800009093932680939226009721F41092992624
:1018100010929826809192269091932690939E26DE
:1018200080939D2641C010939C26709299266092C9
:10183000982680919A2690919B2612C0E09192263C
:10184000F09193261193F0939326E0939226809142
:1018500094269091952601979093952680939426AF
:10186000892B11F5F0929926E09298261DC0143A22
:1018700069F460919A2670919B2640919D26509123
:101880009E2680919C260E948C3B06C080919D26BE
:1018900090919E260E942CAE109299261092982626
:1018A00010929E2610929D2690910A3880910B38B6
:1018B000981709F01CCFDF91CF911F910F91FF90E6
:1018C000EF90DF90CF90BF90AF909F908F907F90E0
:1018D0006F905F904F900895E82FF0E0EE0FFF1F9C
:1018E000EE0FFF1FE250F74C20813181428153817E
:1018F000B901CA010895509A589A5898589A589818
:10190000589A5898589A5898589A509A519859985D
:1019100084E090E00E94100E84E090E00E94100E9F
:10192000519A84E090E00E94100E589884E090E074
:101930000E94100E589A5898589A58985198519A4F
:101940005198519A5198589A84E090E00E94100E54
:10195000519A84E090E00E94100E08950F931F9317
:10196000082F10E007FF02C0519801C0519A589A01
:1019700084E090E00E94100E589884E090E00E946D
:10198000100E1F5F183011F0000FECCF51981F910F
:101990000F9108950F931F93082F84E090E00E9409
:1019A000100E519A84E090E00E94100E589884E046
:1019B00090E00E94100E82E70E94AE8C589A84E05C
:1019C00090E00E94100E19B1589884E090E00E94B7
:1019D000100E11FD19C0802F0E94AE8C589A84E021
:1019E00090E00E94100E89B1589884E090E00E9427
:1019F000100E5198589A84E090E00E94100E519A6F
:101A000084E090E00E94100E1F910F9108950F93B3
:101A10001F9300E010E0110F589A84E090E00E94BC
:101A2000100E49991160589884E090E00E94100EC1
:101A30000F5F083081F7812F1F910F9108951F9339
:101A400084E090E00E94100E519A84E090E00E94A1
:101A5000100E589884E090E00E94100E83E70E94D8
:101A6000AE8C589A84E090E00E94100E19B15898FC
:101A700084E090E00E94100E11FF02C010E01AC036
:101A800080E00E94078D182F519A589A84E090E0C8
:101A90000E94100E589884E090E00E94100E519819
:101AA000589A84E090E00E94100E519A84E090E0F1
:101AB0000E94100E812F1F9108951F93182F8130BF
:101AC00089F1813040F0823009F455C0A0E070E027
:101AD00080E060E093C080E480937C0086E880939F
:101AE0007A0080917A00806580937A0080917A00F4
:101AF00084FFFCCF80917A00806180937A006091AE
:101B000078007091790080E090E00E94A7A620E321
:101B10003EE941E85DE30E9429A52FE135E84FE465
:101B200051E426C081E480937C0086E880937A00AB
:101B300080917A00806580937A0080917A0084FF9A
:101B4000FCCF80917A00806180937A006091780068
:101B50007091790080E090E00E94A7A623E534EE22
:101B600043EB5DE30E9429A520E030E048EC51E41E
:101B70000E94CBA441C0589A509A5198599884E039
:101B800090E00E94100E83E00E94CA8C88E10E94BF
:101B9000CA8C83E40E94CA8C0E941F8D90E0AC0125
:101BA0004F77507034E0569547953A95E1F721E02C
:101BB00030E002C0220F331F4A95E2F741E2249F32
:101BC000A001112430E08F709070289FB001299FF0
:101BD000700D389F700D11246150704056954795D7
:101BE000640F751F80E090E00E94A7A624E13EEA02
:101BF00047EC5EE30E9429A5A62F692FE12FF0E0B4
:101C0000EE0FFF1FEE0FFF1FE250F74C2A2F372F6A
